:100000000C9447120C9466120C9466120C946612AF
:100010000C9466120C945E140C94F4150C946612F5
:100020000C9466120C94CE1A0C9466120C94661200
:100030000C9466120C9466120C94E22F0C946612C7
:100040000C9466120C948E170C9405170C942214C1
:100050000C9466120C9487230C9466120C9466120E
:100060000C9466120C9466120C9466120C94661230
:100070000C9466120C94292F0C948D160C94B315C5
:100080000C9466120C9422800C946612322E312E3F
:100090003100696E636F6D70617469626C652048D0
:1000A000570020202530325800204D430045617311
:1000B00079436F6E74726F6C005F03AF01D7006B92
:1000C00000470035001A001100010203171804054B
:1000D00006151107080916120A000B0C13100F0E53
:1000E0000D14040E1F0E0E0E0E000E0E0E0E1F0E21
:1000F0000400040E1F001F0E04000004040400107E
:10010000081300100B1300130B1300010219000158
:100110001A1900191A19080C1E1F1E0C08000206D5
:100120000F1F0F0602000E11111F1B1B1F001F0ABD
:100130000A0A0A0A1F001C101810160505050C17DC
:10014000141714170C00040A110A0A0E00001C10E0
:100150001812160202071C101816110204071C10B0
:100160001816110201061C101815150701010000D0
:1001700000171515151712121212120000000000B8
:1001800000171117141717111311170000000000A2
:100190000015151711111714171117000000070586
:1001A00005050505050707070707070707070305EF
:1001B00009121418100003070F1E1C181000000667
:1001C00009121412090600060917170906001F1163
:1001D0001F001F111F001F111F001F1F1F001F1FC7
:1001E0001F001F111F001F1F1F001F1F1F00040ED5
:1001F0001F04041F0E04010101050D1F0C0411044E
:100200000A11111F1100110E111111110E000A0017
:10021000111111110E000E11111611111610001CE2
:100220001F1F1F131010001C13111D131010001896
:10023000171119171010001F11111F101010C303F0
:10024000F333CF0FFF3F00C030F00CCC3CFC03C3B6
:1002500033F30FCF3FFFAAC08030F0B020E0A00CF6
:10026000CC8C3CFCBC2CECAC08C88838F8B828E82E
:10027000A803C38333F3B323E3A30FCF8F3FFFBFA1
:100280002FEFAF0BCB8B3BFBBB2BEBAB02C2823216
:10029000F2B222E2A20ECE8E3EFEBE2EEEAE0ACA12
:1002A0008A3AFABA2AEA0040609770486858784457
:1002B0006454744C6C5C7C426252724A6A5A7A464C
:1002C0006656764E6E5E7E41615171496959794537
:1002D000659F754D6D5D7D436353734B6B5B7B47D2
:1002E0006757774F6F5F7F1018141C121A161E1174
:1002F00019151D131B171FD0D8D4DCD2DAD6DED1C6
:10030000D9D5DDD3DBD7DF9098949C929A969E91B5
:1003100099959D939B505504060507C4C6C5C7848F
:1003200086858734363537F4F6F5F7B4B6B5B72495
:10033000262527E4E6E5E7A4A6A5A701C18131F1BA
:10034000B121E1A10DCD8D3DFDBD2DEDAD09C989D9
:1003500039F9B929E9A9206D332020200000204D6A
:100360004D4920200000204D4D0220200000204457
:100370004343202000002053544F50200000534896
:100380004F52542100002048414C542000002020AE
:100390002020202000002050524F472000005245CE
:1003A000534554200000202054504D20000055504B
:1003B00044415445000020202020002533640025BE
:1003C0002D31312E31317300252D35640025632FF9
:1003D00025632025630025630046253032643D25D2
:1003E000630020200102202020202020200025332F
:1003F000640025336400252D3564002D2D2D2D201E
:1004000020004144523A20256C64202020202020E6
:100410002020202000232D007E0E0E0E0E1B1B1C04
:100420000E1B1B7E0E0E0E0E0D5D00435645520038
:100430004D525354004D4658005357555044415463
:1004400045005243520052430054504D004346472A
:10045000535953004346474143430043464744559D
:100460004D50004D415044554D500054524B434C5B
:100470004541520054524B4144440054524B445560
:100480004D50004C4F43434C454152004C4F43416B
:100490004444004C4F4344554D50004C530050547D
:1004A000574C005054524C00505457420050545234
:1004B0004200505457440050545244005054575036
:1004C0000050545250005054575200505452520051
:1004D000504100504400434100435600534F0042F6
:1004E000004040005345005353005352004D540008
:1004F000560059005400464D0046580046004C43F3
:10050000004C0048414C5400474F00210053544FC9
:1005100050002E00484600485400484C0048003F18
:10052000005A7A41004D4320696E2053544F5000C9
:100530004D4320696E2048414C5400696C6C6567DE
:10054000616C207475726E6F75742061647265736E
:1005500073006C6F6B2062757379006E6F20736C23
:100560006F7420617661696C61626C65006E6F20EA
:100570006461746100636F6D6D616E642071756597
:1005800075652066756C6C007475726E6F7574207D
:1005900071756575652066756C6C00706F77657236
:1005A000206973204F666600626164207061726129
:1005B0006D657465722076616C756500756E6B6E25
:1005C0006F776E20636F6D6D616E64004552524FA0
:1005D000523A20005741524E494E473A20002A4590
:1005E0004E442A002564203F0D00322E312E31006A
:1005F000432025642025530D002564002563002534
:10060000642025642025642E25642E25640045522F
:10061000524F52002530386C5800524352202575F5
:10062000202564202575005243202564004D4D008F
:100630004D4D00444343004D4D004D4D002A454E65
:10064000442A0042415544524154452025750D002D
:100650004D41474D415854494D452025640D004DAD
:1006600041474D494E54494D452025640D0073388E
:10067000384D4F44554C45532025640D0053484F89
:10068000525454494D452025640D0044454641557A
:100690004C54444343004E45474154495645534802
:1006A0004F5254004C4F4E475041555345005B53F9
:1006B000595354454D5D0D00444343004D4D0025B5
:1006C000642C20005B414343464D545D0D005B4666
:1006D000554E434D4150535D0D005B5452414B54B8
:1006E000494F4E535D0D005B4C4F434F5D0D005322
:1006F000455249414C20256C750D004D4355204114
:10070000544D6567613132380D00484152445741BC
:10071000524520485725640D00322E312E310056A7
:10072000455253494F4E20005B494E464F5D0D00E8
:1007300025732564002025642C2564002564006E43
:100740006F00796573002C202573004D33004443FE
:1007500043004D4D32004D4D31002C200025642CBE
:10076000202564002A454E442A002A454E442A008A
:100770004D3300444343004D4D32004D4D31002A6E
:10078000454E442A0054696D656F75740042697462
:100790002072656164206572726F72004E6F207006
:1007A000616765004E6F2061636B004E6F2064656A
:1007B000636F6465720053686F72742100427573D1
:1007C0007921004E6F00596573004572726F720097
:1007D0004F6B002564002564203D202425303258CD
:1007E000203D2000504100505800504100416464B9
:1007F00072202575203D20242530345820203D3E90
:10080000202043563137203D2025642028242530E0
:100810003258292C202043563138203D2025642091
:1008200028242530325829004C6F6E6720416464BB
:1008300072203D202575002564002564000D5D00B3
:100840002575003537363030005345202564004D7E
:100850006F64756C65202325642028696E7075743B
:1008600020312E2E38202620392E2E313629203DBB
:1008700020005352202564004D5420256420256417
:10088000000D5365724E722E2025386C7500322E85
:10089000312E31004D43205265766973696F6E20A9
:1008A0000052455345540054504D2070726F67728A
:1008B000616D004443432070726F6772616D005038
:1008C0007772206F6E0048616C7465642100507708
:1008D00072206F66660054202564202563202564FD
:1008E00000464D2025752025752C256400202564A3
:1008F0002C256400464D202575004658202575009E
:100900004620257500444343004D6F746F726F6C31
:1009100061204E6577004D6F746F726F6C61204F70
:100920006C64006D3300756E75736564004C202532
:10093000752025752025632025630000020C151DF8
:10094000263039434C565F69727F0002070C101540
:100950001A1E23282C31363A3F44484D52565B60CC
:1009600064696E73797F0002070B1014191D22262B
:100970002B3035393F43484C51565B5F64696D728B
:10098000767B7F48616C746564210D5D0046207B39
:100990004C6F6B232C205B46315D2C205B46325D17
:1009A0002C205B46335D2C205B46345D2C205B465F
:1009B000355D2C205B46365D2C205B46375D2C2058
:1009C0005B46385D7D0054207B54726E74232C206E
:1009D0005B436F6C6F725D2C205B53746174757335
:1009E0005D7D004C207B4C6F6B232C205B5370652E
:1009F00065645D2C205B464C5D2C205B4469725D18
:100A00002C205B46315D2C205B46325D2C205B4602
:100A1000335D2C205B46345D7D0048542048656C76
:100A20007020666F72207475726E6F757420636FBC
:100A30006D6D616E64730048462048656C70206679
:100A40006F722066756E6374696F6E20636F6D6D73
:100A5000616E64730D00484C2048656C7020666FB1
:100A600072206C6F6B20636F6D6D616E64730D002F
:100A70002530386C75004B75727A2028312E356D13
:100A80007329202000004C616E672028342E3032FC
:100A9000356D732900004D6F746F726F6C610000CB
:100AA00000000000000044434320202020200000DC
:100AB0000000000000004D4D20000000000000007C
:100AC000000000000000444343000000000000005C
:100AD000000000000000706F736974697620284D73
:100AE0004D29000000006E65676174697620284416
:100AF000434329000000303A2061757320202020F4
:100B0000202020202000313A205461696C626974F1
:100B1000732020202000323A202B2049644E6F742D
:100B2000696679202000333A202B20416363657386
:100B3000736F72792000416E6C6167656E7A7573B0
:100B400074616E642000416E6C6167656E7A7573C6
:100B500074616E64200057696564657268657273BC
:100B600074656C6C6E0053706569636865726E20A5
:100B700020202020200020776965646572686572F6
:100B800073742E2020002073706569636865726E2F
:100B9000202020202000436F7572742028312E35CC
:100BA0006D73292000004C6F6E672028342E303280
:100BB000356D732900004D6F746F726F6C610000AA
:100BC00000000000000044434320202020200000BB
:100BD0000000000000004D4D20000000000000005B
:100BE000000000000000444343000000000000003B
:100BF000000000000000706F73697469766520283A
:100C00004D4D290000006E65676174697665202886
:100C1000444343290000303A206F6666202020209C
:100C2000202020202000313A205461696C626974D0
:100C3000732020202000323A202B2049644E6F740C
:100C4000696679202000333A202B20416363657365
:100C5000736F727920005265737461757261746983
:100C60006F6E20202000456E72656769737472652F
:100C70006D656E742000526573746175726174697C
:100C80006F6E20202000456E72656769737472650F
:100C90006D656E7420002045746174205265736523
:100CA00061752E20200020457461742052657365A3
:100CB00061752E2020004B6F72722028312E356D09
:100CC0007329202000004C616E672028342E3032BA
:100CD000356D732900004D6F746F726F6C61000089
:100CE000000000000000444343202020202000009A
:100CF0000000000000004D4D20000000000000003A
:100D00000000000000004443430000000000000019
:100D1000000000000000506F736974696566202848
:100D20004D4D290000004E65676174696566202895
:100D3000444343290000303A206F6666202020207B
:100D4000202020202000313A205461696C626974AF
:100D5000732020202000323A202B2049644E6F74EB
:100D6000696679202000333A202B20416363657344
:100D7000736F727920004D6F64656C6261616E7390
:100D800069742E2020004D6F64656C6261616E7322
:100D900069742E2020004865727374656C6C656EF2
:100DA0002020202020004F70736C61616E20202075
:100DB000202020202000206865727374656C6C65AB
:100DC0006E2020202000206F70736C61616E2020E7
:100DD00020202020200073686F72742028312E3567
:100DE0006D73292000006C6F6E672028342E30321E
:100DF000356D732900004D6F746F726F6C61000068
:100E00000000000000004443432020202020000078
:100E10000000000000004D4D200000000000000018
:100E200000000000000044434300000000000000F8
:100E3000000000000000706F7369746976652028F7
:100E40004D4D290000006E65676174697665202844
:100E5000444343290000303A206F6666202020205A
:100E6000202020202000313A205461696C6269748E
:100E7000732020202000323A202B2049644E6F74CA
:100E8000696679202000333A202B20416363657323
:100E9000736F72792000526573746F726520202021
:100EA0002020202020005361766520202020202053
:100EB000202020202000526573746F72652020204E
:100EC0002020202020005361766520202020202033
:100ED000202020202000206C61796F7574207374AD
:100EE000617475732000206C61796F757420737460
:100EF0006174757320005B756E6B6E6F776E207317
:100F000074617475735D00696E6B6F6D7061742EC2
:100F100020466F726D617400466F726D6174206956
:100F20006E636F6D7061742E00496E636F6D702E0D
:100F300020466F726D6174202000696E636F6D7062
:100F400061742E20466F726D6174005B756E6B6EFE
:100F50006F776E206572726F725D002E2E2E207775
:100F6000617274656E202E2E2E202000233D4CF6DB
:100F7000736368656E0000000000000000286B6568
:100F8000696E2045696E7472616729000000202E29
:100F90002E2E206CF673636865202E2E2E200020E6
:100FA0004665686C657200000000000000000000EB
:100FB000206E75722066FC7220444343212020205D
:100FC00000206572737420474F206472FC636B6568
:100FD0006E002A3D41626272756368000000000085
:100FE0000000002050726F6772616D6D69657275E7
:100FF0006E6700002D2D204B75727A7363686C75D7
:10100000DF202D2D00204E617469762028313A3181
:10101000292020202000204C696E65617220283232
:101020003A3129202020002050726F677265737357
:1010300069762031202020002050726F677265731E
:10104000736976203220202000204143204D6F64B8
:1010500075732020202020202000204443204D6F45
:101060006475732020202020202000204175746F9B
:101070005374657020202020202020002A6C657386
:10108000656E00000000000000000000002A73638D
:1010900068722E00000000000000000000002E2EEC
:1010A0002073636872656962656E202E2E00002EC3
:1010B0002E2E206C6573656E202E2E2E20200000B3
:1010C000212121204665686C6572202121212000A4
:1010D00000204F4B202020202020202020202020D6
:1010E00000002E2E2073706569636865726E202E75
:1010F0002E00007769656465726865727374656C4B
:101100006C656E00233D4CF6736368656E202A3D66
:101110004162627200233D4A61202A3D416262724F
:10112000756368000000206CF6736368656E2020AC
:101130002020202020200041555300000000000006
:1011400000000000000000002A2A206B65696E651F
:10115000204C6F6B202A2A20002A2A204B75727A95
:101160007363686C75DF202A2A002A205A65697427
:10117000FC626572736368722E2A00576569636842
:1011800065202534642F2534640000004B6F6E66A3
:10119000696775726174696F6E20202000204B6F43
:1011A0006E66696775726174696F6E2020005061A8
:1011B0007469656E74657A00000000000000002309
:1011C0003D7375707072696D6572000000000000FB
:1011D0007669646500000000000000000000000067
:1011E000005375707072657373696F6E0000000054
:1011F000000020457272657572000000000000005A
:101200000000002044434320756E697175656D656B
:101210006E74200020707265737320474F206669DA
:1012200072737400002A3D4162616E646F6E00004B
:101230000000000000002050726F6772616D6D61E8
:1012400074696F6E0000002D436F7572742D6369B1
:1012500072637569742D2000206E61746976652053
:1012600028313A312920202000206C696E65617296
:101270002028323A3129202020002070726F6772B6
:1012800065737369766520312020002070726F6766
:1012900072657373697665203220200020414320F7
:1012A0004D6F646520202020202020200020444312
:1012B000204D6F6465202020202020202000204128
:1012C00075746F5374657020202020202020002A20
:1012D0004C6563742E000000000000000000000058
:1012E0002A456372697400000000000000000000DD
:1012F000002E2E2E204563726974757265202E2E85
:101300002E002E2E2E204C656374757265202E2EB5
:101310002E20002121212045727265757220212125
:1013200021202000204F4B20202020202020202082
:10133000202020200020456E7265676973747265F5
:101340006D656E74200020526573746175726174EE
:10135000696F6E20202000233D5375707072202A23
:101360003D4162616E642E00233D4F7569202A3D28
:101370004162616E646F6E200020537570707269F7
:101380006D657220202020202000496E6163746901
:1013900066202020202020202020002A2050617359
:1013A000206465206C6F636F202A20002A20436F21
:1013B0007572742D6369726375697420002A2054F4
:1013C000656D707320646570617373652000416999
:1013D0006775696C2E2534642F2534640000004540
:1013E0006E72656769737472656D656E7420200036
:1013F000526573746175726174696F6E202020206C
:10140000002E2E2E207761636874656E202E2E2E9E
:101410002000233D77697373656E000000000000B3
:10142000000000286765656E20696E766F65722919
:1014300000000000202E2E2E2077697373656E2029
:101440002E2E2E000020666F757400000000000034
:1014500000000000000020416C6C65656E20444374
:101460004321202020200020707265737320474F95
:1014700020666972737400002A3D41666272656B72
:10148000656E000000000000002050726F677261FE
:101490006D6D6572656E000000002D2D4B6F7274CE
:1014A000736C756974696E672D2D00206E617469A7
:1014B00076652028313A312920202000206C696E81
:1014C0006561722028323A31292020200020707274
:1014D0006F67726573736976652031202000207014
:1014E000726F677265737369766520322020002001
:1014F0004143204D6F6465202020202020202000C3
:10150000204443204D6F646520202020202020208F
:1015100000204175746F53746570202020202020B6
:1015200020002A4C657A656E000000000000000073
:101530000000002A53636872690000000000000088
:10154000000000002E2E2073636872696A76656E53
:10155000202E2E00002E2E2E206C657A656E202EF9
:101560002E2E202000002021212120466F7574207E
:1015700021212120200000204F4B2020202020204E
:1015800020202020202000002E2E2E204F70736C53
:1015900061616E202E2E2E00004865727374656C9A
:1015A0006C656E20202020200000233D7769737336
:1015B000656E202A3D616662720000233D4A61200B
:1015C0002A3D41666272656B656E20002077697303
:1015D00073656E20202020202020202000554954B3
:1015E00000000000000000000000000000002A2AA7
:1015F0002A206765656E204C6F63202A2A2A002AFC
:101600002A6B6F7274736C756974696E672A2A002D
:101610002A2054696A646F766572736368722E2A31
:101620000057697373656C732534642F2534640027
:101630000000436F6E666967202020202020202054
:1016400020200020436F6E66696720202020202024
:10165000202020002E2E2E2077616974696E67206D
:101660002E2E2E2000233D64656C657465000000FD
:10167000000000000000286E6F20656E74727929EA
:10168000000000000000002E2E2E2064656C6574A2
:10169000696E67202E2E2E00206661756C74000026
:1016A00000000000000000000020444343206F6E53
:1016B0006C79212020202020200020707265737317
:1016C00020474F20666972737400002A3D43616EA3
:1016D00063656C0000000000000000002070726F65
:1016E0006772616D696E670000000000002D73680D
:1016F0006F727420636972637569742D2000206EA7
:1017000061746976652028313A3129202020002033
:101710006C696E6561722028323A312920202000E0
:101720002070726F6772657373697665203120204F
:10173000002070726F67726573736976652032205E
:101740002000204143204D6F646520202020202070
:10175000202000204443204D6F646520202020205D
:1017600020202000204175746F5374657020202064
:1017700020202020002A7265616420000000000003
:101780000000000000002A77726974650000000004
:10179000000000000000002E2E2E20777269746970
:1017A0006E67202E2E2E20002E2E2E207265616454
:1017B000696E67202E2E2E20002121212066617562
:1017C0006C742021212120202000204F4B2020203C
:1017D00020202020202020202020002E2E2E2073AC
:1017E0006176696E67202E2E2E2020002E2E20720C
:1017F0006573746F72696E67202E2E2000233D443E
:10180000656C2E202A3D43616E63656C2000233D8C
:10181000596573202A3D43616E63656C202000206A
:10182000636F6E66696775726174696F6E20200000
:101830004F464600000000000000000000000000CD
:10184000002A2A2A206E6F20547261696E202A2A8B
:101850002A002A2073686F72742063697263756945
:101860007420002A2A2A2074696D65206F757420FF
:101870002A2A2A00506F696E7420202534642F258F
:101880003464000000436F6E666967757261746945
:101890006F6E2020200020636F6E6669677572612D
:1018A00074696F6E2020005B6E6F206D65737361CD
:1018B00067655D0025642A2A2A204641494C555215
:1018C00045202A2A2A0025643A2030782530386CB1
:1018D00058002532642030782530386C582020207C
:1018E00000204D3320656E61626C656420202020ED
:1018F00020003D2535640030782530386C580020B4
:10190000253564002534646D73002533642C25640B
:101910007300202E2E2E2E2020202020202020205C
:10192000002564206D7300202532640031320000F0
:1019300032340000343800003936000031343400CD
:1019400031393200333834003537360030302042F8
:101950006175640025346400202D2D2D0020202089
:101960002020202000204F4B202020200025336401
:10197000002D2D2D002534643A20002536640020EA
:101980002D2D2D2D2D0025346400202D2D2D0043CF
:10199000563A253464204269743A25643D00435622
:1019A0003A20202020204269743A203D200025352D
:1019B0007500202D2D2D2D004142434445464748BA
:1019C000494A4B4C4D4E4F5051525354555657580F
:1019D000595A303132333435363738392E2C3A2D86
:1019E0002B232F3D3C7C3E20004D4D2049202031B3
:1019F0003420004D4D20492020323761004D4D20CC
:101A0000492020323762004D4D2002202031342001
:101A1000004D4D20022020323761004D4D20022024
:101A200020323762004443432020203134200044D8
:101A300043432020203238200044434320203132C9
:101A40003820006D3320202031323820003A200029
:101A5000253575005365724E722E2025386C750041
:101A6000322E312E3100536F6674772E20560025AA
:101A70003364004E723A202532642020004C6F6B94
:101A8000204D656EFC000000000000000044434350
:101A90002D50726F6772616D6D672E00006D33207F
:101AA00050726F6772616D6D672E000000416E6C41
:101AB0006167656E7A757374616E64000045696E66
:101AC0007374656C6C756E67656E000000536F66AD
:101AD000747761726520557064617465004C43448D
:101AE0002042656C6575636874756E67004D61733F
:101AF000746572436F6E74726F6C00000045786994
:101B00007400000000000000000000000041757338
:101B100077E4686C656E200000000000004461748A
:101B2000656E666F726D617400000000004E616D3D
:101B30006520202020202000000000000045696E64
:101B400074726167202020000000000000435620CE
:101B500028627974652900000000000000435620C7
:101B600028626974290000000000000000426173CF
:101B700069732D416472657373650000006C616E5A
:101B80006765204164726573736500000052656784
:101B90006973746572000000000000000050616706
:101BA000652D4D6F64650000000000000048617500
:101BB0007074676C65697300000000000052616911
:101BC0006C436F6D20435600000000000031323836
:101BD0004653204D6F6465000000000000526567A9
:101BE0006C65726D6F6475730000000000733838A7
:101BF0002D45696E7374656C6C756E67004B6F6E06
:101C000066696775726174696F6E000000426F6F7C
:101C100073746572000000000000000000496E74DB
:101C2000657266616365204261756400005765698D
:101C30006368656E0000000000000000004C6F6BE0
:101C4000666F726D6174000000000000004D4D2D44
:101C50005369676E616C20506175736500526169EC
:101C60006C436F6D20537570706F727400733838E9
:101C70002D4D6F64756C65000000000000733838EE
:101C80002D4D6F64756C746573740000004B757234
:101C90007A7363686C2E2D506F6C2E00004B75723A
:101CA0007A7363686C2E2D456D70662E00616C6CC6
:101CB00065205765696368656E00000000576569B7
:101CC0006368656E666F726D61740000006D696EA9
:101CD0002E20536368616C747A656974006D617855
:101CE0002E20536368616C747A656974006D3320CB
:101CF000416472657373650000000000004D656EFD
:101D000075204C6F636F0000000000000050726F80
:101D10006772616D2E20444343000000006D332044
:101D200050726F6772616D6D672E000000457461BF
:101D300074205265736561752E000000005265675E
:101D40006C6167657300000000000000004D414AAF
:101D5000206C6F67696369656C000000004C756DED
:101D6000696E6F736974650000000000004D617357
:101D7000746572436F6E74726F6C00000045786911
:101D80007400000000000000000000000053656CBB
:101D9000656374696F6E20000000000000466F727A
:101DA0006D617420646F6E6E65657300004E6F6DBB
:101DB0002020202020202000000000000053616926
:101DC0007369652020202000000000000043562099
:101DD0002862797465290000000000000043562045
:101DE000286269742900000000000000004164724C
:101DF0006573736520646520626173650041647278
:101E000065737365206C6F6E67756500005265675A
:101E10006973746572000000000000000050616783
:101E2000652D4D6F646500000000000000566F696D
:101E300065207072696E636970616C6500526169DA
:101E40006C436F6D204356000000000000313238B3
:101E50004653204D6F64650000000000004A6F6724
:101E60006469616C204D6F64650000000052656715
:101E70006C616765207338380000000000436F6EA6
:101E800066696775726174696F6E000000426F6FFA
:101E900073746572000000000000000000496E7459
:101EA00065726661636520426175640000436F6E10
:101EB000662E2041696775696C6C612E00466F72F1
:101EC0006D6174206C6F636F0000000000506175DD
:101ED0007365207369676E616C204D4D00526169B6
:101EE0006C436F6D20537570706F7274004D6F642A
:101EF000756C6573207338380000000000546573FA
:101F000074206D6F64756C652073383800506F6C89
:101F10002E6372742D636972637569740053656E04
:101F2000732E206372742D636972637400746F750D
:101F3000732061696775696C6C612E0000466F7271
:101F40006D61742061696775696C6C2E00547073E3
:101F5000206D696E2E696D70756C732E00547073F0
:101F6000206D61782E696D70756C732E00416472FE
:101F700065737365206D330000000000004C6F63D3
:101F80006D656E75000000000000000000444343D2
:101F90002D70726F6772616D6D2E0000006D332DB4
:101FA00070726F6772616D6D672E0000004D6F6417
:101FB000656C6261616E7369742E000000496E7316
:101FC00074656C6C696E67656E00000000536F6627
:101FD000747761726520557064617465004C434488
:101FE000207665726C69636874696E67004D617311
:101FF000746572436F6E74726F6C0000004578698F
:10200000740000000000000000000000004B696543
:102010007A656E200000000000000000004461743A
:1020200061666F726D61740000000000004E6161B6
:102030006D202020202020000000000000496E7646
:102040006F65722020202000000000000043562011
:1020500028627974652900000000000000435620C2
:1020600028626974290000000000000000426173CA
:10207000697361647265730000000000004C616E5A
:10208000672061647265730000000000005265679C
:102090006973746572000000000000000050616701
:1020A000652D4D6F646500000000000000486F6FF3
:1020B000666473706F6F7200000000000052616907
:1020C0006C436F6D20435600000000000031323831
:1020D0004653204D6F64650000000000004A6F67A2
:1020E0006469616C204D6F646500000000733838CE
:1020F0002D696E7374656C6C696E67656E436F6E87
:1021000066696775726174696500000000426F6FEF
:1021100073746572000000000000000000496E74D6
:10212000657266616365204261756400005769737A
:1021300073656C000000000000000000004C6F633D
:10214000666F726D6174000000000000004D4D204C
:102150007369676E61616C7061757A65005261695F
:102160006C436F6D20537570706F727400733838E4
:102170002D6D6F64756C65000000000000733838C9
:102180002D6D6F64756C657465737400004B6F72B0
:1021900074736C2E20706F6C2E000000004B6F72F9
:1021A00074736C2E206765762E00000000616C6CE5
:1021B000652057697373656C73000000005769737D
:1021C00073656C666F726D6174000000004D696E1E
:1021D0002E736368616B656C74696A64004D617825
:1021E0002E736368616B656C74696A64006D33207B
:1021F000616472657300000000000000004C6F63B2
:102200006F6D6F74697665206D656E75004443432C
:102210002070726F6772616D6D696E67006D33203B
:1022200070726F6772616D6D696E6700004C6179E5
:102230006F75742073746174757300000053657456
:1022400074696E67730000000000000000536F6641
:10225000747761726520557064617465004C434405
:10226000206261636B6C696768740000004D617384
:10227000746572436F6E74726F6C0000004578690C
:102280007400000000000000000000000053656CB6
:1022900065637420000000000000000000446174C9
:1022A0006120666F726D617400000000004E616D08
:1022B00065202020202020000000000000456E74D2
:1022C00072792020202020000000000000435620CA
:1022D0002862797465290000000000000043562040
:1022E0002862697429000000000000000050726933
:1022F0006D617279206164647265737300457874EE
:10230000656E642E20616464726573730052656744
:10231000697374657200000000000000005061677E
:10232000652D4D6F6465000000000000004D61697F
:102330006E20747261636B000000000000526169DE
:102340006C436F6D204356000000000000313238AE
:102350004653204D6F64650000000000004A6F671F
:102360006469616C204D6F6465000000007338384B
:102370002073657474696E67730000000044656CB7
:1023800065746500000000000000000000426F6FEF
:1023900073746572000000000000000000496E7454
:1023A00065726661636520426175640000506F6903
:1023B0006E7473000000000000000000004C6F63AA
:1023C0002E20666F726D617400000000004D4D207C
:1023D0007369676E616C2070617573650052616925
:1023E0006C436F6D20537570706F72740073383862
:1023F000206D6F64756C65730000000000733838E1
:10240000206D6F64756C6520746573740053686F1C
:10241000727420632E20706F6C2E00000053686F62
:10242000727420632E2073656E732E0000616C6CD5
:1024300020506F696E7473000000000000506F69D7
:102440006E747320666F726D61740000006D696E4A
:102450002E7377697463682E74696D65006D617899
:102460002E7377697463682E74696D65006D33200F
:1024700061646472657373000000000000446F774C
:102480006E6C6F6164202E2E2E20202020001124DF
:102490001FBECFEFD0E1DEBFCDBF12E0A0E0B1E0C4
:1024A000E4EEF9E501E00BBF02C007900D92A637FC
:1024B000B107D9F71EE0A6E7B2E001C01D92A93628
:1024C000B107E1F70E94C3120C94F0AC0C94000029
:1024D00080917602089581E080937702089580E0EC
:1024E0000E94C26781E00E94C2670E94C1770E9479
:1024F000DB8D0E94863F80917702882311F40E9431
:10250000A61EA8950895982F809176028917C9F183
:102510008630B9F1853011F4963099F590937602B2
:10252000892F8250823010F0973059F40E94423740
:102530001092C30780917602823029F40E943239CA
:1025400002C00E944D3280917602863011F40E94C2
:10255000076C80917602813011F482E003C08823F9
:1025600021F481E064E00E94849084E064E00E94B1
:102570008490809176020E94787981E0809377023E
:10258000089580E00895CF93DF930E94D66E0E9455
:10259000A9130E94CC3A0E94298C0E94CB300E9441
:1025A000C36B68E04EE421E00E94D71387E068E047
:1025B0004EE421E00E9466150E94811778940E94E3
:1025C0004C1C0E94C06BDC0114968C910E94A11ED1
:1025D00082E06DEA70E00E94FE200E94E26B813092
:1025E000D9F482E069EA70E00E94FE2081E060E0B8
:1025F0000E942A1F82E066E50E94242082E06CE8A7
:1026000070E00E94FE200E94C06BEC0181E00E94FD
:10261000221D882349F125C00E94E26B00D000D022
:102620000F92EDB7FEB7319692E0ADB7BEB71196F7
:102630009C9322EA30E032832183838314820E94B8
:10264000A4200F900F900F900F900F9081E060E00A
:102650000E942A1F82E062E970E00E94FE20A89595
:10266000FECF81E00E94826E82E00E94221D8823BC
:1026700019F080E00E94826E83E00E94221D882370
:1026800019F082E00E94826E84E00E94221D88235D
:1026900019F083E00E94826E80E00E94831285E13F
:1026A0000E94221D882311F00E94461D81E00E9495
:1026B000C97F80E00E94221D882319F088E10E94D2
:1026C0009EA50E94FD838FEF60E240E050E00E94F3
:1026D000E36F80E00E941F6B81E00E941F6B0E94ED
:1026E000099002C00E946F128091C5079091C607A1
:1026F000A091C707B091C807805D9740A040B04047
:1027000088F389859A85009749F060E070E040E0A1
:1027100050E00E942D85BC01009711F46A817B81F5
:102720008FEF0E940E6E81E011C00E94E2450E9470
:10273000601DFFEF8F3F9F07C1F70E946F128091CE
:1027400077028823A1F31092770280E00E94B140C3
:10275000EECF8FE78ABB1BBA80E187BB18BA80EF48
:1027600084BB8FEF85BB8BEB81BB8CEC82BB82E0A3
:1027700082B987EF83B987E78093610081EE809308
:10278000620087E18093640089E1809365000E9484
:10279000198010926A001ABE8AB78A608ABF0E94A6
:1027A0004819A89588E181BD8EE081BD08951092F9
:1027B0007F0790917F0790937E0790917E0790937B
:1027C000A1079091A1079093A00791E09093C20771
:1027D0008C9A119A92B19E7E92B9199A93B19E7E6B
:1027E00093B992E09BB99498883008F087E0E82F7D
:1027F000F0E0EE0FFF1FE754FF4FA591B491653055
:1028000010F465E003C0693008F068E04F7D655062
:10281000660F453411F4606203C04F3409F46063FD
:10282000223008F068608B2F992787FD9A958F706A
:1028300080939000A9B96093950088EB8AB980E0F5
:1028400090E008951F920F920FB60F920BB60F9261
:1028500011248F939F93EF93FF939091A007809102
:10286000A107981761F088B7806188BF0C9B09C0E9
:102870008091C20780FF05C089B7806189BF5598E4
:1028800012C0E091A107F0E0E258F84F84A18CB9A2
:102890008091A1078F5F8093A1078091A10780326B
:1028A00010F01092A107FF91EF919F918F910F90DF
:1028B0000BBE0F900FBE0F901F9018951F920F9296
:1028C0000FB60F9211248F9389B78F7E89BF559AC7
:1028D0008F910F900FBE0F901F90189527E0813DAC
:1028E0009207C0F12FE0813A920710F481E01EC0F8
:1028F00023E28932920710F482E018C026E3813B7C
:10290000920710F483E012C026E48135920710F498
:1029100084E00CC028E8893B920710F485E006C0EB
:10292000895D964D10F087E001C086E0789420E044
:1029300030E05E9902C020E030E02F5F3F4FA89565
:1029400097E220313907A8F368E04EE421E00E94C5
:10295000D713089580E0EACF8330C9F0843028F49B
:10296000813061F0823080F40CC08530B1F0853068
:1029700088F08630A9F08730C9F415C020E639E028
:1029800017C020EB34E014C020EC32E111C020E885
:1029900035E20EC020E438E30BC020E03BE408C081
:1029A00020E036E905C020E031EE02C020E030E052
:1029B000C901089539B120919000922F80E0232F12
:1029C00030E0282B392B49EB50E060E0FA0185918B
:1029D00094918217930729F06F5F4E5F5F4F6830C5
:1029E000A9F7862F0E94AC140895482FA89503C01C
:1029F000559A7894A8952091A0078091A10730E07E
:102A000090E001972817390799F38091A0078F313B
:102A100021F48091A107882359F3E091A007F0E009
:102A2000E258F84F44A39FB7F8948091A0078F5FB6
:102A30008093A0078091A007803210F01092A00729
:102A40009FBF559A80E090E00895F89480917E07AA
:102A500090917F07282F30E0291B3109789437FFA8
:102A600002C0205E3F4F2031310534F49498232B6F
:102A700019F42FEF3FEF15C0E0917F07F0E0E25827
:102A8000F84F9281F89480917F078F5F80937F0742
:102A900080917F07803210F010927F07292F30E05D
:102AA0007894C90108959091C207882331F08091EC
:102AB000C20781608093C20706C08091C2078E7FE3
:102AC0008093C207559A892F8170089510923A0712
:102AD00090913A07909339079091390790935C074A
:102AE00090915C0790935B0791E090937D0791B381
:102AF000986291BB8A981598939A92981D9892E043
:102B000090939B009598883008F087E0E82FF0E0DC
:102B1000EE0FFF1FE754FF4FA591B491653010F4FD
:102B200065E003C0693008F068E04F7D6550660FCE
:102B30008B2F992787FD9A958F7080939800A0938B
:102B40009900453411F4606203C04F3409F46063A6
:102B5000223008F0686060939D0088EB80939A00B3
:102B600080E090E008951F920F920FB60F920BB67F
:102B70000F9211248F939F93EF93FF9390915B0794
:102B800080915C07981761F088B7806288BF0D9BC1
:102B90000DC080917D0780FF09C089B7806289BF21
:102BA00080919A008F7D80939A0013C0E0915C071A
:102BB000F0E0E75CF84F84A180939C0080915C0773
:102BC0008F5F80935C0780915C07803210F01092D9
:102BD0005C07FF91EF919F918F910F900BBE0F902B
:102BE0000FBE0F901F9018951F920F920FB60F9265
:102BF0000BB60F9211248F93EF93FF9389B78F7DBC
:102C000089BFEAE9F0E0808180628083FF91EF91E3
:102C10008F910F900BBE0F900FBE0F901F901895C5
:102C2000482FA89507C080919A00806280939A00EF
:102C30007894A89520915B0780915C0730E090E044
:102C400001972817390779F380915B078F3121F4B9
:102C500080915C07882339F3E0915B07F0E0E75C43
:102C6000F84F44A39FB7F89480915B078F5F8093E0
:102C70005B0780915B07803210F010925B079FBF6B
:102C800080919A00806280939A0080E090E008959D
:102C9000F8948091390790913A07282F30E0291B4A
:102CA0003109789437FF02C0205E3F4F2031310553
:102CB00034F49598232B19F42FEF3FEF15C0E091D2
:102CC0003A07F0E0E75CF84F9281F89480913A0778
:102CD0008F5F80933A0780913A07803210F010920C
:102CE0003A07292F30E07894C90108959091C207DE
:102CF000882331F080917D07816080937D070AC031
:102D000080917D078E7F80937D0780919A008062FD
:102D100080939A00892F817008951F920F920FB6A9
:102D20000F920BB60F9211242F933F934F935F9303
:102D30006F937F938F939F93AF93BF93EF93FF9383
:102D40002091390780913A0730E090E001972817E9
:102D5000390741F0809139078F3179F480913A0732
:102D6000882359F480913A078F5F80933A078091C6
:102D70003A07803210F010923A0780919B00E09160
:102D80003907F0E090919C00E75CF84F92839281C4
:102D900084FD0CC0809139078F5F80933907809143
:102DA0003907803278F0109239070CC0992351F41A
:102DB00010923A0780913A0780933907959881E0FD
:102DC0000E941F6B8091390790913A07282F30E0BD
:102DD000291B310937FF02C0205E3F4F21313105E9
:102DE0000CF0959AFF91EF91BF91AF919F918F91C8
:102DF0007F916F915F914F913F912F910F900BBEFB
:102E00000F900FBE0F901F9018951F920F920FB644
:102E10000F920BB60F9211242F933F934F935F9312
:102E20006F937F938F939F93AF93BF93EF93FF9392
:102E300020917E0780917F0730E090E0019728176E
:102E4000390741F080917E078F3179F480917F07B7
:102E5000882359F480917F078F5F80937F0780914B
:102E60007F07803210F010927F078BB1E0917E07D0
:102E7000F0E09CB1E258F84F9283928184FD0CC03F
:102E800080917E078F5F80937E0780917E078032DE
:102E9000A8F010927E0712C0992381F410927F0748
:102EA00080917F0780937E07949880E00E941F6B3B
:102EB00081E068E04EE421E00E94D71380917E0714
:102EC00090917F07282F30E0291B310937FF02C07E
:102ED000205E3F4F213131050CF0949AFF91EF9124
:102EE000BF91AF919F918F917F916F915F914F9122
:102EF0003F912F910F900BBE0F900FBE0F901F9020
:102F0000189587B3876087BBBB9888B3896088BBF7
:102F10001DB88EB18FB187E78DB9089578941F924F
:102F20000F920FB60F920BB60F9211242F938F931F
:102F30009F93EF93FF938FB1E0917802F0E0E85810
:102F4000FD4F8283809178028F5F80937802809119
:102F50007802883110F01092780290917902809175
:102F60007802981759F4809179028F5F80937902E3
:102F700080917902883110F010927902E0919302E9
:102F8000F0E0E858FD4F248D27FF19C0C09A0000DB
:102F90000000000000000000000000000000000031
:102FA0000000000000000000000000000000000021
:102FB00000000000000000000000000000009091F0
:102FC000930280919202981771F0C09880919302B9
:102FD0008F5F8093930280919302883110F010925A
:102FE00093022FB902C0C09A6F98FF91EF919F9101
:102FF0008F912F910F900BBE0F900FBE0F901F90CF
:1030000018958091930290919202282F30E0295ECA
:103010003F4F291B31092831310514F02851304028
:10302000C9010895482F6F9933C0C0988FB16F9A26
:103030009091920280919302981711F44FB94BC06E
:10304000E0919302F0E0E858FD4F848D8FB98091B4
:1030500093028F5F80939302809193028831C0F036
:103060001092930215C06F9913C0E0919302F0E0A3
:10307000E858FD4F848D8FB9809193028F5F8093C4
:10308000930280919302883110F0109293026F9A0C
:10309000809192022091930290E0019630E0821795
:1030A000930709F380919202873121F48091930272
:1030B0008823C9F2E0919202F0E0E858FD4F448F76
:1030C000809192028F5F8093920280919202883168
:1030D00010F01092920280E090E008954FB7F894BB
:1030E0009091780280917902981719F42FEF3FEFB1
:1030F00013C0E0917902F0E0E858FD4F8281282F5B
:1031000030E0809179028F5F80937902809179021B
:10311000883110F0109279024FBFC90108958823B9
:1031200011F0DD9A0895DD980895882351F080917B
:1031300065008460809365000000000000000000CE
:103140000895809165008B7F8093650008950F93AB
:103150001F93DF93CF930F92CDB7DEB7182F8AB3AB
:10316000807F8ABB80E00E94951880916500826014
:1031700080936500112321F080916500816003C078
:10318000809165008E7F809365000000000081E0E3
:103190000E94951809B380E00E94951810E084E021
:1031A000000F111F8A95E1F70000000000000000E9
:1031B00081E00E94951899B39F70902B80E09983CD
:1031C0000E9495188AB38F608ABB9981892F0F90CE
:1031D000CF91DF911F910F91089580E00E94A71871
:1031E000982F87FF11C08091AF029091B00228E024
:1031F0008130920714F080E0089501969093B00218
:103200008093AF0281E008958091B602882319F47B
:103210009F779093B7021092B0021092AF0280E0B5
:1032200008959B01AC018091C5079091C607A091BC
:10323000C707B091C80782179307A407B50798F08E
:103240008091C5079091C607A091C707B091C807A4
:1032500060E0821B930BA40BB50B80509041A04003
:10326000B040A0F412C08091C5079091C607A0910C
:10327000C707B091C80760E0281B390B4A0B5B0BEE
:103280002050304F4F4F5F4F08F061E0862F089578
:1032900010927D0080B7877F80BF17BE11BE89E680
:1032A00083BF8BE085BD8FE183BD87B7806887BF13
:1032B00082EF8FBD3AE13EBD4FEC50E057BD46BDB9
:1032C00085EB90E09BBD8ABD99BD88BD22EC209323
:1032D0008B0030938A00509381004093800090933C
:1032E0008700809386000895EF92FF920F931F93BB
:1032F0002091C5073091C6074091C7075091C80774
:103300007C0100E010E0E20EF31E041F151F01C057
:10331000A895C801B7010E9411198823C9F31F910C
:103320000F91FF90EF900895FF920F931F93082F36
:10333000162FF42E809165008D7F8093650080E0CC
:103340000E9495188AB38F608ABB8BB3902F929599
:103350009F70807F982B9BBB112321F0809165008B
:10336000816003C0809165008E7F8093650081E05D
:103370000E94951880E00E949518FF2029F088E0AF
:1033800090E00E9474190FC08BB30F70807F802B68
:103390008BBB000000000000000081E00E94951837
:1033A00080E00E9495181F910F91FF900895EF9271
:1033B000FF920F931F932091C5073091C60740914C
:1033C000C7075091C8077C0100E010E0E20EF31E31
:1033D000041F151F02C00E946F12C801B7010E948E
:1033E00011198823C1F31F910F91FF90EF90089559
:1033F0000F931F93282F8091B502893018F48F5FA7
:103400008093B5028091B5028430B1F0853048F4E4
:10341000823009F4C0C0833008F0BAC08130E9F4CA
:1034200009C08630B1F0863090F08730A1F0883046
:10343000A1F4B1C0DC9AAFC01092B4021092B302F2
:1034400080E090E89093B2028093B10206C0DD9ACA
:10345000A2C0DD98A0C0DC989EC0222309F098C0CD
:103460006091B3027091B4022091B1023091B20226
:10347000CF9B3CC0FB01EE0FFF1FE150F34F80815B
:10348000918182239323892B61F483EF9CE00E9436
:103490006B916091B3027091B40289EF9CE00E943D
:1034A0006B91E091B302F091B4022091B10230919E
:1034B000B202EE0FFF1FDF01A657B34F8D919C9113
:1034C0001197822B932B8D939C93DF01AE5DB34FAD
:1034D0008D919C911197822B932B8D939C93E1500E
:1034E000F34F80819181822B932B29C0FB01EE0F3A
:1034F000FF1FE150F34F8081918182239323892B19
:1035000061F083EF9CE00E946B916091B302709137
:10351000B40289EF9CE00E946B91E091B302F091BC
:10352000B402EE0FFF1FE150F34F8091B102909172
:10353000B2028095909520813181822393239183DB
:1035400080838091B1029091B20296958795909375
:10355000B2028093B102892BE9F40091B302109179
:10356000B4020F5F1F4F1093B4020093B3020E9486
:10357000C06BFC01808590E00817190710F01092CD
:10358000B50280E090E89093B2028093B10202C04D
:10359000DE9A01C0DE981F910F9108951F920F923D
:1035A0000FB60F920BB60F9211241F932F933F93D8
:1035B0004F935F936F937F938F939F93AF93BF933B
:1035C000EF93FF938091AC02882309F051C181E011
:1035D0008093AC02789480E00E94F8198091AE024A
:1035E0008F5F8093AE028091AE0290E08370907006
:1035F0008130910519F1823091051CF4892B41F03D
:10360000E5C08230910561F1039709F0DFC065C024
:103610008091C5079091C607A091C707B091C807D0
:103620000196A11DB11D8093C5079093C607A09375
:10363000C707B093C8070E942E1DC8C08091C50758
:103640009091C607A091C707B091C807817090708C
:10365000892B19F00E947C1DB9C00E94E61CB6C0DF
:103660000E946812833049F00E946812823029F06B
:103670000E946812873009F0A9C00E94AC302091E6
:10368000C3073091C4078823E9F02E5F3F4F309382
:10369000C4072093C3070E94C06BFC019681992345
:1036A00009F494C08AE0989FC00111242091C307B7
:1036B0003091C4072817390708F488C081E00E94B8
:1036C000831284C02115310509F480C02150304097
:1036D0003093C4072093C30779C00E9468128330D7
:1036E00059F1843028F4813061F0823008F513C03C
:1036F0008730D9F1883009F448C0843009F061C0BE
:1037000024C08091C5079091C607A091C707B091CA
:10371000C80786FF04C080916200816003C0809169
:1037200062008E7F80936200809162008F7E4CC029
:1037300080916200816148C08091620080618093C5
:103740006200809162008E7F3FC0809162008E7F18
:10375000809362008091C5079091C607A091C7072A
:10376000B091C80790FFE0CF1FC0809162008E7FAC
:10377000809362008091C5079091C607A091C7070A
:10378000B091C80791FFD0CF0FC08091C50790912D
:10379000C607A091C707B091C80787FF09C08091ED
:1037A00062008E7F809362008091620080610CC015
:1037B000809162008F7E80936200809162008160C0
:1037C00003C0809162008E7E809362008091AD0282
:1037D000882321F00E94ED188093AD028091AD0204
:1037E000882309F040C09091C9078091CA079817B3
:1037F000B9F18091CA07E82FF0E0E753F84F9281C2
:10380000182F1F5F103108F010E0903801F58091FB
:10381000C907811729F1E12FF0E0E753F84F9281B2
:103820009F3F19F49091B702906897FF02C01092E1
:10383000B602892F807C803419F481E08093B6022F
:103840001F5F103108F010E0892F60E002C0892F5F
:1038500061E040E00E9494191093CA0781E001C022
:1038600080E08093AD0281E00E94F8191092AC02D2
:10387000FF91EF91BF91AF919F918F917F916F9148
:103880005F914F913F912F911F910F900BBE0F9021
:103890000FBE0F901F901895CF93DF9388E290E0B2
:1038A0000E94741980E360E041E00E94941980E373
:1038B00060E041E00E94941980E360E041E00E94F2
:1038C000941980E260E041E00E94941988E20E942D
:1038D000141F80E40E94141F8AE00E94E11E89E206
:1038E0000E94141F8CE10E94141F82E50E94141F85
:1038F00089E60E94141F84E70E94141F80E40E943E
:10390000141F85E10E94E11E88E20E94141F80E4DA
:103910000E94141F0E94123EEC0101C0A8959091D4
:10392000C9078091CA079817C9F70E94ED18882324
:10393000A9F781E00E94A7188A3019F481E089ABC9
:1039400001C019AA88E00E94141F81E00E94141F80
:1039500086E00E94141F8CE00E94141F80E060E04B
:103960000E942A1F80E062EE70E00E940B2081E03E
:1039700066E271E00E940B2082E06EE271E00E943C
:103980000B2083E06EE371E00E940B20DF91CF916A
:1039900008959091BA02E92FF0E0E654FD4F82833A
:1039A0009F5F9093BA02983010F01092BA029091F3
:1039B000BB028091BA02981741F4892F8F5F8093E0
:1039C000BB02883010F01092BB02089531B12091F3
:1039D000B902220F36FD2160822F83708150823020
:1039E00028F424FF02C02E6001C0217F2093B90279
:1039F0009091B802990F37FD9160892F83708150A3
:103A0000823028F494FF02C09E6001C0917F9093A1
:103A1000B802207C892F807C203831F4882341F043
:103A2000803C79F48AE105C0203459F4803C21F4CB
:103A300089E10E94C91C0895882319F48AE10E9433
:103A4000C91C0895893110F080E00895E82FF0E056
:103A5000EB53FD4F8081811181E008953091F70291
:103A6000343029F485B3806F85BB97980895979A71
:103A700025B380E190E002C0880F991F3A95E2F7E4
:103A80008095807F2F70822B85BB089581E0809385
:103A9000C40208958091C402882389F08091C507EB
:103AA0009091C607A091C707B091C8078958934164
:103AB000A040B04020F00E94B06E1092C402089561
:103AC0000E944A1D9091BB028091BA02891719F495
:103AD0002FEF3FEF0FC0E92FF0E0E654FD4F82815A
:103AE000282F30E0892F8F5F8093BB02883010F041
:103AF0001092BB02C90108958F929F92AF92BF921C
:103B0000CF92DF92EF92FF920F931F93CF93DF93A9
:103B10000E946812982F8091F802981729F09093CC
:103B2000F80282E20E94C91C83B3E1B0EE0CEE0CF5
:103B300090E1E9228F70E82ACC24DD2495E0A92EBB
:103B400081E0882E912CBB24B394E091F702EA9D8A
:103B5000F0011124EC0DFD1DE753FF4FF49088E1B7
:103B60008F1508F497C00E2D08250170CF2DD0E0D9
:103B7000FE01E252FD4F1081110F0E94E26B80386E
:103B800019F4002371F009C001111160812F90E038
:103B9000817190708131910511F41F6103C0892BEF
:103BA00009F4107E812F90E080769070803491052A
:103BB00019F41F7182E00CC08032910519F4106E67
:103BC00081E006C08036910511F080E001C083E0FD
:103BD000FE01E252FD4F1083823091F0833099F163
:103BE000813009F057C096E1F91621F48091DA028C
:103BF000882319F48F2D0E94C91CCB53DD4F3DC083
:103C0000CB53DD4F18828F2D80680E94C91C0E9403
:103C10006812853091F485E1F81629F48091DB0271
:103C2000882341F00DC096E1F916A1F58091DA02E2
:103C3000882381F586E00E94831285E1F81651F50C
:103C40001092C40227C0FE01EB53FD4F80818F5FAD
:103C50008083882309F4B08295E1F916D8F086E1D3
:103C60008F1568F497E1F916A9F4CB53DD4F8881DD
:103C7000853680F081E20E94C91CB8820BC0809119
:103C8000DA02893738F08091DB02893718F085E055
:103C90000E9483120894C11CD11C85E0C816D1046F
:103CA00011F0E69452CF8091F7028F5F8093F70274
:103CB000853010F01092F702DF91CF911F910F9194
:103CC000FF90EF90DF90CF90BF90AF909F908F903C
:103CD00008959093F6078093F507892B89F17093E7
:103CE000F4076093F3078091C5079091C607A091F0
:103CF000C707B091C8079B0140E050E0280F391F6B
:103D00004A1F5B1F2093EF073093F0074093F107A2
:103D10005093F2078091EE078E7F8093EE07211576
:103D200031054105510561F481E090E0A0E0B0E08B
:103D30008093EF079093F007A093F107B093F207F9
:103D40000895813308F080E381BF08958091F507DD
:103D50009091F607892BA1F16091EF077091F00720
:103D60008091F1079091F2070E941119882341F187
:103D70008091EE07E091F507F091F60781700995C3
:103D80008091EE0791E089278093EE072091C50787
:103D90003091C6074091C7075091C8078091F3073B
:103DA0009091F407A0E0B0E0820F931FA41FB51F0D
:103DB0008093EF079093F007A093F107B093F20779
:103DC00008951F93182F09C080E00E94C26781E008
:103DD0000E94C2670E94C177A8952091C90780916F
:103DE000CA0730E090E001972817390769F38091FE
:103DF000C9078F3021F48091CA07882329F3F894EA
:103E0000E091C907F0E0E753F84F12838091C907AA
:103E10008F5F8093C9078091C907803110F010929D
:103E2000C90778941F9108951F93182F80E80E9466
:103E3000E11E812F0E94E11E1F9108951092F60746
:103E40001092F50781E00E94141F08958CE00E94F3
:103E5000141F08958295880F880F807C860F8068D4
:103E60000E94141F0895BF92CF92DF92EF92FF92AB
:103E70000F931F93CF93DF93C82EB62E8A01109213
:103E8000F6071092F50721E02817A0F13FE036175A
:103E900088F14115510571F1FA0101900020E9F70F
:103EA0003197DE2ED41A80E18D1510F490E1D92ED1
:103EB0008C2D6B2D0E942A1FE8018BEDE82E87E0E8
:103EC000F82E08C08881F70181937F01699182E013
:103ED0000E9424209E01201B2D15A0F3C092EB0709
:103EE000B092EC07D092ED078DEA9FE164EF71E0AC
:103EF0000E94691EDF91CF911F910F91FF90EF906B
:103F0000DF90CF90BF900895DF93CF93CDB7DEB70A
:103F1000A0970FB6F894DEBF0FBECDBFDE0111969D
:103F20009E01205E3F4F04C09D93A217B30731F05E
:103F3000FA014F5F5F4F94919923B1F71C92AE0144
:103F40004F5F5F4F0E94331FA0960FB6F894DEBFFD
:103F50000FBECDBFCF91DF9108950F931F93CF93E5
:103F6000DF93082F8091EB076091EC070E942A1FD6
:103F700010E0CBEDD7E009C0002311F460E201C0EE
:103F8000699182E00E9424201F5F8091ED0718173D
:103F900098F3DF91CF911F910F9108950E942A1FEE
:103FA0008EE00E94141F0895EF92FF920F931F93CB
:103FB000CF93DF93382F7B01122F883028F54830BC
:103FC00018F5842F90E0820F911D099714F018E0E6
:103FD000141B330F330F330F340F832F80640E9471
:103FE000141FC0E0D0E0012F10E008C0F701EC0F73
:103FF000FD1FE4918E2F0E94E11E2196C017D1076C
:10400000ACF38FEF0E94141FDF91CF911F910F919E
:10401000FF90EF90089540E028E00E94D41F08959B
:10402000813069F0813040F0833019F02FEF3FEF9D
:1040300009C00E94601D05C00E94251502C00E9493
:1040400048169C01C90108951F93162F813009F469
:1040500065C0813008F45EC0823009F062C067FF3D
:1040600055C00E94123EFC0181A98823E1F0143E54
:1040700011F414E84BC0163F11F414E947C01C3F7B
:1040800011F411E843C0143C11F41EE83FC0163D82
:1040900011F419E93BC01C3D11F41AE937C0113F76
:1040A00069F51BE933C0143E11F411EE2FC0163F21
:1040B00011F41FEE2BC01C3F11F415EF27C0113F68
:1040C00011F41EEE23C0143C39F484E06EEF71E06D
:1040D0000E940B2014E01AC0163D39F485E066E01A
:1040E00072E00E940B2015E011C01C3D39F486E0FF
:1040F0006EE072E00E940B2016E008C01F3D31F414
:1041000087E066E172E00E940B2017E0812F0E9499
:10411000E11E07C0862F0E94F51403C0862F0E945F
:1041200010161F9108951F93CF93DF93182FEB0163
:1041300004C02196812F0E94242068816623C9F73C
:10414000DF91CF911F9108950F931F93DF93CF932A
:10415000CDB7DEB7C055D0400FB6F894DEBF0FBE66
:10416000CDBF9E01265A3F4F8E010F5F1F4FC801E2
:104170006A966EAD7FAD6A97A9010E94CDA9689637
:104180008FAD6897B8010E949320C05BDF4F0FB6D8
:10419000F894DEBF0FBECDBFCF91DF911F910F917D
:1041A00008950F931F93DF93CF93CDB7DEB7C0551C
:1041B000D0400FB6F894DEBF0FBECDBF9E01265A89
:1041C0003F4F8E010F5F1F4FC8016A966EAD7FADE6
:1041D0006A97A9010E94A4A968968FAD6897B80153
:1041E0000E949320C05BDF4F0FB6F894DEBF0FBE76
:1041F000CDBFCF91DF911F910F9108951F93CF9362
:10420000DF93182FEB0104C0812F0E9424202196F8
:10421000FE0164916623C1F7DF91CF911F9108954C
:10422000582F5F705F3011F45EE001C051115F5F85
:10423000442311F490E001C098E0623061F06330F3
:1042400018F4613069F405C0633039F0643041F42A
:1042500006C0936005C0946003C0966001C097607B
:10426000951739F4442319F4592F95E002C0592FBA
:104270009AE080E020E030E0880F880F50FD8260F7
:1042800090FD81602F5F3F4F2430310519F0569526
:104290009695F2CF90E00895962F9F709F3011F47D
:1042A00091E002C091119F5F8370813071F480E0D2
:1042B00020E030E0880F880F90FD83602F5F3F4F34
:1042C0002430310501F19695F5CF67FD06C0983091
:1042D00010F44DE007C045E005C0983010F042E012
:1042E00001C04AE080E020E030E0880F880F90FDB8
:1042F000826040FD81602F5F3F4F2430310519F00F
:1043000096954695F2CF90E008959C01FB01803888
:10431000910520F48F77808388E00895832F806C47
:104320008183208380E10895F90108969C0153E080
:10433000369527955A95E1F72F73206821839C01C4
:104340002095309595E0369527959A95E1F7207759
:104350008770282B2083662319F0216020830BC0EF
:10436000822F80688083442311F028682083808115
:1043700091E08927808380E108950F93CF93DF93A5
:10438000EC01A62FA695A695A695862F877078E0B6
:10439000781B04C0220F331F441F551F8A95D2F784
:1043A00012C0FE01EA0FF11D8081822B8083872FCE
:1043B000071708F4802F680F081B232F342F452F71
:1043C0005527AF5F78E0002361F7862FDF91CF910B
:1043D0000F9108950F93E42F8038910530F4916088
:1043E0009C0140E050E009E01AC022E080309207D2
:1043F00030F49C609C0140E050E00CE010C028E0EC
:104400008030920730F490679C0140E050E00FE06C
:1044100006C09C0140E050E0306C436002E1CB01FB
:104420006E2F0E94BD210F9108956FB7F8944091AF
:10443000F7078091F807242F30E090E001972817C4
:10444000390749F04F3011F050E006C08091F8076D
:1044500050E0882309F451E06FBF6FB7F8944091A2
:10446000A5088091A608242F30E090E00197281736
:10447000390749F04F3011F090E006C08091A6084E
:1044800090E0882309F491E06FBF892F852B089570
:10449000AF92BF92CF92DF92EF92FF920F931F9352
:1044A000CF93DF93EC015A01122F809138038823B8
:1044B00009F057C0013009F054C08981282F30E03D
:1044C0008881482F50E03BC08081918186179707F3
:1044D00061F5828193818A159B0539F5848181304C
:1044E00021F586819781A085B1850097A105B10549
:1044F000E1F0F90183E0EE0FFF1F8A95E1F7220F4B
:10450000331FE20FF31FEC0FFD1F84899589A689E5
:10451000B7898C159D05AE05BF0509F48FC0C48A07
:10452000D58AE68AF78A138B89C0C90101963A9623
:1045300020E030E08031910514F49C010EC0F901B7
:10454000EE0FFF1FC901A3E0880F991FAA95E1F79D
:10455000E80FF91F3E96EC0FFD1F2417350709F0F1
:10456000B3CFEFB7F8943881A32FB0E0898190E002
:104570000197A817B90741F03F3011F090E005C04E
:10458000898190E0882309F491E0EFBF992311F02D
:1045900080E055C0FD0193E0EE0FFF1F9A95E1F713
:1045A000AA0FBB1FEA0FFB1FEC0FFD1F7787668763
:1045B000888190E0FC0163E0EE0FFF1F6A95E1F750
:1045C000880F991FE80FF91FEC0FFD1FB18AA08A11
:1045D000888190E0FC0143E0EE0FFF1F4A95E1F770
:1045E000880F991FE80FF91FEC0FFD1F138B8881AF
:1045F00090E0FC0123E0EE0FFF1F2A95E1F7880F02
:10460000991FE80FF91FEC0FFD1F028B888190E0C6
:10461000FC01B3E0EE0FFF1FBA95E1F7880F991F79
:10462000E80FF91FEC0FFD1FC48AD58AE68AF78AC6
:1046300088818F5F8883803108F0188281E0DF9164
:10464000CF911F910F91FF90EF90DF90CF90BF908F
:10465000AF9008958091570990E0833009F491E07C
:10466000892F0895FC01009729F1818590E08370DE
:1046700090708330910534F48130910534F4892BA6
:1046800061F018C00397B1F404C0809137038160D2
:1046900007C080913703826003C080913703846034
:1046A000809337038091370390E08770873019F04B
:1046B00091E001C090E0892F089580933903089517
:1046C0008091370380720895809137038F7D8093A6
:1046D00037031092500310924F03089590934E03A6
:1046E00080934D031092500310924F0308958FB79B
:1046F000F8948FBF80914B0390914C0308958FB72E
:10470000F8948FBF80914F0390915003089578944F
:104710001F920F920FB60F920BB60F9211242F9388
:104720003F938F939F93EF93FF9380914A03883039
:1047300010F010924A0324B135B18091370384FF01
:1047400034C080914A03E82FF0E0EE0FFF1FE65CD3
:10475000FC4F318320838F5F80934A03EAE3F3E0C9
:1047600020E030E081919191280F391F83E0EA34F5
:10477000F807C1F730934C0320934B0380914F030C
:10478000909150038217930724F4309350032093A1
:104790004F0380914D0390914E03821793072CF4A1
:1047A00080913703806280933703FF91EF919F914F
:1047B0008F913F912F910F900BBE0F900FBE0F90D6
:1047C0001F901895982F03C0892F862311F4990FF5
:1047D000D9F7892F0895DC0152962C9152972430F5
:1047E00009F04CC053969C915397292F2150539612
:1047F0002C93539758968C915897813009F497C011
:10480000843009F494C0803209F491C0803809F4EE
:104810008EC08230E9F457968C915797883030F0EB
:1048200057961C92579753969C9325C0822F869536
:1048300086958695FD01E80FF11D808190E0277037
:1048400002C0959587952A95E2F780FD09C011C0B1
:10485000803179F0803469F0883011F4223048F4E6
:1048600057968C9157978F5F57968C9323E330E040
:1048700063C057961C922FEF3FEF5EC054968C9109
:1048800054978823C1F555968C915597882399F5AF
:1048900053963C915397932F915053969C935397D3
:1048A000233089F45C968C915C97882361F497702F
:1048B000973049F481E05C968C935C9753963C93D7
:1048C000539790E019C05C961C925C9753962C917C
:1048D0005397822F869586958695FD01E80FF11DE9
:1048E000808190E0277002C0959587952A95E2F720
:1048F000982F917001C091E052968C91823029F0EE
:10490000833099F08130B1F408C0992319F420E183
:1049100030E012C02CE530E00FC0992319F42CE1EF
:1049200030E00AC02EEB30E007C0992319F427E6E7
:1049300030E002C02BE330E0C9010895CF93DF934C
:10494000DC0152969C915297943009F0F2C058962F
:104950008C915897813039F0843029F0803219F0E9
:10496000803809F051C082E0A93FB80761F45C9635
:104970008C915C97882319F08FB58F7A02C08FB520
:1049800080658FBD0EC05C968C915C97882321F06A
:1049900080918B008F7A03C080918B00806580931B
:1049A0008B0053968C91539780FD03C0C7E6D0E0EF
:1049B0000CC090E05C968C915C97882309F491E0A0
:1049C0005C969C935C97CAE9D0E053968C91539780
:1049D0008823A1F458968C915897803879F482E016
:1049E000A93FB80721F48FB580658FBD05C08091C0
:1049F0008B00806580938B00CD5ED94F809137030B
:104A00008F7E8093370351C082E0A93FB807C1F47D
:104A100088B599B58736910540F090E080911503EF
:104A2000882309F491E0909315038091150388235E
:104A300019F08FB58F7A02C08FB580658FBD1FC00A
:104A400080918600909187008736910550F090E024
:104A50005C968C915C97882309F491E05C969C931A
:104A60005C975C968C915C97882321F080918B00F9
:104A70008F7A03C080918B00806580938B0058965D
:104A80008C915897803111F0803441F48091370334
:104A9000806180933703CDE4D8E107C0809137036C
:104AA0008F7E80933703C7E6D0E053968C9153975F
:104AB000882309F0D3C058969C915897923041F4BE
:104AC00057968C915797883018F0C7E6D0E0C6C04B
:104AD00059962C91599703C0892F822311F4990F6D
:104AE000D9F758969C93589757961C9257979031A0
:104AF000D1F0913140F4943091F0983091F09230AF
:104B000009F0ACC008C0903471F0903871F0903268
:104B100009F0A4C006C050968C91509707C08CE253
:104B200005C084E003C081E001C088E053968C9307
:104B300095C082E0A93FB80721F48FB580658FBD8D
:104B400005C080918B00806580938B0054968C917A
:104B50005497882331F455968C915597882331F4D6
:104B60000BC0815054968C93549704C08150559635
:104B70008C93559781E01CC0933039F45C968C91EE
:104B80005C97882311F080E013C053962C915397C3
:104B9000822F869586958695FD01E80FF11D80810F
:104BA00090E0277002C0959587952A95E2F781706D
:104BB00052969C915297923019F0933019F503C098
:104BC000CBE6D0E021C0882319F4CEECD0E002C0BF
:104BD000C7E7D0E053968C9153978823A9F45B964E
:104BE0008C915B97882381F48091390380FD02C00A
:104BF00082E001C086E055968C93559781E05B96E4
:104C00008C932CC0C7EDD0E053968C91539788239A
:104C100029F555968C915597882301F551968C91DD
:104C2000882399F48091370380FF18C0809138035E
:104C30008823A1F481E00E94CD6B882319F0C35B27
:104C4000DF4E0CC0CD5ED94F09C0913029F09230B3
:104C500029F4C857DD4F02C0C05FDA4FCE01DF91A3
:104C6000CF910895FC018089838B8189823010F473
:104C700082E0818B82898330D1F0843018F48130D6
:104C8000C0F00AC08430A9F482E0868B91E0908F56
:104C90008189882309F4918B81E00E94CD6B882360
:104CA00019F423E136E007C02DE430E104C080E1CF
:104CB000848B22E330E0C901089580E1EAE3F3E068
:104CC000DF011D928A95E9F710924A0310924C0376
:104CD00010924B038FEF9FE790934E0380934D0309
:104CE00008952F923F924F925F926F927F928F9290
:104CF0009F92AF92BF92CF92DF92EF92FF920F936B
:104D00001F93CF93DF935C014B01442428E0653A65
:104D1000720711F444244394D40111969C91119785
:104D20008C91891709F036C1442029F4809137030A
:104D300088608093370380913803813041F4C40147
:104D400060E070E040E050E022E000E882C0809146
:104D50003803823071F4C0903503D0903603EE24CE
:104D6000FF24C40160E070E040E050E021E000EC8E
:104D70000FC18091390382FF27C0F40182819381A2
:104D8000A481B5810097A105B105F1F4C40160E0EB
:104D900070E040E050E022E00EE8CC24DD24760113
:104DA0000E9448228091C5079091C607A091C7072D
:104DB000B091C80788519C4FAF4FBF4FF401828319
:104DC0009383A483B583E6C08091390381FF30C00B
:104DD000F40186819781A085B1850097A105B10571
:104DE00039F5C40160E070E040E050E021E00FE8F8
:104DF000CC24DD2476010E944822C40160E070E0EA
:104E000040E050E021E000E90E9448228091C5077F
:104E10009091C607A091C707B091C8078854944FD6
:104E2000AF4FBF4FF40186839783A087B187B2C08D
:104E3000442019F00E94403802C00E94613AEC01FF
:104E4000009759F4C40160E070E040E050E021E0D8
:104E500001E0CC24DD2476019BC0898590E083703D
:104E600090708230910541F0833091050CF469C057
:104E7000039709F08FC051C0C8840E943D3865E097
:104E80000E947AA7923029F1933030F4992351F09F
:104E9000913009F07FC011C0933039F1943009F09E
:104EA00079C02FC068817981DD24EE24FF24C401FC
:104EB00040E050E021E001E06BC068817981CC8066
:104EC000DD80EE80FF80C40140E050E021E001E49D
:104ED0005FC068817981CC80DD80EE80FF80C40175
:104EE00040E050E021E002E453C068817981CC8049
:104EF000DD80EE80FF80C40140E050E021E003E46B
:104F000047C068817981CC80DD80EE80FF80C4015C
:104F100040E050E021E004E43BC00E943D3890E0D6
:104F2000837090708130910581F0823091051CF47E
:104F3000892B39F02FC08230910599F0039751F5F4
:104F40001CC068817981C884AFCF68817981CC80A9
:104F5000DD80EE80FF80C40140E050E021E004E00D
:104F600017C068817981CC80DD80EE80FF80C4012C
:104F700040E050E021E005E00BC068817981CC8001
:104F8000DD80EE80FF80C40140E050E021E006E0DB
:104F90000E944822D40111962C911197822F90E003
:104FA000FC0153E0EE0FFF1F5A95E1F7880F991FA0
:104FB000E80FF91FE80DF91DC685D78511962C91CC
:104FC0001197822F90E0FC0133E0EE0FFF1F3A951E
:104FD000E1F7880F991FE80FF91FE80DF91D2088E8
:104FE000318811962C911197822F90E0FC0103E0FB
:104FF000EE0FFF1F0A95E1F7880F991FE80FF91FC1
:10500000E80DF91D028911962C91822F90E0FC0188
:10501000B3E0EE0FFF1FBA95E1F7880F991FE80F75
:10502000F91FE80DF91DC488D588E688F788802F18
:105030008C50823008F05BC0442049F18091C50754
:105040009091C607A091C707B091C80780935C09EB
:1050500090935D09A0935E09B0935F0980915C090C
:1050600090915D09A0915E09B0915F090097A1053B
:10507000B105A9F581E090E0A0E0B0E080935C0983
:1050800090935D09A0935E09B0935F0928C0809159
:10509000C5079091C607A091C707B091C807809334
:1050A000580990935909A0935A09B0935B098091CC
:1050B000580990915909A0915A09B0915B0900973C
:1050C000A105B10561F481E090E0A0E0B0E080933B
:1050D000580990935909A0935A09B0935B09CE01DE
:1050E0000E94638C582E6624772410E040C0809183
:1050F0003803813009F443C080913803823041F491
:10510000209709F48FC6CE010E948E383C018CC6D0
:10511000CE010E948E383C01009731F01C2DFC011D
:105120005184F3E05F2221C0802F90E0807C90705A
:105130008038910539F0803C910561F0803491050B
:1051400061F404C010E0E3E05E2E0FC010E05524CF
:1051500053940BC010E0552408C0D5011C9201E007
:1051600010E055245394C0E0D0E041101078552051
:1051700001F582E00E94CD6B8823C9F006C073E080
:10518000572E6624772410E014C0F401828593859D
:10519000A485B5850097A105B10511F0552409C076
:1051A00080913503909136036C0100EC69C1552460
:1051B0005394D40111963C91832F90E0FC0163E05D
:1051C000EE0FFF1F6A95E1F7880F991FE80FF91F8F
:1051D000E80DF91D23892150832F90E0FC0143E065
:1051E000EE0FFF1F4A95E1F7880F991FE80FF91F8F
:1051F000E80DF91D238B222309F035C18091580950
:1052000090915909A0915A09B0915B090097A105A5
:10521000B105C1F0609158097091590980915A09FE
:1052200090915B09685D7F4F8F4F9F4F0E941119CE
:10523000882341F0109258091092590910925A0986
:1052400010925B0980915C0990915D09A0915E09C3
:10525000B0915F090097A105B105C1F060915C09AB
:1052600070915D0980915E0990915F09685D7F4F43
:105270008F4F9F4F0E941119882341F010925C09B3
:1052800010925D0910925E0910925F09F40162812B
:10529000738184819581611571058105910559F0AE
:1052A0000E941119882339F0D40112961D921D9283
:1052B0001D921C921597F4016681778180859185F6
:1052C000611571058105910559F00E941119882316
:1052D00039F0D40116961D921D921D921C921997B9
:1052E000F401628573858485958561157105810555
:1052F000910559F00E941119882339F0D4011A96AA
:105300001D921D921D921C921D97442039F580918B
:10531000570980FD88C08091580990915909A09142
:105320005A09B0915B090097A105B10509F07BC04E
:10533000809157098160809357098091C5079091AA
:10534000C607A091C707B091C807809358099093EA
:105350005909A0935A09B0935B0926C08091570957
:1053600081FD61C080915C0990915D09A0915E0909
:10537000B0915F090097A105B10509F054C0809173
:1053800057098260809357098091C5079091C6079D
:10539000A091C707B091C80780935C0990935D09FD
:1053A000A0935E09B0935F09F401218140915309F4
:1053B00050915409822F90E0FC01B3E0EE0FFF1FE3
:1053C000BA95E1F7880F991FE80FF91FE80DF91D4D
:1053D00057874687D40111962C9111973091550922
:1053E000822F90E0FC0173E0EE0FFF1F7A95E1F74A
:1053F000880F991FE80FF91FE80DF91D328B1196E0
:105400002C9130915609822F90E0FC0153E0EE0F71
:10541000FF1F5A95E1F7880F991FE80FF91FE80D54
:10542000F91D338B20C0F4012181822F90E0FC0113
:1054300023E0EE0FFF1F2A95E1F7880F991FE80F71
:10544000F91FE80DF91D128AD40111968C9111975C
:105450008F5F11968C93119711968C9111978031D3
:1054600010F011961C92B2E0B51528F0E1E05E163E
:1054700008F097C105C0F3E05F1609F0D7C4B3C2C6
:105480008091370384608093370384E0D50152967E
:105490008C935A2C4B2C80E1D5011D928A95E9F70B
:1054A00091E0F501918B83E8818F908F013C09F4A5
:1054B0008FC0023C78F40330D1F0043020F4013086
:1054C00009F047C118C0043009F445C0003C09F098
:1054D00040C155C0033C09F4C9C0033C08F49FC057
:1054E000043C09F4E8C0053C09F033C110C1D30104
:1054F00018961C911F67812F90E08F77907000970E
:1055000031F08F37910511F4117801C01F5FF3015D
:105510002481358140E050E04760852D942D68E07E
:1055200004E10E94BD21682FD50150968C9310583C
:10553000212F30E03160442737FD4095542F852DD1
:10554000942D0BE00E94BD21482FF501808BCE01E8
:10555000652D742D0EC0960140E050E04760C501F6
:1055600068E004E10E94BD21482FF501808BCE0147
:10557000B5010E94EA21D50150968C93EAC0809132
:10558000C5079091C607A091C707B091C807805181
:10559000954FAF4FBF4FF40182879387A487B5879C
:1055A000960140E050E0C50168E000E10E94BD21A5
:1055B000682FC50124E332E140E050E000E20E94A0
:1055C000BD21682FC5012DE330E040E050E047C029
:1055D0009E0140E050E0A90133272227C101A0E04D
:1055E000B0E0282B392B4A2B5B2BC50168E000E289
:1055F0000E94BD21682F2C2D30E040E050E0C50115
:1056000006E00E94BD21682FC5012AE330E040E09A
:1056100050E00E94BD21482F80E090E044C09E01F0
:1056200040E050E0A90133272227C101A0E0B0E00B
:10563000282B392B4A2B5B2BC50168E000E20E9426
:10564000BD21682F960140E050E0C5010EE00E94A8
:10565000BD21682FC5012BE330E040E050E006E0BB
:105660000E94BD21482F80E090E082CF9E0140E063
:1056700050E0A90133272227C101A0E0B0E0282B88
:10568000392B4A2B5B2BC50168E000E20E94BD214B
:10569000682FC5012CE330E040E050E006E00E94B6
:1056A000BD21482FC601B5010E94EA21F501808B7A
:1056B0008FEF818F4EC0222D30E040E050E02F77F9
:1056C00030704070507072E0220F331F441F551F1E
:1056D0007A95D1F7386080E090E0A0E0B0E0CC208F
:1056E00021F081E090E0A0E0B0E0282B392B4A2B9C
:1056F0005B2B852D942D68E00CE00E94BD21482F86
:10570000D50150968C93CE01652D742D1EC091014C
:1057100040E050E06AE0220F331F441F551F6A9596
:10572000D1F7546E8C2D90E0A0E0B0E0282B392BFF
:105730004A2B5B2BC50168E000E20E94BD21482F87
:10574000D50150968C93CE01B5010E94EA21F50156
:10575000808BD50150962C91222309F467C3422FE8
:1057600041503FE767E051E017C0832F330F87FDBB
:105770003627842F869586958695F501E80FF11DCD
:10578000808190E0242F277002C0959587952A95F7
:10579000E2F780FD352741504F3F39F7F50130835F
:1057A00045C380913703816080933703D4011A96F3
:1057B0001D921D921D921C921D97802F8C5082303D
:1057C000B0F482E0F501828BFE0133E0F695E795B7
:1057D0003A95E1F7F070319621E0E030F20711F4EC
:1057E000E0E0F0E0EA5AFD4F949184E00FC081E0E0
:1057F000F501828BCF3FD10521F018F0E0E0F0E019
:1058000001C0FE01EA5AFD4F949182E0D501519604
:105810008C93892F8295869586958370F501828376
:10582000990F990F918382E1808B6114710409F4BF
:105830004AC0043041F0013431F0023421F0033425
:1058400011F0043491F4C60181709070892B39F005
:10585000D50111968C911197836011968C93F30169
:105860001085442051F0107808C0D30114968C9113
:1058700080FF03C09360F5019183812F90E08F77C3
:105880009070892B01F1D30119968C910E94FB3DF8
:105890000F97CCF01F5FF30181850E941138892B8F
:1058A00051F410FF08C0D50111968C91119791E029
:1058B000892711968C93812F90E08F719070959528
:1058C00087951078182B0E3070F40C30F8F40430F3
:1058D00030F4023070F5013009F0A8C225C0043060
:1058E00009F0A4C221C00234D1F1033430F40034F1
:1058F000D9F0013409F09AC229C0043409F44BC02C
:105900000434C8F1053409F091C255C0C770D07095
:10591000C25CDD4FFE012491D5012C930C3009F0BF
:1059200085C22C7F2C9382C2852D612F0E944C2131
:105930003FC0D30118966C9160786F60852D0E94EE
:105940004C21F501808384E0818B70C2F694E7944A
:10595000D794C7944C2D4170812F61E017C0B2E0FD
:10596000F694E794D794C794BA95D1F74C2D41702B
:10597000812F62E01BC0A3E0F694E794D794C7940C
:10598000AA95D1F74C2D4170812F63E00E94102120
:10599000D5018C934BC2F4E0F694E794D794C79466
:1059A000FA95D1F74C2D4170812F64E00E941021AF
:1059B000F50180833BC2D50111968C9111978360CC
:1059C00011968C93119782E052968C935297F6948D
:1059D000E794D794C794F601EF70F070EA5BFD4F3F
:1059E000E491EC9323C28091370382608093370364
:1059F000F4011286138614861586D50152965C92A0
:105A0000529781E051968C93519788E150968C93F0
:105A1000063818F5033808F049C1063009F4D0C03B
:105A2000073078F40330F1F1043020F4013009F04C
:105A3000E1C139C0043009F495C0053009F0DAC17C
:105A4000ADC0023808F02AC1003808F013C1802F19
:105A50008C50823008F0CEC119C0013950F40F3893
:105A600008F09DC10E3808F094C1083808F05AC1FA
:105A700041C1023909F4AFC0023908F4ABC103399E
:105A800009F4B6C0043909F0B5C1C8C040E00D3012
:105A900009F441E095012F5F3F4FCE0160E00E9485
:105AA0009421A8C11F67F30181858C70883099F417
:105AB0008FE3D50112968C93812F90E08F779070B1
:105AC000009731F08F37910511F4117801C01F5FF5
:105AD000F5011183B8C017FF04C080E6F50181838A
:105AE00004C080E4D50111968C93F30181850E9456
:105AF000FB3D212F30E00F97E4F0C9018F779070C4
:105B0000009731F08F37910511F412E001C01D5F4D
:105B1000912F96959F70D50111968C911197982B86
:105B200011969C93119710FF46C0906111969C931B
:105B300042C0C9018F779070009731F08F3791057F
:105B400011F411E001C01F5F212F2F70F501818139
:105B5000282B2183D30114968C9180FF2CC02061C7
:105B6000218329C0D701C601B695A795979587953A
:105B70008F708068D50111968C93C60181709070EA
:105B8000892BC9F0F30181850E94FB3D0F979CF0A2
:105B9000D50111968C91119780610BC065E0F69448
:105BA000E794D794C7946A95D1F78C2D8F70806B4A
:105BB000D50111968C93B5016E5F7F4FCE016BC0FE
:105BC00059E0F694E794D794C7945A95D1F78C2D61
:105BD0008F70806AEDCF4DE0F694E794D794C79428
:105BE0004A95D1F7D5011196CC9211978EED0CC044
:105BF00035E1F694E794D794C7943A95D1F7D50157
:105C00001196CC9211978FED12968C93B5016D5F22
:105C10007F4FCE010E948521885EEAC0822D8F775A
:105C2000D50111968C931197C114D104E104F104AC
:105C300019F0806811968C93B0E82B16310470F43B
:105C40008DEDF5018283B5016D5F7F4FCE010E941E
:105C50008521885ED50150968C93CCC0F501818159
:105C60008283220C232C221C33083194218280EC65
:105C7000838387C0F501118295012E5F3F4F013864
:105C800041F4CE01816060E040E00E949421805F99
:105C9000E1CFCE01B9010E948521A9C08FEFD501C6
:105CA00012968C93129711961C92A4C0053811F489
:105CB00088E708C0043829F484E7D50113968C934B
:105CC00003C08CE7F50183834E01992D9370D501B4
:105CD00013968C911397892B13968C931397129686
:105CE000CC9312971196CC92119780E250968C9398
:105CF000509714C080E7F5018283063811F488E7D5
:105D000082839E012770D50112969C911297922B47
:105D100012969C9312971196CC9211978AE0519605
:105D20008C9368C0802F8B58833030F4832D837020
:105D3000846EF501838306C0832D83708C6ED5013C
:105D400013968C93F5012282C182093811F00C3828
:105D500051F495012C5F3F4FCE01816060E040E03F
:105D60000E94942114C00A3811F00D3851F49501A5
:105D70002C5F3F4FCE0161E040E00E949421805EA5
:105D800037C0B5016C5F7F4FCE010E948521805ED8
:105D900061CF8FEBF50182838FE081832BC00E945E
:105DA000D46B8FEFD50115968C93159714968C9321
:105DB00014978EE313968C93139712967C931297F5
:105DC00011966C931197003919F48FE714968C9300
:105DD00080E30EC08C2D8F71D50111968C939501A7
:105DE0002E5F3F4FCE0161E040E00E949421805F32
:105DF000F501808BD50150969C9196959695969538
:105E00009150E92FFF27E7FDF095EA0DFB1D20E0FB
:105E100004C080812827915031971916D4F3F501D9
:105E2000208304C06624772410E0A3C9DF91CF91BA
:105E30001F910F91FF90EF90DF90CF90BF90AF90A8
:105E40009F908F907F906F905F904F903F902F909A
:105E500008951F920F920FB60F920BB60F92112456
:105E60000F931F932F933F934F935F936F937F9362
:105E70008F939F93AF93BF93EF93FF9380913403DE
:105E80008823B1F08091370380FD07C08BE390E059
:105E9000909387008093860004C010928700109230
:105EA000860087E790E0909381008093800075C022
:105EB00087E193E00E949E24AC01209188003091FC
:105EC000890005972817390728F4509381004093DB
:105ED000800017C08091880090918900C2969093AD
:105EE000810080938000009188001091890087E1F3
:105EF00093E00E943226080F191F1093810000932F
:105F0000800080912A03882309F03FC080912C03F0
:105F10008823D9F580912F038823B9F58091280330
:105F2000882399F481E08093340380917C0084601D
:105F300080937C001FB7789487E193E065EA78E06E
:105F40000E9471261FBF1092340380912803815054
:105F5000809328038091270380932A03909129033B
:105F6000933021F480E180932B0309C0943029F40D
:105F700081E080932F0390932A0310922B031092B9
:105F80002C03109233031092320387E193E00E94B6
:105F9000EB239093870080938600FF91EF91BF9150
:105FA000AF919F918F917F916F915F914F913F91B1
:105FB0002F911F910F910F900BBE0F900FBE0F905E
:105FC0001F9018951F920F920FB60F920BB60F925B
:105FD00011240F931F932F933F934F935F936F93CE
:105FE0007F938F939F93AF93BF93EF93FF93809192
:105FF0003803882331F08091370385FF02C0109267
:106000000A03809116038823A1F08091370380FD55
:1060100005C08BE390E099BD88BD02C019BC18BCD7
:106020008BE390E09BBD8ABD87E790E097BD86BD7E
:1060300070C089EF92E00E949E24AC012CB53DB562
:1060400005972817390718F457BD46BD0FC08CB502
:106050009DB5C29697BD86BD0CB51DB589EF92E082
:106060000E943226080F191F17BD06BD80910C0330
:10607000882309F044C080910E03882309F03FC0B3
:10608000809111038823D9F580910A03882389F42C
:1060900081E08093160386B7846086BF1FB778942B
:1060A00089EF92E067EF77E00E9471261FBF1092A0
:1060B000160380910A03815080930A03809109039B
:1060C00080930C0390910B03933051F4809138032B
:1060D000882311F084E101C080E180930D0309C0A1
:1060E000943029F481E08093110390930C03109273
:1060F0000D0310920E03109215031092140389EFF2
:1061000092E00E94EB239BBD8ABD8AB59BB599BDE9
:1061100088BDFF91EF91BF91AF919F918F917F913A
:106120006F915F914F913F912F911F910F910F9020
:106130000BBE0F900FBE0F901F9018950E94681213
:10614000833020F0853020F0873011F081E0089511
:1061500080913703887008950E94C06BFC01808194
:1061600082FF0DC096B3809163009095991F992787
:10617000991F8695869586958095817009C086B30E
:1061800090916300969596959695909591708078EC
:10619000982B892F08950E94C06BFC01808182FF9B
:1061A00002C0C79A0895C79808959C018091570925
:1061B000833011F080E008953093540920935309FF
:1061C000662311F08DE001C08CE08093550983E0D7
:1061D00080935609109257090E94C06BFC01808180
:1061E00086FF05C08091570981608093570980819F
:1061F00087FD02C081E008958091570982608093F5
:10620000570981E008952F923F924F925F926F92CB
:106210007F928F929F92AF92BF92CF92DF92EF9236
:10622000FF920F931F93CF93DF93EC012B013A0161
:10623000222E302E46015701009731F485EA98E06E
:106240000E940331C7EFD7E080913803882321F003
:1062500088E0C53AD80701F10E9468128230E0F068
:10626000853010F08730C1F41FB7F894CE01B20129
:10627000A301222D032D750164010E9448221FBF36
:10628000882329F485E090E00E947419E5CF80917D
:106290003703877F80933703DF91CF911F910F9151
:1062A000FF90EF90DF90CF90BF90AF909F908F9036
:1062B0007F906F905F904F903F902F900895CF9276
:1062C000DF92EF92FF920F93982F809138038823EB
:1062D000E9F59923D9F11092F8078091F807809396
:1062E000F7078EE1E9EFF2E0DF011D928A95E9F709
:1062F0000E946812873031F4809137038160809367
:10630000370311C082E393E20E941B3887EF97E0C6
:1063100060E070E040E050E02AE002E8CC24DD24B8
:1063200076010E9403318BE390E099BD88BD88B56A
:1063300099B59BBD8ABD87E790E097BD86BD1DBC22
:106340001CBC87B7846087BFBE9A05C0BE98C6983C
:1063500087B78B7F87BF0F91FF90EF90DF90CF9033
:106360000895CF92DF92EF92FF920F93982F809132
:106370003803882399F5992389F11092A608809112
:10638000A6088093A5088EE1E7E1F3E0DF011D9206
:106390008A95E9F785EA98E060E070E040E050E037
:1063A00022E002E8CC24DD2476010E9403318BE355
:1063B00090E0909387008093860087E790E0909329
:1063C0008100809380001092890010928800809153
:1063D0007D00846080937D00139A07C013981B98FA
:1063E00080917D008B7F80937D000F91FF90EF90D7
:1063F000DF90CF9008951F93182F8823E1F180E05C
:106400000E945F3180E00E94B13181E064E00E942F
:106410008490809162008B7F809362008EE1E9EF2F
:10642000F2E0DF011D928A95E9F782E0809337035D
:1064300083E080930B038FEF8093F9028BE390E06E
:1064400099BD88BD88B599B59BBD8ABD87E790E0A9
:1064500097BD86BD1092F8078091F8078093F707E3
:1064600010933803BD9A87B7846087BF82E090E0BD
:106470000E94D71907C087B78B7F87BF1092380358
:10648000BD98C5981F91089581E00E94FB318091CD
:106490003703806180933703089580E00E94FB31C9
:1064A000E2E6F0E080818B7F808380E00E945F31B4
:1064B00080E00E94B13181E064E00E948490089500
:1064C000CF92DF92EF92FF920F93009711F485EA3B
:1064D00090E090933603809335036C01EE24FF2403
:1064E00087EF97E060E070E040E050E024E000ECEF
:1064F0000E9403310F91FF90EF90DF90CF900895AD
:1065000082E00E94FB31809137038F7E80933703B6
:106510008091C5079091C607A091C707B091C807A1
:1065200090E00E9460320895CF92DF92EF92FF9246
:106530000F931F938B019C016A01A901662777279E
:10654000EE24FF2487EF97E0BA01A80122E003ECD4
:106550000E94033181E01F910F91FF90EF90DF9037
:10656000CF900895CF92DF92EF92FF920F931F93F7
:106570008B019C016A01A90166277727EE24FF247D
:1065800087EF97E0BA01A80122E002EC0E940331F4
:1065900081E01F910F91FF90EF90DF90CF900895D1
:1065A000CF92DF92EF92FF920F931F938B019C018A
:1065B000C42EAC0166277727DD24EE24FF2487EF65
:1065C00097E0BA01A80122E001EC0E94033181E0CA
:1065D0001F910F91FF90EF90DF90CF900895CF9291
:1065E000DF92EF92FF920F93FC01613091F06130E6
:1065F00018F0623049F51AC0002309F400E4C22EF5
:10660000DD24EE24FF2480E090E0BF01202F0BE882
:1066100019C0002309F400E1C22EDD24EE24FF247A
:1066200080E090E0BF01202F0CE80CC0002309F4AB
:1066300000E1C22EDD24EE24FF2480E090E0BF01C3
:10664000202F0DE80E94033181E00F91FF90EF9021
:10665000DF90CF900895CF92DF92EF92FF920F9349
:10666000FC01613091F0613018F0623049F51AC0D8
:10667000002309F400E4C22EDD24EE24FF2480E090
:1066800090E0BF01202F08E819C0002309F400E1C1
:10669000C22EDD24EE24FF2480E090E0BF01202FF5
:1066A00009E80CC0002309F400E1C22EDD24EE2429
:1066B000FF2480E090E0BF01202F0AE80E94033110
:1066C00081E00F91FF90EF90DF90CF900895CF92EF
:1066D000DF92EF92FF920F939C01809138038130FB
:1066E00011F080E00EC0C62EDD24EE24FF2487EFDB
:1066F00097E0B90140E050E021E004E80E94033156
:1067000081E00F91FF90EF90DF90CF900895CF92AE
:10671000DF92EF92FF920F939C01809138038130BA
:1067200011F080E00EC0C62EDD24EE24FF2487EF9A
:1067300097E0B90140E050E021E003E80E94033116
:1067400081E00F91FF90EF90DF90CF900895CF926E
:10675000DF92EF92FF920F939C018091380381307A
:1067600011F080E00EC0C62EDD24EE24FF2487EF5A
:1067700097E0B90140E050E021E007E80E940331D2
:1067800081E00F91FF90EF90DF90CF900895CF922E
:10679000DF92EF92FF920F939C018091380381303A
:1067A00011F080E00EC0C62EDD24EE24FF2487EF1A
:1067B00097E0B90140E050E021E006E80E94033193
:1067C00081E00F91FF90EF90DF90CF900895CF92EE
:1067D000DF92EF92FF920F939C01809138038130FA
:1067E00011F080E015C06770862F806E442311F091
:1067F000862F886EC82EDD24EE24FF2487EF97E0D5
:10680000B90140E050E021E005E80E94033181E059
:106810000F91FF90EF90DF90CF900895CF92DF928D
:10682000EF92FF920F939C0180913803813011F019
:1068300080E015C06770862F806F442311F0862F8B
:10684000886FC82EDD24EE24FF2487EF97E0B9017E
:1068500040E050E021E005E80E94033181E00F9123
:10686000FF90EF90DF90CF900895CF92DF92EF925C
:10687000FF920F93282F80E090E060E070E040E00E
:1068800050E002E8CC24DD2476010E94033181E04F
:106890000F91FF90EF90DF90CF900895CF92DF920D
:1068A000EF92FF920F93FC01242F662311F400E86E
:1068B00001C001E880E090E0BF0140E050E0CC245E
:1068C000DD2476010E94033181E00F91FF90EF906B
:1068D000DF90CF900895CF92DF92EF92FF920F93C7
:1068E0009C01C62EDD24EE24FF2480E090E0B90157
:1068F00040E050E021E001E90E94033181E00F9186
:10690000FF90EF90DF90CF9008952F923F924F929B
:106910005F926F927F928F929F92AF92BF92CF922F
:10692000DF92EF92FF920F931F93DF93CF93CDB738
:10693000DEB72A970FB6F894DEBF0FBECDBF1C019D
:106940002A013B0148015901009709F493C1DC0178
:1069500019968C9190E0837090708130910571F060
:106960008230910524F4892B09F41CC183C1823043
:10697000910591F1039709F07DC198C08426952671
:10698000A626B726C40181709070892B69F0F101A9
:106990006081718180E090E040E050E024E004E01C
:1069A000730162010E9403318EE190E0A0E0B0E04B
:1069B00088229922AA22BB2281149104A104B10445
:1069C00009F458C1D1016D917C9180E090E040E0E4
:1069D00050E024E005E4E1C0D901C80184279527EF
:1069E000A627B7278D839E83AF83B8878D819E812D
:1069F00081709070892B69F0D1016D917C9180E05C
:106A000090E040E050E024E004E0730162010E9465
:106A10000331BD81B1FF0DC0F1016081718180E062
:106A200090E040E050E024E001E4730162010E9444
:106A30000331FD81F2FF0DC0D1016D917C9180E0A9
:106A400090E040E050E024E002E4730162010E9423
:106A5000033188E090E0A0E0B0E088229922AA22E9
:106A6000BB22D301C20184709070A070B0708816F0
:106A70009906AA06BB0669F0D1016D917C9180E070
:106A800090E040E050E024E003E4730162010E94E2
:106A90000331BD81B4FFEEC0F1016081718180E0FE
:106AA00090E040E050E024E004E477C0842695269E
:106AB000A626B726D501C4018F719070A070B07062
:106AC0000097A105B10569F0D1016D917C9180E03D
:106AD00090E040E050E024E004E0730162010E9495
:106AE0000331D501C401807E9170A070B070009711
:106AF000A105B10569F0F1016081718180E090E04C
:106B000040E050E024E005E0730162010E9403319F
:106B1000D501C40180709E71A070B0700097A1056E
:106B2000B10569F0D1016D917C9180E090E040E089
:106B300050E024E006E0730162010E940331D501B8
:106B4000C4018070907EAF71B0700097A105B1054F
:106B500069F0F1016081718180E090E040E050E0F7
:106B600024E002E9730162010E94033180E090E0B9
:106B7000A0EEBFE188229922AA22BB2281149104AF
:106B8000A104B10409F476C0D1016D917C9180E03B
:106B900090E040E050E024E003E9730162010E94CC
:106BA000033168C0D901C80184279527A627B727D4
:106BB00089839A83AB83BC83892BA9F0D1016D9122
:106BC0007C911FEFC12E1FEFD12EE12CF12CC420A0
:106BD000D520E620F72080E090E040E050E023E080
:106BE00004E00E94033189819A81AB81BC8180706D
:106BF00090700097A105B105E9F1812C912CB1E0CD
:106C0000AB2EB12CE0E1F0E0FA87E98789819A8127
:106C1000AB81BC8188219921AA21BB210097A105C4
:106C2000B105E9F0D1016D917C91CC24DD24760190
:106C3000D501C40184219521A621B7210097A10582
:106C4000B10529F0A1E0CA2ED12CE12CF12C80E075
:106C500090E049855A8523E004EC0E940331880CBA
:106C6000991CAA1CBB1CE985FA85EF31F10511F0CE
:106C70003196CACF81E02A960FB6F894DEBF0FBED8
:106C8000CDBFCF91DF911F910F91FF90EF90DF90DB
:106C9000CF90BF90AF909F908F907F906F905F90BC
:106CA0004F903F902F900895CF92DF92EF92FF92F6
:106CB0000F937C010E948E38FC01009739F1818589
:106CC000282F30E02370307021303105FCF0233064
:106CD000310584F023303105C9F40E94FB3D0E9745
:106CE000A9F480E090E060E070E040E050E021E056
:106CF00002E807C080E090E0B70140E050E027E004
:106D000002E0CC24DD2476010E94033181E00F9162
:106D1000FF90EF90DF90CF900895CF92DF92EF92A7
:106D2000FF920F93CF93DF93EC010E948E38FC010A
:106D3000009761F1818583708150C084823090F426
:106D4000DD24EE24FF2480E890E0A0E0B0E0C8223B
:106D5000D922EA22FB2280E090E0BE0140E050E030
:106D60002BE011C0DD24EE24FF2480E890E0A0E0B9
:106D7000B0E0C822D922EA22FB2280E090E0BE01E6
:106D800040E050E024E003E00E94033181E0DF9125
:106D9000CF910F91FF90EF90DF90CF900895CF9219
:106DA000DF92EF92FF920F93CF93DF93EC01C62E09
:106DB0000E948E38892B61F0DD24EE24FF2487EFBA
:106DC00097E0BE0140E050E026E000E40E9403317D
:106DD00081E0DF91CF910F91FF90EF90DF90CF9006
:106DE0000895CF92DF92EF92FF920F931F93CF936C
:106DF000DF938C01C62E0E948E38EC010097C1F102
:106E0000898590E0837090708330910534F48130EF
:106E1000910534F4892B79F02BC0039749F50BC009
:106E2000DD24EE24FF2487EF97E0B80140E050E036
:106E300024E001E01BC0DD24EE24FF2487EF97E06F
:106E4000B80140E050E022E001E00E940331898572
:106E50008F70833069F480E090E060E070E040E0A3
:106E600050E021E002E8CC24DD2476010E940331C9
:106E700081E0DF91CF911F910F91FF90EF90DF9014
:106E8000CF90089583E08093570910925C09109287
:106E90005D0910925E0910925F0980915C099091E2
:106EA0005D09A0915E09B0915F09809358099093A4
:106EB0005909A0935A09B0935B098091C507909135
:106EC000C607A091C707B091C80788519C4FAF4F24
:106ED000BF4F8093F9079093FA07A093FB07B093F5
:106EE000FC078093A7089093A808A093A908B093E3
:106EF000AA088091C5079091C607A091C707B091D5
:106F0000C8078854944FAF4FBF4F8093FD079093AD
:106F1000FE07A093FF07B09300088093AB089093FF
:106F2000AC08A093AD08B093AE081092010810927F
:106F3000020810920308109204081092AF081092F1
:106F4000B0081092B1081092B20885EA90E09093D0
:106F500036038093350380E00E94FB310E94C76BAB
:106F6000809339031092370381E00E945F3181E002
:106F70000E94B131E2E6F0E0808184608083089570
:106F8000CF92DF92EF92FF920F937C01062F0E9427
:106F9000B63883708150823060F487EF97E0B70194
:106FA00040E050E0202F02E0CC24DD2476010E9456
:106FB000033181E00F91FF90EF90DF90CF90089523
:106FC000CF92DF92EF92FF920F931F93CF93DF93B5
:106FD000EC018B01C42E0E94B6388370833011F00F
:106FE00080E00CC0DD24EE24FF2480E090E0BE01B0
:106FF000A80124E004E90E94033181E0DF91CF91F0
:107000001F910F91FF90EF90DF90CF90089520E0B7
:1070100030E08F708950823010F421E030E0C901F7
:10702000089520E030E08F708550823010F421E028
:1070300030E0C9010895EF92FF920F931F93CF9311
:10704000DF937C0100E619E0C0E0D0E00BC02196A0
:10705000E114F10429F0C801F7010995882329F00A
:10706000055F1F4FC034D10591F7CE01DF91CF915D
:107070001F910F91FF90EF90089580915303089511
:107080009091200C992319F420E030E011C08091F8
:1070900052038F5F80935203891710F010925203AE
:1070A000909152038BE0989F90011124205A364F03
:1070B000C9010895CF92DF92EF920F931F93CF9360
:1070C000DF93EC01162F6901442361F00E94C76B26
:1070D0008823E1F0CE01612FA601202F0E2D0E9402
:1070E000EF3205C0A901202F0E2D0E942B33EE2078
:1070F00069F484E00E94353460E0111161E0CE0152
:1071000041E00E944E348AE00E943534DF91CF91F5
:107110001F910F91EF90DF90CF900895CF93DF9361
:10712000EC010E946812873019F424E533E01AC09C
:107130002097B1F03091200CE0E6F9E020E00EC09D
:10714000808191813B968C179D0739F48BE0289FB5
:1071500090011124205A364F05C02F5F231780F36A
:1071600020E030E0C901DF91CF9108950E948E3870
:10717000FC01009711F480E0089581858F700895D7
:107180008F929F92AF92BF92CF92DF92EF92FF9237
:107190000F931F93DF93CF9300D000D000D0CDB7D3
:1071A000DEB74C01062F0E946812873009F447C0F1
:1071B000C4010E948E385C01009709F440C07E0132
:1071C0000894E11CF11CC701B4010E94256FF50170
:1071D00024813581468157810023B9F0C701BA0166
:1071E000A9010E94316F8FEF6DE0A7010E94E36F4C
:1071F000F50124813581468157819A01442755271D
:10720000C401B9010E94C43E1AC0C701F5016085DE
:1072100000E00E944A6F8FEF6AE0A7010E94E36FCF
:10722000F501C480D580E680F780870122273327C7
:107230000170C4016085A601202F0E94EC3E2696B5
:107240000FB6F894DEBF0FBECDBFCF91DF911F9177
:107250000F91FF90EF90DF90CF90BF90AF909F90F5
:107260008F9008951F93CF93DF93C0E6D9E010E08D
:107270001BC08A85989FC00111248035910534F088
:10728000888590E08F779070892B61F08885807871
:107290008887888199810E948D368881998160E0F4
:1072A0000E94C0381F5F2B969091200C191708F38D
:1072B000DF91CF911F9108958F929F92AF92BF92CD
:1072C000CF92DF92EF92FF920F931F93DF93CF93B2
:1072D0000F92CDB7DEB74C017A018B01922F81144A
:1072E0009104E1F1F401A480B580C680D780A41692
:1072F000B506C606D70691F1243061F429830E94B1
:1073000068129981873031F5F401E482F5820683B1
:10731000178324C0F4011286992329F081858062A5
:107320008187913031F0F4018185806481879430C8
:1073300021F0F401818580618187F401E482F58286
:1073400006831783C401B801A701960185010E9435
:10735000853404C0F401818584FFDCCF0F90CF9188
:10736000DF911F910F91FF90EF90DF90CF90BF9032
:10737000AF909F908F900895EF92FF920F931F937D
:10738000CF93DF93EC01162F042F009709F492C0DE
:10739000443051F40E946812873009F087C0188782
:1073A00089C08F7E898786C089850E94FB3D482FD2
:1073B0005985812F90E08F779070242F30E0281727
:1073C000390714F41078142B6885611709F472C01A
:1073D0001A86002329F0898580628987013029F087
:1073E000898580648987043019F08985806189875F
:1073F000E62EFF24812F862787FF34C097012F7741
:1074000030702115310509F01078852F8370833095
:1074100011F08823D1F4232B29F0888199810E94CF
:107420008D3610C089858C70883061F4812F90E092
:107430008F779070892B31F4612F616088819981F9
:107440000E94F136888199810BC088819981232B14
:1074500039F00E94F136888199810E948D3602C0F0
:107460000E9454361887212F30E0C9018F77907021
:10747000892BB1F089858F708550823088F410FD9A
:1074800003C0612F6F5F08C00894E108F1082E1552
:107490003F0531F4612F6150888199810E94CF3678
:1074A00088819981612F0E94F13604C0898584FF0B
:1074B0007BCF77CFDF91CF911F910F91FF90EF900E
:1074C00008950F931F93CF93DF930E946812873024
:1074D00041F4809153038F5F80935303C4E5D3E05D
:1074E0001DC09091200C992319F4C0E0D0E04EC04B
:1074F000809151038F5F80935103891738F08091F9
:1075000053038F5F80935303109251039091510363
:107510008BE0989FE0011124C05AD64F809153030D
:1075200090E087709070892BA1F46885262F30E059
:10753000C9018F779070892B61F089858F70855094
:10754000823038F460FD05C06F5F888199810E94A8
:10755000CF36809153038770843099F48985837086
:10756000813079F44C815D816E817F810EE110E084
:1075700020E030E00427152726273727CE010E9478
:1075800085348A858F3F11F08F5F8A87CE01DF9126
:10759000CF911F910F91089580EC92E0E0E6F9E021
:1075A000DF019C011D9221503040E1F710925203FF
:1075B000109251031092200C08959F92AF92BF92A7
:1075C000CF92DF92EF92FF920F931F93DF93CF93AF
:1075D00000D00F92CDB7DEB76C01962E009719F44C
:1075E00000E010E028C020E2E22EF12C00E010E0E4
:1075F0005E010894A11CB11CA895C501B70143E028
:1076000050E00E94FCAB69817A81CB0101978F5FCA
:107610009F4340F4892D4B8120E030E0F60109952D
:107620000F5F1F4F84E090E0E80EF91E9CEDE91615
:107630009FE0F90609F7C8010F900F900F90CF91C6
:10764000DF911F910F91FF90EF90DF90CF90BF904F
:10765000AF909F900895AF92BF92CF92DF92EF923A
:10766000FF920F931F93DF93CF93CDB7DEB727978A
:107670000FB6F894DEBF0FBECDBF8FEF9FEFAFEF19
:10768000BFEF8C839D83AE83BF8300E210E05E0179
:107690000894A11CB11C34E0C32ED12CCC0EDD1EED
:1076A000F02EE12EC501B80143E050E00E94FCAB92
:1076B00089819A818F5F9F4F19F48B818F3F39F0B9
:1076C000C6016F2D7E2D44E050E00E9414AC0E9454
:1076D0006F120C5F1F4F8FE00C3D180709F72796BC
:1076E0000FB6F894DEBF0FBECDBFCF91DF911F91D3
:1076F0000F91FF90EF90DF90CF90BF90AF900895E3
:10770000CF92DF92EF92FF920F931F93DF93CF936D
:1077100000D00F92CDB7DEB78C01009709F441C0BD
:10772000FC018081918101978F5F9F4310F540E2BA
:10773000E42EF12C6E010894C11CD11CA895C60141
:10774000B70143E050E00E94FCAB29813A81F80187
:10775000808191812817390719F48B818F7020C09F
:1077600084E090E0E80EF91E9CEDE9169FE0F90632
:1077700029F7F80180819181F8E280309F0718F0A5
:10778000F80111860EC08F3F910509F028F488E0BA
:107790000E94CD6B882311F087E001C082E0F801E0
:1077A00081870F900F900F90CF91DF911F910F91D4
:1077B000FF90EF90DF90CF900895FF920F931F936B
:1077C000CF93DF938C01F62E0E9468128730E9F484
:1077D00080915403909155038017910709F455C087
:1077E000109355030093540384E593E00E94803B7B
:1077F00080915D0390E0837090700197029708F488
:1078000044C082E080935D0340C0C80101978F5F50
:107810009F4318F0C0E0D0E03CC0C8010E948E3801
:10782000AC010097A9F52091200C203450F48BE096
:10783000289FE0011124C05AD64F2F5F2093200CBF
:1078400010C0E0E6F9E0EF0192858A85891708F417
:10785000EF013B968CE0E032F807B1F78A85882388
:10786000B9F019830883CE010E94803B80E88887A5
:107870001C821D821E821F821B821A821A86FF2092
:1078800041F0C8010E94E58604C0C4E5D3E001C010
:10789000EA01CE01DF91CF911F910F91FF900895E2
:1078A000CF92DF92EF92FF921F93CF93DF936B0102
:1078B0005FEFE52E5FE7F52EE822F922C70160E0D1
:1078C0000E94DD3BEC010097E1F018851078D7FCB1
:1078D00010588FEF9FE7C822D922C60160E00E94AE
:1078E000DD3BFC01009769F080858F77182B1087AE
:1078F000DB82CA821A86F382E2821286C7010E9464
:107900003586DF91CF911F91FF90EF90DF90CF9060
:10791000089561E00E94DD3B0895CF93DF93EC0171
:107920000E9417860BC0CE010E94893CFC01009783
:1079300039F0C281D381138212821286209799F77F
:10794000DF91CF910895CF93DF93C0E6D9E08A818C
:107950009B81892B21F0888199810E948D3C8CE04C
:10796000C531D80711F02B96F2CFDF91CF91089552
:10797000DF92EF92FF920F931F937A018B01D22E29
:107980000E94893C009729F0B801A7012D2D0E9483
:107990005C391F910F91FF90EF90DF9008951F9336
:1079A000CF93DF93EB01142F0E94893CFC010097D9
:1079B000A1F0AE0160E070E0BA0155274427848150
:1079C0009581A681B781A070B070482B592B6A2B86
:1079D0007B2BCF01212F0E945C39DF91CF911F912A
:1079E00008951F93CF93DF93EB01142F0E94893CDE
:1079F000FC01009789F0AE0160E070E08481958120
:107A0000A681B78180709070482B592B6A2B7B2BF5
:107A1000CF01212F0E945C39DF91CF911F910895F2
:107A20000E94893CFC01009729F420E030E040E00E
:107A300050E004C02481358146815781B901CA01D3
:107A400008950E94893CFC01009711F480E008959C
:107A500080850895FF920F931F93CF93DF93EC01DE
:107A6000062FF42E0E946812833041F00E946812A3
:107A7000873021F084E0F81609F40078CE010E94E6
:107A8000893CEC010097C1F01885602F4F2D0E94B2
:107A9000BC398A819B81009779F060E00E94DD3BD0
:107AA000FC01009749F08085182717FD0058CF0189
:107AB000602F4F2D0E94BC39DF91CF911F910F9104
:107AC000FF9008958F929F92BF92CF92DF92EF9294
:107AD000FF920F931F93DF93CF9300D00F92CDB7F8
:107AE000DEB76C01B62E2FE0B22251F482E00E9484
:107AF000CD6B882329F482E00E94526E0E942C6E86
:107B000000E210E0EE24EA94FE2C4E010894811C61
:107B1000911CA895C401B80143E050E00E94FCAB61
:107B200089819A818C159D0511F478010FC02FEF82
:107B3000E2162FEFF20621F48050904408F078010D
:107B40000C5F1F4F8FE00C3D180719F729813A8110
:107B50002C153D0541F08FEFE8168FEFF80619F46C
:107B60002FEF3FEF17C08B818B1519F42C153D05B6
:107B700079F0BB82DA82C982A895CE010196B7015D
:107B800044E050E00E9414ACC6016B2D0E94F984C1
:107B900020E030E0C9010F900F900F90CF91DF915E
:107BA0001F910F91FF90EF90DF90CF90BF909F902B
:107BB0008F9008951F93CF93DF93EC01162F0E94AF
:107BC000893CFC01009799F0412F4F706185862F09
:107BD00090E08F709070242F30E08217930739F077
:107BE000607F642B61871286CE010E94623DDF9127
:107BF000CF911F910895E82FF0E0EF70F070E85EEC
:107C0000FB4FE4918E2F90E0089590E08370907088
:107C1000009731F0039711F48CE1089584E0089502
:107C20008FE1089584E693E008958091800382FFB8
:107C300005C0809166039091670308958091640365
:107C40009091650308958091800381FD0CC082604E
:107C5000877F809380031092840380E090E060E04F
:107C600070E00E94691E08958823E9F082E06EE6C4
:107C700071E00E940B2083E066E771E00E940B2018
:107C800084E06EE771E00E940B2085E066E871E019
:107C90000E940B2086E06EE871E00E940B2087E0D6
:107CA00066E971E01CC082E06EE271E00E940B2088
:107CB00083E06EE371E00E940B2084E06EE471E0EB
:107CC0000E940B2085E066E571E00E940B2086E0B3
:107CD0006EE571E00E940B2087E066E671E00E948D
:107CE0000B20089580916303833014F01092630396
:107CF000809163038F5F809363038150813041F0F3
:107D0000823061F0882379F481E066E372E003C099
:107D100081E06EE272E00E940B20089581E066E24D
:107D200072E00E940B200895882321F082E066EB28
:107D300071E003C082E06EEA71E00E940B200895BA
:107D4000882321F081E066EA71E003C081E06EE9FA
:107D500071E00E940B200895809394030E946B129F
:107D600008952091800321FD0EC02B7F2160209378
:107D70008003909367038093660370936F0360930F
:107D80006E030E946B120895E0916403F091650305
:107D90008E179F0711F0EF2BF1F49B0140E050E0AC
:107DA000A9013327222780916A0390916B03A09148
:107DB0006C03B0916D03A070B070282B392B4A2B47
:107DC0005B2B20936A0330936B0340936C035093B7
:107DD0006D030E946B120895FC01809164039091E1
:107DE0006503E817F90711F5109283036093820386
:107DF00060E070E080916A0390916B03A0916C0346
:107E0000B0916D0380709070482B592B6A2B7B2B9F
:107E1000222311F0616001C06E7F40936A0350938A
:107E20006B0360936C0370936D030FC080916603C6
:107E300090916703E817F90751F410928303609358
:107E4000820350936F0340936E030E946B12089558
:107E50001F93182F80E06CE00E942A1F112309F164
:107E600000D000D00F92EDB7FEB7319682E0ADB7EB
:107E7000BEB711968C938BEB93E0928381838091B4
:107E8000840390E08F779070948383830E94A42072
:107E90000F900F900F900F900F9080E00E94E11EC6
:107EA00005C082E066EB73E00E94FE201F910895FA
:107EB000EF92FF920F931F93182F80FF02C083E071
:107EC00001C085EA0E94E11EE12E11FF02C084E09C
:107ED00001C085EA0E94E11EE2FE02C085E001C009
:107EE00085EA0E94E11EE3FE02C086E001C085EA49
:107EF0000E94E11EE4FE02C087E001C085EA0E9404
:107F0000E11E1F910F91FF90EF9008956091700313
:107F100070917103809172039091730361157105E3
:107F20008105910561F00E941119882341F010929A
:107F30007003109271031092720310927303609198
:107F400074037091750380917603909177036115A6
:107F500071058105910571F00E941119882351F076
:107F600010927403109275031092760310927703A7
:107F70000E946B12609178037091790380917A036B
:107F800090917B03611571058105910561F00E9457
:107F90001119882341F010927803109279031092FE
:107FA0007A0310927B038091830318166CF420915E
:107FB000820330E02F7730708091850390E028179E
:107FC000390714F0109283038091830387FF09C05F
:107FD0008091820390E08F779070892B11F410923A
:107FE00083038091830320915F033091600340916C
:107FF000610350916203882381F421153105410505
:10800000510511F00E946B1210925F0310926003F1
:108010001092610310926203089521153105410504
:10802000510539F0CA01B9010E941119882309F4D8
:108030006CC080918303181644F40E946812833048
:1080400049F4809182038F5F03C080918203815045
:108050008093820380918303813059F08F3F49F0F0
:10806000823061F08E3F51F028E833E140E050E08B
:1080700009C020E335E740E050E004C020EE3EE2D6
:1080800040E050E0809185038E3781F48091C507F0
:108090009091C607A091C707B091C807E7E0569531
:1080A000479537952795EA95D1F721C08E3081F411
:1080B0008091C5079091C607A091C707B091C807E6
:1080C00074E056954795379527957A95D1F70FC067
:1080D0008091C5079091C607A091C707B091C807C6
:1080E00065E056954795379527956A95D1F7280FFE
:1080F000391F4A1F5B1F20935F0330936003409337
:108100006103509362030E946B1208958091800373
:1081100080FD25C06091700370917103809172039E
:1081200090917303611571058105910521F00E94FD
:1081300011198823A1F01092670310926603109220
:1081400087031092860310926503109264031092C5
:108150008003109288030E946B1281E0089580E0F2
:108160000895DF92EF92FF920F931F931091940363
:10817000112399F081E060E00E942A1F812F815035
:108180000E94756BBC0182E00E94FE201092940355
:1081900088EE93E00E94D71902C0882319F00E944C
:1081A0001E1F04C080E060E00E942A1F80916403CB
:1081B00090916503892BF9F00E94C06BFC014091FE
:1081C000640350916503828193818417950749F474
:1081D000218532858091860390918703281739077E
:1081E00051F0538342838091860390918703928755
:1081F00081870E942C6E20916403309165032115C4
:108200003105C9F410926A0310926B0310926C034B
:1082100010926D031092830310926F0310926E03FD
:108220001092820310928403809180038F7E80934A
:108230008003109281038091800382FD0DC08091A4
:108240007C0390917D03A0917E03B0917F03009702
:10825000A105B10531F430C082E065E174E00E940F
:10826000FE208DB79EB707970FB6F8949EBF0FBE3E
:108270008DBFEDB7FEB7319682E0ADB7BEB71196B0
:108280008C9382E094E09283818380917C0390912F
:108290007D03A0917E03B0917F0383839483A583A4
:1082A000B6830E94A420EDB7FEB737960FB6F894B8
:1082B000FEBF0FBEEDBF51C02115310531F482E084
:1082C0006BEF73E00E94FE2021C000D000D00F921F
:1082D000EDB7FEB7319682E0ADB7BEB711968C937D
:1082E00086EF93E092838183348323830E94A420CA
:1082F000809180030F900F900F900F900F9080FF50
:1083000002C081E001C080E20E94E11E1091810361
:108310000E946812682F863008F06150633091F433
:108320008091640390916503892B61F0612F70E067
:108330006370707013E0660F771F1A95E1F76A5A41
:108340007C4F08C070E0B3E0660F771FBA95E1F785
:108350006A587C4F82E00E94FE2080E06CE00E9420
:108360002A1F8091800383FF12C000D000D00F929B
:10837000EDB7FEB7319682E0ADB7BEB711968C93DC
:1083800082EF93E0928381838091840311C000D0B7
:1083900000D00F92EDB7FEB7319682E0ADB7BEB711
:1083A00011968C938EEE93E0928381838091820369
:1083B00090E08F779070948383830E94A4200F9025
:1083C0000F900F900F900F90809164039091650330
:1083D000892B89F0809181038370813081F487E15A
:1083E0000E94221D882339F080E00E94E11E80E077
:1083F0006EEE71E05BC080E20E94E11E59C080E039
:108400000E94E11E0E94C06BFC01808185FF43C079
:108410008091820387FF04C080E062EF70E003C0B8
:1084200080E066EF70E040E024E00E94D41F80917D
:1084300083038823E1F018163CF08E3F81F08F3FD4
:1084400094F48D3FA9F507C08230C9F082309CF0CA
:10845000833071F518C080E062E171E017C080E000
:108460006EE071E013C080E06AE071E00FC080E070
:108470006AEF70E00BC080E06EEF70E007C080E054
:1084800062E071E003C080E066E071E044E024E077
:108490000E94D41F0DC08091820387FF04C080E03A
:1084A00062EE70E003C080E06AEE70E00E940B2094
:1084B0000E946812813049F489E00E94916BAC01FE
:1084C00081E060E00E94841F03C28091800383FDED
:1084D00006C080E060E040E050E00E94331F8091E1
:1084E000800387FD03C000E010E014C080916603A4
:1084F00090916703892B19F001E010E00BC0809187
:1085000081030E94053E20E030E0853010F021E03C
:1085100030E08901F02E81E060E00E942A1F809106
:108520007C0390917D03A0917E03B0917F0300971F
:10853000A105B10509F429C18DE00E94221D8823FF
:1085400029F48EE00E94221D882381F100D00F9231
:1085500082E0EDB7FEB7818382EE93E0938382835E
:108560000E94A4200F900F900F908DE00E94221D7A
:10857000882369F081E066EA71E00E940B2082E0C6
:108580006EEA71E00E940B2080EA9EE30CC081E05D
:108590006EE971E00E940B2082E066EB71E00E94C0
:1085A0000B2084E99EE36CE271E0ECC087E00E945E
:1085B000916BBC0182E00E94FE2087E00E94916BDB
:1085C0000E9423A9182F04C080E20E94E11E1F5FB1
:1085D0001031D0F310918103812F0E94053E90E06D
:1085E000A0E0B0E020917C0330917D0340917E03B8
:1085F00050917F0382179307A407B5070CF44DC071
:1086000081E06BE00E942A1F60917C0370917D03E2
:1086100081E090E0A0E0B0E0062E04C0880F991F32
:10862000AA1FBB1F0A94D2F720916A0330916B03F3
:1086300040916C0350916D0382239323A423B523AF
:108640000097A105B10519F425EA30E002C023E046
:1086500030E08DB79EB707970FB6F8949EBF0FBE58
:108660008DBFEDB7FEB7319682E0ADB7BEB71196BC
:108670008C9389ED93E092838183CB016383948310
:10868000368325830E94A420EDB7FEB737960FB638
:10869000F894FEBF0FBEEDBFC0C01370133009F0D9
:1086A000BCC08FE00E94221D882351F480E10E940B
:1086B000221D882329F48CE00E94221D882369F161
:1086C00080E10E94221D882321F081E066E272E0B1
:1086D00003C081E06EE172E00E940B2081E06FE058
:1086E0000E942A1F00D000D00F92EDB7FEB731963E
:1086F00082E0ADB7BEB711968C9386ED93E092837E
:10870000818381E090E0948383830E94A4200F9072
:108710000F900F900F900F90DBC081E066E272E047
:108720000E940B2081E06BE00E942A1FEDB7FEB78C
:1087300039970FB6F894FEBF0FBEEDBF319682E0B9
:10874000ADB7BEB711968C938DEC93E09283818385
:1087500086E090E09483838387E090E0968385832E
:1087600081E090E0908787830E94A420EDB7FEB758
:1087700039960FB6F894FEBF0FBEEDBF82E79EE3B9
:1087800068EC70E00E94691EA3C0209166033091DE
:1087900067032115310539F100D000D00F92EDB7F4
:1087A000FEB7319682E0ADB7BEB711968C9388ECD8
:1087B00093E092838183348323830E94A4200F90CB
:1087C0000F900F900F900F9080916E038F710E9409
:1087D000583F002321F08CE30E94E11E2DC080E26F
:1087E0000E94E11E1CC000D000D00F92EDB7FEB772
:1087F000319682E0ADB7BEB711968C938FEB93E0C4
:108800009283818388E893E0948383830E94A420E9
:108810000F900F900F900F900F90FF2069F48091B0
:10882000740390917503A0917603B091770300973C
:10883000A105B10509F444C08091660390916703D6
:10884000892BF1F5809181030E94053E8530C0F1AE
:1088500081E060E00E942A1F86E40E94E11EA2E0FF
:10886000EA2EF12C012D112DDD24D39480916A0381
:1088700090916B03A0916C03B0916D038E219F21A9
:10888000A023B1230097A105B10549F0B9E0BD15BA
:1088900018F08D2D805D04C08D2D885001C085EAB3
:1088A0000E94E11ED394E0E1DE1629F0EE0CFF1CDD
:1088B000001F111FDBCF80E20E94E11E81E006C095
:1088C00080916A038F710E94583F80E00E94343E7D
:1088D0001F910F91FF90EF90DF900895CF93DF935A
:1088E000EB0180938103E82FF0E0EF70F070E85E19
:1088F000FB4FE491E09385036115710559F0CB01BD
:1089000060E070E048E853E00E942D85D093870333
:10891000C09386030E946B12DF91CF9108951F933D
:10892000FC01009769F4109280031092700310927A
:10893000710310927203109273030E94864064C008
:108940007091800371FD60C060938203CA01A0E052
:10895000B0E020916A0330916B0340916C03509119
:108960006D0320703070822B932BA42BB52B80933A
:108970006A0390936B03A0936C03B0936D03809193
:10898000C5079091C607A091C707B091C807885145
:108990009C4FAF4FBF4F81608093700390937103E2
:1089A000A0937203B093730372FF25C071607B7F45
:1089B00070938003F0936703E0936603CF010E94F6
:1089C0008E38FC01009761F08091820390858927A1
:1089D00087FF06C06091660370916703706804C0EA
:1089E00060916603709167038091640390916503C1
:1089F0000E94503C07C07E7F70938003F093650314
:108A0000E09364030E946B121F910895AC01809162
:108A100080038C7F809380031092870310928603DB
:108A2000662309F045C010928803209164033091B9
:108A300065032115310521F0309369032093680304
:108A400010926A0310926B0310926C0310926D03E4
:108A500010926F0310926E031092670310926603D8
:108A600010926503109264031092830310928103A5
:108A70001092210C4115510551F18FEFBA010E945E
:108A80000E6E8091800381FD22C010926A031092C5
:108A90006B0310926C0310926D0310926703109297
:108AA00066031092650310926403109281030DC057
:108AB0001092210C60916403709165038FEF0E9406
:108AC0008C6D8091800381FD02C090E001C091E037
:108AD000809180038B7F826080938003892F08952B
:108AE000CF93DF93EC01288D398D4A8D5B8D20303B
:108AF00088E2380780E0480780E058071CF08C8D3A
:108B000086FF5DC0203080E4380780E0480780E0C1
:108B100058070CF054C06A817B812115310541054D
:108B2000510509F443C061157105E1F0888199810F
:108B3000A0E0B0E082179307A407B50741F0CB018E
:108B4000A0E0B0E082179307A407B50759F48C8D15
:108B50008E7F8C8F888199810E948D3C1B821A8226
:108B60001982188288819981A0E0B0E0288D398D22
:108B70004A8D5B8D82179307A407B50729F48C8D66
:108B800091E089278B7F16C081E060E00E942A1F58
:108B900080E00E94916BBC0182E00E94FE206C8DFF
:108BA0006470888D998D0E94064505C0672B19F465
:108BB0008C8D84608C8F188E198E1A8E1B8EDF918F
:108BC000CF910895DF92EF92FF920F931F939C0134
:108BD0008531910509F465C38631910524F58C3002
:108BE000910509F480C18D309105A4F48A30910576
:108BF00044F4813091050CF0AAC3009709F45BC3DB
:108C0000F0C38A30910509F4D4C38B30910509F083
:108C1000E8C3C6C3813191050CF054C28F30910571
:108C20000CF0BFC206C28A38910509F4BEC38B3866
:108C30009105C4F48B31910564F4893191053CF5BB
:108C40008631910509F4E1C28731910509F0C9C364
:108C50000FC18132910509F4D0C28332910509F028
:108C6000C0C3B6C38F3891054CF48D3891050CF014
:108C7000E0C18C38910509F0B4C3B5C181399105C3
:108C80000CF4ADC28739910509F0ABC3A8C380913C
:108C9000800383FF03C01091840302C010918203FC
:108CA00000E02931310509F401E0E09085030E94DC
:108CB000C06BFC01F7800E94C06BFC01808184FFC7
:108CC00035C017FD05C080E0002309F481E0082FBE
:108CD000002311F001E02CC0812F90E08F7790707D
:108CE000892B79F48091780390917903A0917A038C
:108CF000B0917B030097A105B10519F4212F2058ED
:108D0000ADC08091C5079091C607A091C707B091EB
:108D1000C807845D9E4FAF4FBF4F809378039093F9
:108D20007903A0937A03B0937B0324C0002311F14D
:108D30000E94C06BFC01808185FF07C08091830386
:108D400083300CF08AC08F5F21C00E94681283308C
:108D500009F083C0812F90E08F7790702E2D30E046
:108D6000821793070CF079C0FEE7EF16E1F5FF20BC
:108D7000E1F439C00E94C06BFC01808185FF09C00D
:108D8000809183038E3F0CF468C0815080938303ED
:108D900064C0812F90E08F779070892B09F45DC0BB
:108DA0004EE7E41641F5FF2031F181E0F81619F4A1
:108DB00060E820E00EC0E2E0FE1619F46EE324E164
:108DC00008C0F3E0FF1619F466E12AE002C060E88B
:108DD00020E8812F90E030E0002341F08F77907001
:108DE000821793075CF4212F2F5F38C08F77907024
:108DF000281739071CF0212F215030C0462F50E092
:108E0000812F90E08F779070481759071CF0212F21
:108E10002E7F04C0212F261B2C7F260F211719F02F
:108E2000002319F41BC0002361F0822F90E08F779C
:108E300090708417950714F482E001C084E0280F35
:108E40000DC0822F90E08F7790704817590714F06B
:108E500082E001C084E0281B01C0212F80918003A3
:108E600083FF03C020938403207820938203B7C23A
:108E70009091800397FF21C088E089278093800329
:108E800083FF0EC080918203809384038078809357
:108E900082031092830388E29FE360E971E00AC0D5
:108EA00080918403809382031092840380E090E099
:108EB00060E070E00E94691E92C28091810383701D
:108EC000813029F480E06EEE71E00E940B208091E9
:108ED000820380588078809382031092830380916C
:108EE0008003877F72C28091660390916703009729
:108EF00009F049C0E0907C03F0907D0300917E036F
:108F000010917F031E141F0410061106E4F5D09083
:108F100081038D2D0E94053E90E0A0E0B0E08E150B
:108F20009F05A007B1071CF181E090E0A0E0B0E050
:108F300004C0880F991FAA1FBB1FEA94D2F7209183
:108F40006A0330916B0340916C0350916D0382274B
:108F50009327A427B52780936A0390936B03A0936C
:108F60006C03B0936D038091800380683BC143E044
:108F7000D422D41609F033C2809164039091650322
:108F8000B70141E026C16091800367FF10C0892BC3
:108F900071F080916E0390916F0321E030E08227A1
:108FA000932790936F0380936E03606119C0809143
:108FB0006A0390916B03A0916C03B0916D0321E063
:108FC00030E040E050E082279327A427B527809324
:108FD0006A0390936B03A0936C03B0936D036F7E51
:108FE00060938003FCC18091660390916703892B95
:108FF00029F4809180038F77809380038091800390
:1090000085FFEDC120917C0330917D0340917E036B
:1090100050917F0312161306140615060CF0DFC0DC
:109020008091640390916503B90140E00E94E037AC
:10903000D6C080917C0390917D03A0917E03B09176
:109040007F030097A105B105D9F1893FE7E09E07AD
:10905000E0E0AE07E0E0BE070CF0C1C1AC0141505A
:109060005040440F551FC9018F7790700E9709F437
:10907000416027FF1FC0CA0160E044E00E94E58E06
:109080008091800383FD05C080E090E060E070E0A7
:1090900004C088E29FE360E971E00E94691E81E0FC
:1090A00066E271E00E940B2082E06EE271E00E94B5
:1090B0000B209AC0CA0161E044E00E94E58E8FC196
:1090C00027FD8DC1022F0D501091800317FF0AC09C
:1090D0008091660390916703892B21F4213131053A
:1090E0000CF40C5F809181030E94053E081708F084
:1090F00076C10430A0F08091C5079091C607A09179
:10910000C707B091C8078C509E4FAF4FBF4F809399
:10911000740390937503A0937603B093770317FFBE
:109120001DC08091660390916703892BB9F082E09E
:1091300090E0A0E0B0E004C0880F991FAA1FBB1FF9
:109140000A95D2F720916E0330916F0328273927B3
:1091500030936F0320936E03106120C082E090E093
:10916000A0E0B0E004C0880F991FAA1FBB1F0A959A
:10917000D2F720916A0330916B0340916C035091B8
:109180006D0382279327A427B52780936A039093C2
:109190006B03A0936C03B0936D031F7E1093800349
:1091A0001EC1E0907C03F0907D0300917E0310913E
:1091B0007F03E114F1040105110509F483CF8091C7
:1091C00064039091650340E02F30310509F441E0DC
:1091D000B7010E94E037809180038062F6C08091E1
:1091E00080038F7D8093800310927C0310927D0317
:1091F00010927E0310927F03F2C0809164039091DD
:1092000065036CE30E94C037EAC080917C039091B3
:109210007D03A0917E03B0917F030097A105B10566
:1092200071F18091800382FD2AC00E946812833010
:1092300019F580918503282F30E040E050E08091BF
:109240007C0390917D03A0917E03B0917F0328174A
:1092500039074A075B0744F420937C0330937D036E
:1092600040937E0350937F03809182038078909196
:109270007C03892B8093820310928303B5CFF894EB
:1092800083E00E94831287E10E94221D882339F027
:1092900080916403909165036BE40E94C0377894D9
:1092A0009EC08091800387FF02C082E001C080E001
:1092B0000E94831294C08091800387FF12C0809126
:1092C000680390916903009709F48BC0A0E0B0E0B7
:1092D00080937C0390937D03A0937E03B0937F03E0
:1092E0001EC082FF21C080917C0390917D03A091DC
:1092F0007E03B0917F030097A105B105A9F489E031
:109300000E949EA580917C0390917D03A0917E0395
:10931000B0917F030097A105B10509F462C084E60E
:1093200093E00E9470455DC080917C0390917D0325
:10933000A0917E03B0917F030097A105B10539F498
:109340008FEF0E949EA581E00E94B1404AC0790142
:109350000027F7FC0095102F60917C0370917D032E
:1093600080917E0390917F032AE030E040E050E05E
:109370000E945BA7E60EF71E081F191FF0E0EF160C
:10938000F0E8FF06F0E00F07F0E01F0754F5E09269
:109390007C03F0927D0300937E0310937F031FC034
:1093A00084E693E00E9470451AC0809180038F7715
:1093B0000CC010927C0310927D0310927E031092D9
:1093C0007F03809180038B7F80688093800307C038
:1093D00080918203807880938203109283030E949D
:1093E0006B121F910F91FF90EF90DF900895FC0199
:1093F000EC5AFF4F2081E455F0402223C1F0E95A96
:10940000FF4F8081E755F040948180FD08C098357A
:1094100011F0983761F4223020F481E00895892F0B
:1094200001C085818095881F8827881F089580E066
:10943000089580E008950F931F93CF93DF93182F23
:10944000EB01622F9E0170E02EC0CA0180959095BD
:1094500028233923DA01AC23BD23109711F0A1E0B2
:10946000B0E06031B8F46117A8F4862F90E0FC01F9
:10947000E295F295F07FFE27E07FFE27E81BF90BCF
:10948000EA5BFB4F8685882329F0808191818230B9
:10949000910508F0CD01892B11F0242B352B7F5F2E
:1094A000440F551F6F5F701780F2C901DF91CF9194
:1094B0001F910F910895E82F4423E9F088E5E89F74
:1094C000F0011124EA56FC4F80915404882371F076
:1094D00080914604909147048230910538F4892B9D
:1094E00029F0E95AFF4F8081816004C0E95AFF4F9B
:1094F00080818E7F808381E00895653069F16630D8
:1095000070F4623001F1633028F46623B1F0613009
:10951000B1F516C06330D1F0643089F51AC06830F7
:1095200021F1693028F46630D1F0673041F51AC076
:109530006930F1F0603119F51EC060ED77E01DC0B3
:109540006AEC77E01AC066EC77E017C063EC77E06E
:1095500014C06DEB77E011C066EB77E00EC06BEAEC
:1095600077E00BC064EA77E008C06CE977E005C0FB
:109570006DE877E002C065E877E00E94FE2081E0B8
:1095800008956DE879E00E94FE2081E0089566EC80
:1095900079E00E94FE2081E0089563EE79E00E9468
:1095A000FE2081E008951F93182F66E57AE00E945F
:1095B000FE20812F67E37AE00E94FE20812F6AE17E
:1095C0007AE00E94FE2081E01F910895CF93DF93FF
:1095D000EC01009719F16BE777E00E941AA9892B3B
:1095E00011F481E01CC0CE0167E777E00E941AA960
:1095F000892B11F482E013C0CE0163E777E00E946B
:109600001AA9892B11F483E00AC0CE0160E777E044
:109610000E941AA9892B11F480E001C08FEFDF911D
:10962000CF9108952F923F924F925F926F927F92C7
:109630008F929F92AF92BF92CF92DF92EF92FF9262
:109640000F931F93DF93CF9300D0CDB7DEB79A83EC
:10965000898380EFE6E4F4E0DF011D928A95E9F763
:1096600049805A80F2019081992399F09C3289F0C7
:10967000943279F0953269F0892F80538A3048F01E
:10968000892F992787FD90950E940BA9892B09F4B2
:10969000DFC096E4692E94E0792EAA24A3941E01DB
:1096A0000894211C311CADC00F5F1F4F1A83098322
:1096B00009811A81D801BC908B2D992787FD90953F
:1096C0000E940BA9892B81F7BB2009F4AAC0BCE238
:1096D000BB1609F48DC0E7E2BE1629F0F2E2BF1610
:1096E00011F0BB2404C00F5F1F4F1A83098382E06F
:1096F000882E912C860C971CC980DA80EE24FF24DA
:1097000009C0D4011D934D010894C11CD11C0894BB
:10971000E11CF11CBBE0EB16F1049CF4F601108196
:10972000112379F0BB2019F01B1559F70AC01C3220
:1097300041F0812F992787FD90950E940BA9892BD5
:1097400001F3D4011C92E981FA818081843241F4D1
:10975000CF0101969A838983B10140E150E013C0A3
:10976000853269F4CF0101969A838983B10142E081
:1097700050E00E94ADA7D3016D937C9309C0CF0147
:10978000B1014AE050E00E94ADA7F301718360830C
:10979000E1E0D3011E96EC9304C00F5F1F4F1A83C4
:1097A000098309811A81D801FC90FF2081F08F2D57
:1097B000992787FD90950E940BA9892B41F4BCE263
:1097C000FB1659F704C00F5F1F4F1A8309830981E5
:1097D0001A81F801F080FF2079F08F2D992787FDFD
:1097E00090950E940BA9892B71F7FCE2FF1621F4DA
:1097F0000F5F1F4F1A830983A3948FE090E0680ED8
:10980000791EFA2CFA94E981FA818081882321F06B
:1098100091E1A91609F04CCF4114510411F0D20185
:109820001C928F2D90E00F900F90CF91DF911F91A0
:109830000F91FF90EF90DF90CF90BF90AF909F90EF
:109840008F907F906F905F904F903F902F900895F2
:109850000894411C511C5A82498202CF0F931F93D6
:10986000082F162F603418F064ED75E002C06CEC20
:1098700075E00E94FE201A30A1F11B3080F41630F2
:1098800021F1173030F41130C1F0123009F045C029
:1098900018C0183011F1193009F03FC01AC01E303D
:1098A00071F11F3028F41B3001F11D30B1F521C0DA
:1098B000113449F1123489F52AC0802F6CEB75E020
:1098C0001BC0802F68EA75E017C0802F6BE975E038
:1098D00013C0802F68E875E00FC0802F65E775E042
:1098E0000BC0802F6DE675E007C0802F6BE575E03B
:1098F00003C0802F62E575E00E94FE2014C0802F17
:109900006BE375E0F9CF802F60E375E003C0802F33
:1099100065E275E00E94FE2002C0103420F0802F26
:109920006DE00E94242081E01F910F910895782F0F
:109930006031C8F46417B8F4862F90E0FC0144E06D
:10994000EE0FFF1F4A95E1F7E81BF90BEA5BFB4FAF
:109950008685882341F0408151812417350718F00E
:109960004115510531F4872F62E00E942E4C40E0F2
:1099700050E0CA0108950F931F93082F142F0E94DF
:10998000FE20802F60E20E942420112319F46FE34F
:1099900077E002C062E477E0802F0E94FE20802FF3
:1099A0006DE00E9424201F910F910895DF92EF92A5
:1099B000FF920F931F93CF93DF93082F7B01EA0150
:1099C000D22E10E012C0802F60E20E942420CE012F
:1099D0008E219F21892B11F460E301C061E3802F68
:1099E0000E9424201F5FCC0FDD1F1D1560F3DF9147
:1099F000CF911F910F91FF90EF90DF90089560E05D
:109A00000E9424208FEF08950F931F93182FFB01BE
:109A10000181002311F482E011C060E00E94242043
:109A2000E02FF0E0EA59F24F60816095812F0E94AB
:109A30002420812F60E00E9424208FEF1F910F913E
:109A40000895982F442309F440C08091540488233A
:109A5000E1F1609146047091470461157105A9F127
:109A600020E46030720788F5272F33272F7330707A
:109A700020543F4FAB015070ADB7BEB71F970FB624
:109A8000F894BEBF0FBEADBFEDB7FEB731961196CD
:109A90009C938DEE97E092838183748363837683B6
:109AA000658330872783328721875487438756878A
:109AB00045870E94A42081E0EDB7FEB73F960FB620
:109AC000F894FEBF0FBEEDBF0895892F61E00E949C
:109AD0007D4A0895682F442371F0809154048823AF
:109AE00051F08091460490914704803C910518F014
:109AF000883E910510F080E090E0582F423060F0F1
:109B000080916304882341F02091550430915604DC
:109B10002F3F310519F010F020E030E0852F805CF8
:109B2000883228F0862F61E00E947D4A089500D097
:109B300000D00F92EDB7FEB73196ADB7BEB7119614
:109B40006C9388E298E092838183852F90E08F73F5
:109B50009070982F8827820F911D948383830E9491
:109B6000A42081E00F900F900F900F900F90089518
:109B7000CF92DF92EF92FF920F931F93DF93CF93D9
:109B800000D000D000D0CDB7DEB7D82E2DB73EB76D
:109B9000275030400FB6F8943EBF0FBE2DBFEDB733
:109BA000FEB73196ADB7BEB711968C9380EF95E0B6
:109BB000928381838DE090E0948383838AEE95E0A5
:109BC000968385830E94A420EDB7FEB737960FB623
:109BD000F894FEBF0FBEEDBFDD2019F48CE49FE4C6
:109BE00002C087E49FE40E941B6F88E0E6E3F5E093
:109BF000DF011D928A95E9F700E010E031E0E32EE5
:109C0000F12C802F0E94776F8823A9F0F80123E0C0
:109C1000F595E7952A95E1F7EA5CFA4FC801877058
:109C20009070970102C0220F331F8A95E2F7C90195
:109C30002081282B20830F5F1F4F0034110509F767
:109C40008E010F5F1F4F86E0D8011D928A95E9F7BC
:109C50008FEF6CE1A8010E94E36F94E1E92EF12CF3
:109C6000C02E012F23C0F901EA5CFA4F80818823BE
:109C700029F42F5F3F4F28303105A9F728303105EF
:109C8000C0F48AE090E00E94D7190894E108F10836
:109C9000BAE0EB16F10439F48FEF6CE14C2D502F44
:109CA0000E94E36F03C01E141F041CF420E030E088
:109CB000E2CF80E090E00E941B6F00E010E084EEB5
:109CC000E82E85E0F82EF801B3E0F595E795BA9512
:109CD000E1F7EA5CFA4F808190E0980127703070DC
:109CE00002C0959587952A95E2F780FF15C000D0B0
:109CF00000D00F92EDB7FEB73196ADB7BEB7119653
:109D0000DC92F282E182148303830E94A4200F90EC
:109D10000F900F900F900F900F5F1F4F00341105A1
:109D200091F68D2D6EED75E00E94FE2081E0269665
:109D30000FB6F894DEBF0FBECDBFCF91DF911F915C
:109D40000F91FF90EF90DF90CF9008951F93CF93E6
:109D5000DF93182FEB0198819F3F31F089818C317F
:109D600019F48A81882321F4CE010E9443778BC0A5
:109D70009F77892F869586958695E82FF0E0EA5C97
:109D8000FA4F4081692F70E09B0127703070842F5B
:109D900090E0022E02C0959587950A94E2F780FF25
:109DA00072C081E090E002C0880F991F2A95E2F707
:109DB0008095842380838E81863211F48FED8E838B
:109DC0008DB79EB70D970FB6F8949EBF0FBE8DBF8F
:109DD000EDB7FEB73196ADB7BEB711961C938FEFB6
:109DE00095E092838183748363838A81858316825D
:109DF0008B81878310868C81818712868D818387F2
:109E000014860E94A4202E818DB79EB70D960FB6A2
:109E1000F8949EBF0FBE8DBF222389F100D000D0E1
:109E20000F92EDB7FEB73196ADB7BEB711961C9342
:109E30008CEF95E092838183238314820E94A42077
:109E40006F810F900F900F900F900F906623B9F0D5
:109E500000D000D00F92EDB7FEB73196ADB7BEB7C8
:109E600011961C9389EF95E092838183638314821A
:109E70000E94A4200F900F900F900F900F90812FB1
:109E80006DE00E942420DF91CF911F910895BC01C5
:109E900081E00E94A64E0895BC0180E00E94A64E7B
:109EA00008950E944D3284E06EEB71E00E940B2019
:109EB00085E066EC71E00E940B2085E99DE968EC85
:109EC00070E00E94691E80E060E00E942A1F0E94EC
:109ED0002B3B0E949B830E94876E0E94076C81E04F
:109EE00008950F931F93082F142F82E00E94CD6BCB
:109EF000882329F482E00E94526E0E942C6E112366
:109F000079F080915404882359F06091460470914F
:109F100047046115710531F080E46030780710F076
:109F200060E070E08FEF0E946A7D9B01AC016115DB
:109F300071058105910501F1ADB7BEB717970FB651
:109F4000F894BEBF0FBEADBFEDB7FEB73196119608
:109F50000C9384E196E09283818323833483458349
:109F600056830E94A420EDB7FEB737960FB6F8943B
:109F7000FEBF0FBEEDBF12C000D00F92ADB7BEB78F
:109F800011960C9311978EE096E013969C938E9306
:109F900012970E94A4200F900F900F9081E01F91C4
:109FA0000F91089563E879E00E94FE2082E00E940C
:109FB000831280E0089583E00E94831280E0089578
:109FC00080E00E94831280E0089560E00E942420D7
:109FD00082E00E9483128FEF089580E00E94831236
:109FE0000E94E9A581E008951F93182F0E9468122E
:109FF0008430D1F0853038F4823071F0833080F4D1
:10A00000882331F01EC08730B8F08730D1F410C0FB
:10A01000812F6EEC78E013C0812F66EC78E00FC0E2
:10A02000812F6FEB78E00BC0812F63EB78E007C0E6
:10A03000812F67EA78E003C0812F61EA78E00E940F
:10A04000FE2081E01F910895EF92FF920F931F93DE
:10A05000182F7B01042F83E00E948312812FB70108
:10A06000402F0E94F44F1F910F91FF90EF900895A1
:10A07000EF92FF920F931F93182F7B01042F80E024
:10A080000E948312812FB701402F0E94F44F1F912D
:10A090000F91FF90EF9008951F93182F0E94681260
:10A0A000833041F0873031F0823011F468E103C031
:10A0B00060E001C068E0812F0E9424208FEF1F9193
:10A0C0000895AF92BF92CF92DF92EF920F931F93BA
:10A0D000CF93DF93182F042F0E946812882319F45E
:10A0E000812F66E016C0002391F0809154048823EC
:10A0F00071F0A0904604B0904704A114B10439F067
:10A1000020E0A21628E2B20610F4023028F4812FD3
:10A1100062E00E942E4C58C0809163048823B9F3FA
:10A12000C0905504D0905604C114D10481F331E09D
:10A13000C31634E0D30658F7023061F08091720400
:10A14000882341F0C0916404D0916504CF3FD105CC
:10A1500019F010F0C0E0D0E0C5010E94B63883705D
:10A16000833019F0812F6AE0D4CF9601215030401E
:10A17000C50160E041E000E0EC2E0E945A388DB746
:10A180009EB709970FB6F8949EBF0FBE8DBFEDB76F
:10A19000FEB73196ADB7BEB711961C938AE196E033
:10A1A00092838183B482A382D682C582D087C783FB
:10A1B0000E94A42081E02DB73EB7275F3F4F0FB626
:10A1C000F8943EBF0FBE2DBFDF91CF911F910F912D
:10A1D000EF90DF90CF90BF90AF900895AF92BF9275
:10A1E000CF92DF92EF92FF920F931F93CF93DF9363
:10A1F000B82E7B0180916304882309F47DC080918F
:10A200007204423008F478C000915504109156044D
:10A210000115110509F470C024E00130120708F49B
:10A220007AC06AC0423029F480E090E020E030E05B
:10A2300019C020916404309165042F3F310519F055
:10A2400010F020E030E0443058F080918104882301
:10A2500039F080917304909174048138910510F065
:10A2600080E090E0D22EC82EC7016AEE77E00E940F
:10A270001AA9892B39F0C70167EE77E00E941AA965
:10A28000892B01F5809154048823B1F1C0914604D3
:10A29000D091470481E0CF3FD80770F5C70164EE45
:10A2A00077E00E941AA9892B11F062E001C061E0F9
:10A2B000219701501040CE0143E0880F991F4A9525
:10A2C000E1F711C0809154048823B1F080914604D5
:10A2D00090914704009781F020E48030920760F469
:10A2E0000150104060E04A2D98010D2DEC2C0E9489
:10A2F0005A388B2D60E002C08B2D61E00E947D4AB0
:10A30000DF91CF911F910F91FF90EF90DF90CF9051
:10A31000BF90AF900895AA24882309F083CFAA2480
:10A32000A394CC24DD24A0CFEF920F93FB01828174
:10A3300090E087709070582F4427818190E0482BDF
:10A34000592B6381848197E0483F590700F590E0DD
:10A3500087709070382F2227862F90E0282B392B7A
:10A360002150304083E02F3F380788F48081893DB9
:10A3700029F4CA0162E040E0058104C0CA0162E03C
:10A3800041E000E0EE240E945A3880E001C082E003
:10A390000F91EF9008951F93182F442359F0809147
:10A3A0005404882339F08091460490914704883002
:10A3B000910510F08FEF90E0883010F40E945E6EEF
:10A3C0000E94C76B00D000D00F92EDB7FEB7319658
:10A3D000ADB7BEB711961C9327E236E032832183D6
:10A3E000838314820E94A4200F900F900F900F90EF
:10A3F0000F9081E01F9108951F93CF93DF93142F47
:10A4000080E00E94831288EE93E00E94D719112306
:10A4100071F080915404882351F0C0914604D0918A
:10A420004704209721F0CF3FD10519F010F0CEE47A
:10A43000D0E0F89487E00E948312CE010E94893C0C
:10A44000CE0166E90E94C037789481E0DF91CF9118
:10A450001F910895875E934091F5613069F06130F6
:10A4600028F06230A9F0633051F51EC00E94C06B25
:10A47000FC0180818F731DC00E94C06BFC01808134
:10A480008F7780830E94C06BFC018081806411C043
:10A490000E94C06BFC018081806880830E94C06B39
:10A4A000FC0180818F7B05C00E94C06BFC01808114
:10A4B000806C80830E942C6E20E030E002C02FEF81
:10A4C0003FEFC9010895FB01928180E0218130E0D6
:10A4D000822B932B63810E942A52892F881F882701
:10A4E000881F880F08951F938130910531F0875E92
:10A4F0009340A9F02FEF3FEF26C00E94C06BFC01F4
:10A500008181882311F484E608C0843011F485E643
:10A5100004C08150843008F08150282F13C00E945D
:10A52000C06BFC01808190E0B6E096958795BA9566
:10A53000E1F7182F11700E94C06BFC01808187FD2C
:10A540001260212F30E0C9011F9108951F93CF930E
:10A55000DF93182F4423A9F180915404882341F0FC
:10A56000209146043091470483E0283E380710F0DC
:10A570002FEF3FEF423039F580916304882341F09B
:10A58000C0915504D0915604CF3FD10519F010F079
:10A59000C0E0D0E0C9016C2F0E942A5297FD19C07B
:10A5A00000D000D00F92EDB7FEB73196ADB7BEB771
:10A5B00011961C938AE398E092838183C38314826B
:10A5C0001EC02FEF3FEFC9010E9473529C0197FFFD
:10A5D00005C0812F62E00E942E4C19C000D000D02F
:10A5E0000F92EDB7FEB73196ADB7BEB711961C937B
:10A5F00087E398E0928381833070348323830E94C1
:10A60000A42081E00F900F900F900F900F90DF919A
:10A61000CF911F9108951F93CF93DF93182FFB01C4
:10A62000928180E0218130E0822B932B0E94735233
:10A63000EC0197FF02C082E009C0812F60E00E9418
:10A640002420812F6C2F0E9424208FEFDF91CF9147
:10A650001F9108950F931F93CF93DF93082F142F0B
:10A660000E94C06BDC0118968C91C82FD0E0CC0FF3
:10A67000DD1F112361F080915404882341F0809103
:10A680004604909147048134910508F4EC010E943E
:10A69000C06BFE01EF5F2E2F2695DC0118962C93E0
:10A6A0000E94C06B00D000D00F92EDB7FEB731967C
:10A6B000ADB7BEB711960C9329E438E032832183FD
:10A6C000DC0118968C9190E0880F991F9483838306
:10A6D0000E94A4200F900F900F900F900F9081E098
:10A6E000DF91CF911F910F9108950F931F93CF93F7
:10A6F000DF93082F142F0E94C06BEC01112351F13E
:10A700004B8580915404882339F020914604309180
:10A7100047042531310518F0842F90E09C012B87E8
:10A720008C85282F30E0220F331F123078F0809173
:10A730006304882359F08091550490915604823027
:10A74000910520F041E08F3F940708F0C9019695EC
:10A7500087958C870E942C6E8DB79EB707970FB692
:10A76000F8949EBF0FBE8DBFEDB7FEB73196ADB763
:10A77000BEB711960C9388E798E0928381838B850E
:10A78000838314828C8590E0880F991F968385833C
:10A790000E94A4208DB79EB707960FB6F8949EBF6F
:10A7A0000FBE8DBF81E0DF91CF911F910F91089572
:10A7B0000F931F93FB0102818181882319F083305D
:10A7C000C1F40CC00936A8F410E00F5F1F4F1595B7
:10A7D00007950E94C06BFC01008709C08091F20CB4
:10A7E000002311F0816001C08E7F8093F20C80E025
:10A7F00001C082E01F910F9108950F931F93082FBE
:10A80000FB018181882321F0833041F082E012C076
:10A810000E94C06BFC011085110F03C01091F20C57
:10A820001170802F60E00E942420802F612F0E94F1
:10A8300024208FEF1F910F910895EF92FF920F93B5
:10A840001F93CF93DF93082F142F0E94C06B7C01BE
:10A8500080915404882389F088E494E060E376E0F2
:10A860000E941AA9F7012081892B11F42B7F02C0C5
:10A870002460F70120830E94CB30809163048823F9
:10A8800079F0123008F453C0809155049091560429
:10A89000893C910508F04BC097FD49C0F7018683BC
:10A8A00080917204882379F086E694E06DE276E088
:10A8B0000E941AA9F7012081892B11F4277F02C079
:10A8C0002860F701208380918104882359F08091CA
:10A8D0007504F7012081893511F4216002C02E7FB3
:10A8E000F701208380919004882369F01530F8F0F7
:10A8F000809182049091830485339105C0F497FD83
:10A9000016C0F701808780919F048823F1F01630EC
:10A9100070F0C0919104D0919204F4E0C03BDF0745
:10A9200030F081EEC130D80710F410E006C0802F5F
:10A9300062E00E942E4C0CC01F5F812F0E94AC145D
:10A940008C179D07C8F3F70111830E942C6E81E0DC
:10A95000DF91CF911F910F91FF90EF9008950F938A
:10A960001F93082F142F87E594E06AE376E00E9496
:10A970001AA9892B19F063E070E002C061E070E071
:10A9800090915404992341F480916304882321F029
:10A99000CB010E94E48C2DC0112361F0992351F06A
:10A9A00020914604309147042F3F310509F010F4FF
:10A9B00037FF05C0802F62E00E942E4C1BC08091A3
:10A9C0006304E3E0220F331FEA95E1F7882371F473
:10A9D000C9010E94638C019719F063E376E002C01D
:10A9E00067E376E0802F0E94FE2003C0C9010E9429
:10A9F000948C81E01F910F9108951F93182F64E9A3
:10AA000078E00E94FE20812F6EE878E00E94FE2010
:10AA10000E94D46B2DB73EB7275030400FB6F89444
:10AA20003EBF0FBE2DBFEDB7FEB73196ADB7BEB777
:10AA300011961C9321E838E0328321836383748369
:10AA4000858396830E94A4202DB73EB7295F3F4F90
:10AA50000FB6F8943EBF0FBE2DBF81E01F91089541
:10AA60008F929F92AF92BF92CF92DF92EF92FF921E
:10AA70000F931F93DF93CF93CDB7DEB760970FB6D9
:10AA8000F894DEBF0FBECDBFE82E82E00E94168193
:10AA90009A8389834E010894811C911CA3E0AA2EFD
:10AAA000B12CAC0EBD1EF0E3CF2EF7E0DF2E4BC075
:10AAB00080E1B4010E948C818501FF24D8018D9131
:10AAC0009C910097E1F19C013F77B0E420303B0777
:10AAD000B0F5FF2019F480E091E002C081E091E040
:10AAE000EDB7FEB737970FB6F894FEBF0FBEEDBFB8
:10AAF0003196ADB7BEB71196EC92D282C1829483E3
:10AB00008383368325830E94A420EDB7FEB7379652
:10AB10000FB6F894FEBF0FBEEDBFFF2049F0D8017D
:10AB20008D919C9197FF04C08E2D61E20E9424209C
:10AB3000F3940E5F1F4FB7E0FB1609F0BFCF8E2DC9
:10AB40006DE00E94242089819A81892B09F0B0CF81
:10AB500060960FB6F894DEBF0FBECDBFCF91DF91E8
:10AB60001F910F91FF90EF90DF90CF90BF90AF902B
:10AB70009F908F9008951F93182F0E943055812F1A
:10AB80006AE677E00E94FE2081E01F9108954F92CF
:10AB90005F926F927F928F929F92AF92BF92CF926D
:10ABA000DF92FF920F931F93DF93CF93CDB7DEB762
:10ABB00060970FB6F894DEBF0FBECDBFF82E83E0CE
:10ABC0000E9416819A8389832E010894411C511C8E
:10ABD0008CE3682E87E0782E05E0802E912C8C0E79
:10ABE0009D1E15E3A12E17E0B12EB1E1CB2ED12C85
:10ABF000CC0EDD1E4BC080E1B2010E948C8100D0E2
:10AC000000D00F92EDB7FEB73196ADB7BEB7119633
:10AC1000FC92728261828B819C81948383830E94E7
:10AC2000A42084010F900F900F900F900F90F801C7
:10AC30009181992311F12DB73EB7275030400FB6BF
:10AC4000F8943EBF0FBE2DBFEDB7FEB73196ADB73E
:10AC5000BEB71196FC92B282A182D8018C918383F7
:10AC60001482958316820E94A420EDB7FEB7379612
:10AC70000FB6F894FEBF0FBEEDBF0E5F1F4F0C1551
:10AC80001D05A9F68F2D6DE00E94242089819A81EF
:10AC9000892B09F0B0CF60960FB6F894DEBF0FBED7
:10ACA000CDBFCF91DF911F910F91FF90DF90CF909B
:10ACB000BF90AF909F908F907F906F905F904F90DC
:10ACC00008951F93182F0E94C755812F64E677E0DF
:10ACD0000E94FE2081E01F910895EF92FF920F9352
:10ACE0001F93CF93DF93F82E8B01E42EE901842F7D
:10ACF0000E94FB3D2DB73EB7275030400FB6F89469
:10AD00003EBF0FBE2DBFEDB7FEB73196ADB7BEB794
:10AD10001196FC922DE537E032832183148303835F
:10AD2000968385830E94A4202E2D30E0C901837074
:10AD3000907001974DB75EB7495F5F4F0FB6F894BB
:10AD40005EBF0FBE4DBF029778F4C9018C70907042
:10AD50008430910519F48F2D61E604C0089721F421
:10AD60008F2D62E60E9424208F2D6AE577E00E94F5
:10AD7000FE204E2D50E0437050704130510569F077
:10AD8000423051051CF4452BA1F018C0423051054A
:10AD900041F04330510591F408C08F2D66E577E00E
:10ADA0000BC08F2D62E577E007C08F2D6EE477E052
:10ADB00003C08F2D6BE477E00E94FE202097D1F036
:10ADC00088818823B9F000D000D00F92EDB7FEB78C
:10ADD0003196ADB7BEB71196FC9286E497E09283A8
:10ADE0008183D483C3830E94A4200F900F900F907F
:10ADF0000F900F908F2D6DE00E942420DF91CF9156
:10AE00001F910F91FF90EF9008959F92AF92BF9284
:10AE1000CF92DF92EF92FF920F931F93DF93CF9326
:10AE2000CDB7DEB72D970FB6F894DEBF0FBECDBFFE
:10AE3000982E80E090E00E94B2847C018C0192E028
:10AE4000C92ED12CCC0EDD1E5E010894A11CB11CB4
:10AE500014C0C801B501A6010E942D85BC01009750
:10AE600079F0892D498196010E946D56C8010E9492
:10AE7000B2848C018E159F0519F00115110549F753
:10AE80002D960FB6F894DEBF0FBECDBFCF91DF91E8
:10AE90001F910F91FF90EF90DF90CF90BF90AF90F8
:10AEA0009F900895AF92BF92CF92DF92EF92FF9260
:10AEB0000F931F93CF93DF93082F0E94C06B6C01F9
:10AEC000802F68E277E00E94FE20802F6FE177E01C
:10AED0000E94FE20802F69E177E00E94FE20802FF3
:10AEE0006DE00E94242000D000D00F92EDB7FEB795
:10AEF0003196ADB7BEB711960C938AE097E0928376
:10AF000081838DE090E0948383830E94A4200F903E
:10AF10000F900F900F900F90802F6BEF76E00E94B4
:10AF2000FE200E94D46BEDB7FEB737970FB6F894AA
:10AF3000FEBF0FBEEDBF3196ADB7BEB711960C93F5
:10AF40002FEE36E032832183638374838583968377
:10AF50000E94A420EDB7FEB737960FB6F894FEBF57
:10AF60000FBEEDBF802F67EE76E00E94FE208DE6DB
:10AF700096E5602F0E94DD3A802F0E940557802FB2
:10AF80006AED76E00E94FE20802F0E943055802FCF
:10AF90006EEC76E00E94FE20802F0E94C755802F25
:10AFA00064EC76E00E94FE20C0E0D0E0EE24FF24B6
:10AFB0002FEBA22E26E0B22EC7010E94638C182F21
:10AFC00000D000D00F92EDB7FEB73196ADB7BEB747
:10AFD00011960C93B282A182D483C3830E94A420D1
:10AFE0000F900F900F900F900F90113019F068EBA9
:10AFF00076E002C06CEB76E0802F0E94FE20802F6E
:10B000006DE00E9424202196E8E0F0E0EE0EFF1EA5
:10B01000CF3FD10589F6802F6EEA76E00E94FE20B0
:10B02000D6014C914170802F64EA76E00E94BB4CBF
:10B03000F60140814470802F66E976E00E94BB4CA7
:10B04000D6014C914870802F6BE876E00E94BB4C93
:10B0500000D000D00F92EDB7FEB73196ADB7BEB7B6
:10B0600011960C938DE796E092838183D601169614
:10B070008C91838314820E94A420EDB7FEB7319691
:10B08000ADB7BEB711960C938EE696E0928381839E
:10B09000D60118968C91838314820E94A420EDB768
:10B0A000FEB73196ADB7BEB711960C938FE596E01B
:10B0B00092838183D6011B968C9122E3829FC001EB
:10B0C0001124948383830E94A420EDB7FEB73196A8
:10B0D000ADB7BEB711960C9380E596E0928381835D
:10B0E000D6011C968C9124E6829FC0011124948382
:10B0F00083830E94A4200F900F900F900F900F90C9
:10B10000F60181810E94AC1400D000D00F92EDB7FF
:10B11000FEB73196ADB7BEB711960C9323E436E077
:10B1200032832183948383830E94A4200F900F9005
:10B130000F900F900F90802F6DE376E00E94FE201D
:10B1400081E0DF91CF911F910F91FF90EF90DF9001
:10B15000CF90BF90AF9008951F93182F0E9405576E
:10B16000812F6FE777E00E94FE2081E01F91089514
:10B170001F93182F1F7701F11150862F0E94FB3D5E
:10B180008B3141F08C3171F08E30B1F4812F90E031
:10B1900008960DC083E0189FC00111240B966EE045
:10B1A00070E007C0812F90E0880F991F079669E033
:10B1B00070E00E949AA7162F812F1F9108951F9368
:10B1C000182F1F7711F480E01DC0862F0E94FB3DD1
:10B1D0008B3151F08C3171F08E3091F4E12FF0E031
:10B1E000E55CF64F84910EC0E12FF0E0E65BF64F90
:10B1F000849108C0E12FF0E0EA59F64F849102C033
:10B20000812F8F5F1F910895EF92FF920F931F93ED
:10B21000CF93DF93182F882319F0E0E4FE2E02C0AD
:10B2200070E2F72EC0E6D9E000E0EF2CE09430C0E9
:10B2300069858F2D862351F188850E94DF58682FFC
:10B24000812F0E9424202C813D814E815F81569563
:10B25000479537952795812F622F0E942420812FB3
:10B2600068810E94242069816F738C8180FD6064F5
:10B27000888587FD6068812F0E94242068856F770C
:10B28000812F0E94242089858E2189870F5F2B962C
:10B290008091200C081760F280E8DF91CF911F9118
:10B2A0000F91FF90EF9008950E94A33C81E00895D4
:10B2B000FF920F931F93CF93DF93042F442309F43E
:10B2C00041C0809154048823E9F1C0914604D09193
:10B2D00047042097B9F180E4C030D80798F511E011
:10B2E000BFE0FB2E2DC01031C0F4812F90E0FC0197
:10B2F000A4E0EE0FFF1FAA95E1F7E81BF90BEA5B4C
:10B30000FB4F8685882349F0608171816115710545
:10B3100031F080E46030780710F060E070E01F9D4D
:10B32000F0011124E85BFB4F01C031968081882336
:10B3300019F08132D1F70DC0CE010E94503C1F5F41
:10B34000101788F281E0DF91CF911F910F91FF904C
:10B3500008957068F1CF0E942B3B03C080E00E94EB
:10B36000988380E00E941681BC010097B9F703C062
:10B3700083E00E94988383E00E941681BC010097BD
:10B38000B9F703C082E00E94988382E00E94168190
:10B39000BC010097B9F781E008951F93182F60E072
:10B3A0002FEF3FE30E94974C009769F10E948E387F
:10B3B000FC01009721F4812F66E279E022C08185AB
:10B3C00090E0837090708130910581F0823091051A
:10B3D0001CF4892B39F017C08230910559F003977E
:10B3E00091F40CC0812F63E279E00BC0812F66E1FC
:10B3F00079E007C0812F69E079E003C0812F65E023
:10B4000079E00E94FE2081E01F9108950F931F9321
:10B41000CF93DF93182FFB01042F928180E02181CD
:10B4200030E0282B392BC90101978F5F9F4338F0FB
:10B43000812F62E00E942420C0E0D0E015C00023EC
:10B4400021F0C9010E94893C03C0C9010E948E38C5
:10B45000EC01009749F4002319F0812F6BE002C042
:10B46000812F6AE00E942420CE01DF91CF911F91AD
:10B470000F9108951F93CF93DF93182F41E00E94FF
:10B48000065AEC01009711F1812F60E00E94242000
:10B490002C813D814E815F8191E15695479537958D
:10B4A00027959A95D1F7812F622F0E9424202C8115
:10B4B0003D814E815F8189E1569547953795279566
:10B4C0008A95D1F7812F622F0E9424208FEFDF9180
:10B4D000CF911F9108951F93CF93DF93182F41E0D1
:10B4E0000E94065AEC01009799F0812F60E00E94BB
:10B4F00024202C813D814E815F8169E056954795DE
:10B50000379527956A95D1F7812F622F0E942420C5
:10B510008FEFDF91CF911F9108951F93CF93DF930A
:10B52000182F41E00E94065AEC01009781F0812F0C
:10B5300060E00E9424202C813D814E815F815695E0
:10B54000479537952795812F622F0E9424208FEFF2
:10B55000DF91CF911F9108951F93CF93DF93182F01
:10B5600041E00E94065AEC01009741F1812F60E012
:10B570000E942420888569850E94DF58682F812FCA
:10B580000E9424208C819D81AE81BF819C01AD01F0
:10B590005695479537952795622F6F7081709070FB
:10B5A000892B09F06061888587FD6062812F0E9488
:10B5B000242068856F77812F0E9424208FEFDF91F0
:10B5C000CF911F910895CF93DF93EB0141E00E944B
:10B5D000065AFC01009711F48FEF2DC08B8181304A
:10B5E00069F18130E0F0823019F0833019F50AC03A
:10B5F00022E025C06B3111F4246015C06C31D1F408
:10B60000286011C06C816E3011F423E00CC06C31E5
:10B6100011F427E008C06E3769F42BE004C08C8178
:10B620008E3741F420E080819181622F0E94DA3DC3
:10B6300080E001C082E0DF91CF91089521E06C812C
:10B640006E30C1F6F0CF1F93CF93DF93182FEB012D
:10B650006115710559F18F3F51F11370CB010E94B3
:10B66000DCA88F3708F08EE7133018F4113020F47F
:10B670001BC01330E1F40DC08B3199F4CE0162E4AC
:10B6800070E00E9441A9009711F0186010C014608A
:10B690000EC08C3111F417E00AC08E3711F41BE094
:10B6A00006C08E3019F403C08E3709F01FEF812FCA
:10B6B000DF91CF911F9108950F931F93CF93DF9345
:10B6C000082F442301F1809154048823E1F0C091B4
:10B6D0004604D09147042097B1F080E4C030D807E9
:10B6E000E8F111C080917204882369F086E694E045
:10B6F0000E94E64A8F3F39F067E574E00E94235BC1
:10B70000182F8F3F29F4802F62E00E942E4C21C019
:10B71000CE010E948E38892B21F0CE01612F0E942C
:10B72000DA3DCE01612F0E94623DCE010E94C184AC
:10B73000BC0180918104882341F0CB01BE01412FDF
:10B7400025E734E00E94848503C080E00E9498834E
:10B7500081E0DF91CF911F910F9108958091630453
:10B76000882309F0BFCFCFCF1F93CF93DF93182F3C
:10B77000442361F180915404882341F1C09146042F
:10B78000D0914704209711F180E4C030D80748F1E8
:10B790001DC0812F6BE00E942E4C1FC061858091DF
:10B7A0006304882339F087E594E00E94E64A682F15
:10B7B0008F3F61F080917204882359F0862F66E6EE
:10B7C00074E00E94235B682F8F3F19F4812F62E0A1
:10B7D000E2CFCE010E94DA3D81E0DF91CF911F914F
:10B7E0000895CE010E94893CFC010097B9F6D1CFA3
:10B7F000EF92FF921F93CF93DF93182F442351F1C1
:10B8000080915404882331F1C0914604D0914704BB
:10B81000C038D105F8F080E4C030D807D8F47E01F4
:10B820006F2D606C80E190E00E94C67C99233CF013
:10B8300081E190E06C2F0E94C67C97FF03C0812FAE
:10B8400067E00DC08CE190E065E041E00E94DC7CA7
:10B8500097FF03C0812F61E002C0812F60E00E944A
:10B860007D4ADF91CF911F91FF90EF9008950F9344
:10B870001F93CF93DF93182F80E190E00E94BC7C50
:10B8800097FD10C0082F805C883228F0812F61E07E
:10B890000E947D4A32C081E190E00E94BC7CEC01B4
:10B8A00097FF03C0812F67E0F3CF8CE190E065E064
:10B8B00041E00E94DC7C97FDE9CF00D000D00F92E0
:10B8C000EDB7FEB73196ADB7BEB711961C9383EDB9
:10B8D00097E092838183802F90E08F739070982FF0
:10B8E00088278C0F911D948383830E94A42081E07C
:10B8F0000F900F900F900F900F90DF91CF911F91AD
:10B900000F9108951F93182FFB01809163048823E2
:10B9100009F461C0442309F45EC080915404882373
:10B9200009F459C02091460430914704211531058E
:10B9300009F451C084E02130380708F45AC04BC0E4
:10B9400060915504709156046F3F710519F010F025
:10B9500060E070E083818434B1F085341CF482347B
:10B96000D1F516C0803551F08235A9F52930310561
:10B9700090F5822F81500E94A57C30C0C9010197AB
:10B980000E948F7C2BC0C90101970E94C67C26C0F3
:10B99000423038F06091550470915604683071055A
:10B9A00010F06FEF70E06F3FB1F0433058F08091CE
:10B9B0007204882339F04091640450916504423048
:10B9C000510510F04FEF50E04F3F29F0C9010197AA
:10B9D0000E94DC7C03C0812F61E007C0892B19F035
:10B9E000812F67E002C0812F60E00E947D4A1F9195
:10B9F0000895423008F0A4CFABCFFF920F931F936E
:10BA0000CF93DF93082FFB01442311F1809154045D
:10BA10008823F1F080914604909147040097C1F08B
:10BA200024E08130920708F459C012C08930910592
:10BA300078F481500E949A7C07C001970E94857C0F
:10BA400003C001970E94BC7CEC0197FF09C003C0B2
:10BA5000802F61E002C0802F67E00E947D4A38C0DD
:10BA60008DB79EB707970FB6F8949EBF0FBE8DBFD8
:10BA7000EDB7FEB73196ADB7BEB711960C9386ED14
:10BA800097E092838183D483C383D683C5830E9446
:10BA9000A420FC2E8DB79EB707960FB6F8949EBFD4
:10BAA0000FBE8DBF802F65E20E94242010E8C0E009
:10BAB000D0E0812F8F2111F460E301C061E3802F7A
:10BAC0000E94242016952196C830D10591F781E077
:10BAD000DF91CF911F910F91FF900895638164349E
:10BAE00009F4AFCF653424F4623409F0B1CFA9CFA3
:10BAF000603509F4A2CF623509F0AACF97CF1F9322
:10BB0000182F442319F5813031F481E063E478E0A3
:10BB10000E94FE201DC00E94DA1400D000D00F92B7
:10BB2000EDB7FEB73196ADB7BEB711961C9320E4C2
:10BB300038E032832183948383830E94A42081E0B0
:10BB40000F900F900F900F900F900FC0813011F455
:10BB500081E00BC06DE378E00E94FE2080914604F6
:10BB6000909147040E946E1480E01F910895EF9217
:10BB7000FF920F931F93CF93DF93082F442371F00D
:10BB800080915404882351F0209146043091470459
:10BB90002115310529F02533310510F020E030E082
:10BBA000122F2223D9F100D000D00F92EDB7FEB7AB
:10BBB0003196ADB7BEB711960C938FE498E092839F
:10BBC0008183238314820E94A4200F900F900F90F2
:10BBD0000F900F90812F8150602F0E94BE7F7C01BB
:10BBE000C0E0D1E010E00BC0183019F0CC0FDD1F21
:10BBF00006C0802F60E20E942420C1E0D0E0CE0188
:10BC00008E219F21892B19F0802F61E302C0802FA4
:10BC100060E30E9424201F5F103131F781E0DF9143
:10BC2000CF911F910F91FF90EF900895FF920F9386
:10BC30001F93F82EFB0181818150843310F082E044
:10BC400011C06F2D0E94BE7F8C018F2D60E00E947D
:10BC500024208F2D612F0E9424208F2D602F0E9481
:10BC600024208FEF1F910F91FF9008951F93182F9D
:10BC70004423A9F08091F20C282F30E0217030701D
:10BC800080915404882341F08091460490914704A8
:10BC90008230910508F49C01822F0E94C97F00D058
:10BCA00000D00F92EDB7FEB73196ADB7BEB7119683
:10BCB0001C9382E798E0928381838091F20C90E05C
:10BCC00081709070948383830E94A4200F900F90C2
:10BCD0000F900F900F9081E01F910895CF92DF9207
:10BCE000EF92FF920F931F93CF93DF93D82E8B0188
:10BCF00021E0281708F45AC0FB01828190E0877088
:10BD00009070D82FCC27818190E0C82BD92B219718
:10BD1000F7E0C83FDF0710F082E049C00E946812D8
:10BD2000982F8250823020F0973011F086E03FC08B
:10BD30007E01EE0CFF1CF801628167FD04C081E00A
:10BD400090E0E82AF92A88E5D89EE0011124CA5635
:10BD5000DC4F862F90E016E0969587951A95E1F7CF
:10BD6000CC24C394C8228E010B5A1F4FF801808146
:10BD70009181FFEF8F3F9F0749F060E04D2D0E94BA
:10BD8000E58E8FEF9FEFF80191838083C7016C2DC3
:10BD90004D2D0E94E58E882311F489E008C0CC2047
:10BDA00029F0FE01EB5AFF4FF182E08280E0DF9143
:10BDB000CF911F910F91FF90EF90DF90CF9008955A
:10BDC0000F931F93CF93DF93082FFB01828190E0A5
:10BDD00087709070D82FCC27818190E0C82BD92B09
:10BDE000219787E0C83FD80710F082E01BC0CE0142
:10BDF0000E94358C873621F0873411F010E001C0A5
:10BE000014E0CE01880F991F0E94638C039709F4F8
:10BE10001160802F60E00E942420802F612F0E94FB
:10BE200024208FEFDF91CF911F910F910895AF9252
:10BE3000BF92DF92EF92FF920F931F93CF93DF9306
:10BE4000D82E142F0E946812882319F48D2D66E0D5
:10BE500061C08D2D60E0412F28EF37E00E94974CA4
:10BE60005C01009709F49CC021E02D1508F498C0EE
:10BE7000123008F459C088E5D89E7001112486E973
:10BE800093E0E80EF91EE701CB5ADF4F88819981D4
:10BE9000AFEF8F3F9A0741F060E04D2D0E94E58E95
:10BEA0008FEF9FEF9983888380915704873411F433
:10BEB00090E012C0823511F491E00EC080916304CD
:10BEC000882339F080915504909156048230910571
:10BED00010F082E090E0982F123059F080917204B7
:10BEE000882339F000916404109165040230110533
:10BEF00010F000E010E0E5012197CC0FDD1FC90F25
:10BF0000D11DCE01602F4D2D0E94E58E882329F48E
:10BF10008D2D69E00E942E4C44C0002329F0F701CA
:10BF2000EB5AFF4FD183C083C50101970E94358C26
:10BF3000082F112707FD1095C8010E9412A97C0146
:10BF4000C8010E94FAA82DB73EB7295030400FB65D
:10BF5000F8943EBF0FBE2DBFEDB7FEB73196ADB71B
:10BF6000BEB71196DC9226ED38E032832183B4828D
:10BF7000A382F682E58220E030E0892B11F021E0F7
:10BF800030E0308727830E94A42081E02DB73EB7A0
:10BF9000275F3F4F0FB6F8943EBF0FBE2DBF01C0C5
:10BFA00081E0DF91CF911F910F91FF90EF90DF9093
:10BFB000BF90AF9008956F927F928F929F92AF92B1
:10BFC000BF92CF92DF92EF92FF920F931F93DF9376
:10BFD000CF93CDB7DEB760970FB6F894DEBF0FBE34
:10BFE000CDBFC82ED42E60E02FEF3FE30E94974CC8
:10BFF0007C01009709F4DFC021E0D21609F063C08C
:10C000000E9442879A83898300D000D00F92EDB7B7
:10C01000FEB73196ADB7BEB71196CC9284EF98E0DB
:10C0200092838183F482E3820E94A4200F900F9078
:10C030000F900F900F903E010894611C711C05E059
:10C04000802E912C8C0E9D1E1DEEA12E18E0B12E7F
:10C05000B1E1EB2EF12CEC0EFD1E30C080E1B301FE
:10C060000E948C818401F8019181992311F12DB7EF
:10C070003EB7275030400FB6F8943EBF0FBE2DBFDD
:10C08000EDB7FEB73196ADB7BEB71196CC92B2827E
:10C09000A182D8018C9183831482958316820E9499
:10C0A000A420EDB7FEB737960FB6F894FEBF0FBECB
:10C0B000EDBF0E5F1F4F0E151F05A9F689819A81EE
:10C0C000892B61F678C0F2E0DF1619F001E012E08A
:10C0D00070C080916304882341F000915504109151
:10C0E00056040F3F110519F010F000E010E0C701F1
:10C0F000602F0E94D5872DB73EB7295030400FB62C
:10C10000F8943EBF0FBE2DBFEDB7FEB73196ADB769
:10C11000BEB71196CC9221EE38E032832183F482AF
:10C12000E38205831682878310860E94A420EDB7E0
:10C13000FEB739960FB6F894FEBF0FBEEDBF3BC0F9
:10C140000031A8F4802F90E0FC01A4E0EE0FFF1F67
:10C15000AA95E1F7E81BF90BEA5BFB4F868588237C
:10C1600031F0608171816F3F710519F010F060E06E
:10C1700070E01031B8F41D15A8F4812F90E0FC0197
:10C1800074E0EE0FFF1F7A95E1F7E81BF90BEA5B0D
:10C19000FB4F8685882331F0408151814F3F510507
:10C1A00019F010F040E050E0C7010E9465880E5F72
:10C1B0001E5F0D1528F281E060960FB6F894DEBF81
:10C1C0000FBECDBFCF91DF911F910F91FF90EF90E8
:10C1D000DF90CF90BF90AF909F908F907F906F90A7
:10C1E0000895EF92FF920F931F93CF93DF93182F31
:10C1F000042F60E02FEF3FE30E94974CEC01009783
:10C2000009F45BC00E948E387C01009771F4023003
:10C2100018F4812F6AE011C0CE010E94893C7C0194
:10C22000009729F4812F6BE008C00230F0F00E94E3
:10C230001522882329F0812F68E00E942E4C3EC0F1
:10C24000D70114966D917C911597802F40E052E0B4
:10C2500021E008E00E941B4ABC01CE01412F0E9450
:10C26000F13CCE0160E00E94C0380E946812882331
:10C2700021F4812F62E40E942E4C00D000D00F9256
:10C28000EDB7FEB73196ADB7BEB711961C938AEFE6
:10C2900098E092838183D483C3830E94A4200F906B
:10C2A0000F900F900F900F90F70164817581812F8F
:10C2B00040E052E028E00E94D64C81E0DF91CF912F
:10C2C0001F910F91FF90EF900895EF92FF920F93BF
:10C2D0001F93CF93DF93182F042F60E02FEF3FE3DE
:10C2E0000E94974CEC01009709F45BC00E948E38C5
:10C2F0007C01009771F4023018F4812F6AE011C0BC
:10C30000CE010E94893C7C01009729F4812F6BE0CB
:10C3100008C00230F0F00E941522882329F0812FF6
:10C3200068E00E942E4C3EC0D70114966D917C911E
:10C330001597802F42E050E021E008E00E941B4A60
:10C34000BC01CE01412F0E94F13CCE0160E00E9471
:10C35000C0380E946812882321F4812F62E40E9471
:10C360002E4C00D000D00F92EDB7FEB73196ADB78E
:10C37000BEB711961C9380E099E092838183D483A9
:10C38000C3830E94A4200F900F900F900F900F90E6
:10C39000F70164817581812F42E050E028E00E941E
:10C3A000D64C81E0DF91CF911F910F91FF90EF90DC
:10C3B0000895DF92EF92FF920F931F93CF93DF9335
:10C3C000D82E142F60E02FEF3FE30E94974C7C01A2
:10C3D000009709F4E8C00E948E38EC01009771F4D0
:10C3E000123018F48D2D6AE012C0C7010E94893CFA
:10C3F000EC01009731F48D2D6BE009C0123008F488
:10C4000081C00E941522882329F08D2D68E00E94AA
:10C410002E4CCAC08C819D81AE81BF81BC016E7FD4
:10C42000AC0141705070123059F080917204882331
:10C4300039F020916404309165042230310508F010
:10C440009A01232B09F06160812F42E050E024E043
:10C4500004E00E941B4ABC01C7014D2D0E94F13C23
:10C46000888569850E94DF58482F8091630488235E
:10C4700039F020915504309156042038310508F0E8
:10C48000242F80917504863411F411E01AC082358E
:10C4900011F410E016C040E050E0888587FF02C02C
:10C4A00041E050E0143058F080918104882339F045
:10C4B00080917304909174048230910508F0CA0150
:10C4C000182F213029F4C7010E948D3600E005C0E5
:10C4D000822F69850E94B858082F1111006868855D
:10C4E000802F862787FF05C06078C7014D2D0E94E9
:10C4F0002A3DC701602F4D2D0E942A3DC70160E0F3
:10C500000E94C0380E946812823019F48D2D61E4B7
:10C5100006C00E946812833021F08D2D62E40E94D3
:10C520002E4C888569850E94DF58682F8C8180FD9C
:10C5300003C040E350E002C041E350E0888587FD3E
:10C5400003C022E730E002C026E630E08DB79EB798
:10C550000B970FB6F8949EBF0FBE8DBFEDB7FEB719
:10C560003196ADB7BEB71196DC928DE299E0928319
:10C570008183F482E3826583168250874783328702
:10C5800021870E94A4208DB79EB70B960FB6F89412
:10C590009EBF0FBE8DBF6C817D818D2D42E050E02E
:10C5A00024E00E94D64C81E0DF91CF911F910F9142
:10C5B000FF90EF90DF900895AF92BF92CF92DF92FD
:10C5C000EF92FF920F931F93CF93DF93C82E882390
:10C5D00049F042E2A42E4CE0B42E39EFE32E3CE0C9
:10C5E000F32E08C02AE8A22E2CE0B22E93EFE92EFB
:10C5F0009CE0F92EDD2433C0F8940D2D10E0C70126
:10C60000B8010E949691882341F1F801EE0FFF1FB7
:10C61000D501AE0FBF1FE150F34FCD91DC911197C3
:10C6200080819181C82BD92B1D921C928081918190
:10C63000C817D90721F4C701B8010E9480917894E6
:10C640006D2D6F5F8C2D0E9424208C2D6D2F0E94EC
:10C6500024208C2D6C2F0E9424207894D3940E9447
:10C66000C06BFC018085D81638F28C2D60E00E94EA
:10C6700024208FEFDF91CF911F910F91FF90EF90CA
:10C68000DF90CF90BF90AF900895CF92DF92EF925E
:10C69000FF920F931F93DF93CF93CDB7DEB7C254B2
:10C6A000D0400FB6F894DEBF0FBECDBFC82EDD243C
:10C6B0007E010894E11CF11C8C2D0E944E908C018F
:10C6C0008FEF0F3F180719F1C8010E94358C282FF2
:10C6D000C8010196F7018083892F877081832734F1
:10C6E00011F0273629F48068F7018183273411F08F
:10C6F000223521F4F701818180648183D394F0E2B3
:10C70000DF1629F082E090E0E80EF91ED5CF8C2DDF
:10C710006D2D0E942420ED2CFF24EE0CFF1C8E01B9
:10C720000F5F1F4FD02E06C0F80161918F018C2D35
:10C730000E942420802F8D1990E08E159F05A4F370
:10C740008FEFCE5BDF4F0FB6F894DEBF0FBECDBFCD
:10C75000CF91DF911F910F91FF90EF90DF90CF90DD
:10C7600008951F93CF93DF93182F0E94F690692F9F
:10C77000629566956695617095FD646080FD686060
:10C7800097FD6062EC01CE7FDF71209709F0606851
:10C79000812F0E9424202097A1F0CE0196958795A5
:10C7A000682F6170C2FD6064C97F209709F06068DE
:10C7B000812F0E942420CD2B21F0812F60E00E9448
:10C7C00024208FEFDF91CF911F910895CF92DF92B8
:10C7D000FF920F931F93DF93CF93CDB7DEB7609790
:10C7E0000FB6F894DEBF0FBECDBFF82E63E00E94F7
:10C7F00024208F2D62E00E9424208F2D61E00E9472
:10C8000024208F2D61E00E9424208F2D64E00E945F
:10C8100024200E94D46B2DB73EB7285030400FB66D
:10C82000F8943EBF0FBE2DBFEDB7FEB731968E0117
:10C830000F5F1F4FADB7BEB712961C930E931197A3
:10C8400020E73AE03383228364837583868397836A
:10C850000E9473A9EDB7FEB738960FB6F894FEBFE5
:10C860000FBEEDBF79E0C72ED12CCC0EDD1ED80156
:10C870006C916295607F11968C918053682B0E5F4E
:10C880001F4F8F2D0E9424200C151D0581F780E07D
:10C8900060960FB6F894DEBF0FBECDBFCF91DF918B
:10C8A0001F910F91FF90DF90CF9008950E94D37F4A
:10C8B00080E008950F931F93CF93DF938B01823015
:10C8C00030F5FB01828190E087709070D82FCC27E3
:10C8D000818190E0C82BD92B2197F7E0C83FDF0773
:10C8E00010F082E015C00E946812982F82508230AA
:10C8F00020F0973011F086E00BC0F8016281669558
:10C9000066956695CE01880F991F0E946B3480E072
:10C91000DF91CF911F910F910895CF93DF93EB019A
:10C9200040E00E94065AFC01009711F48FEF1CC0F2
:10C9300081858370833011F082E016C04B816C8159
:10C9400070E07695762F662777956795842F90E02F
:10C950008F779070682B792B441F4427441F808168
:10C9600091810E94E03780E0DF91CF910895DF92BE
:10C97000EF92FF920F931F93CF93DF93D82EEB018B
:10C9800041E00E94065A7C01009711F48FEF5DC0D0
:10C99000FC0181850E94053EF701048115812681F5
:10C9A00037814B819C818D3100F12170307050E0D6
:10C9B00060E070E0F1E1440F551F661F771FFA95A4
:10C9C000D1F7892F90E0A0E0B0E0E9E1880F991F4E
:10C9D000AA1FBB1FEA95D1F7482B592B6A2B7B2B3B
:10C9E000402B512B622B732B23C02170307E50E0E3
:10C9F00060E070E081E1440F551F661F771F8A9544
:10CA0000D1F7402B512B622B732B892F90E0A0E0A4
:10CA1000B0E08F709070A070B07019E1880F991F0E
:10CA2000AA1FBB1F1A95D1F7482B592B6A2B7B2BBA
:10CA3000F701808191812D2D0E94B83CF701808102
:10CA4000918161E00E94C03880E0DF91CF911F9119
:10CA50000F91FF90EF90DF900895FF920F931F9337
:10CA6000CF93DF93F82E8B0141E00E94065AEC0130
:10CA7000009711F48FEF21C08C819D81AE81BF8121
:10CA80009170AE7FF801438150E060E070E019E002
:10CA9000440F551F661F771F1A95D1F7482B592B46
:10CAA0006A2B7B2B888199812F2D0E94B83C88812D
:10CAB000998160E00E94C03880E0DF91CF911F91A2
:10CAC0000F91FF900895FF920F931F93CF93DF93E1
:10CAD000F82E8B0141E00E94065AEC01009711F4F8
:10CAE0008FEF1EC08C819D81AE81BF8181709E7F42
:10CAF000F801438150E060E070E0440F551F661F6D
:10CB0000771F482B592B6A2B7B2B888199812F2DDE
:10CB10000E94B83C8881998160E00E94C03880E022
:10CB2000DF91CF911F910F91FF900895CF92DF92E7
:10CB3000EF92FF920F931F93CF93DF93C82E8B0139
:10CB4000F42E41E00E94065AEC01009711F48FEF99
:10CB500078C00E941522882311F088E072C0D801A5
:10CB60001396DC90FF2071F0B1E0DB1631F4888180
:10CB700099810E948D36DD2405C08D2D69850E9426
:10CB8000B858D82EF8016481262F30E065FF02C026
:10CB9000F0E8DF2AEC80FD800E811F818EEF9FEF91
:10CBA000AFEFBFEFE822F9220A231B2324FF08C0BE
:10CBB00081E090E0A0E0B0E0E82AF92A0A2B1B2BE4
:10CBC00067FF15C081EE9FEFAFEFBFEFE822F922BC
:10CBD0000A231B232F703070220F331FC901AA278D
:10CBE00097FDA095BA2FE82AF92A0A2B1B2B6885F6
:10CBF0008D2D862787FF06C06078888199814C2D0E
:10CC00000E942A3D888199816D2D4C2D0E942A3DDC
:10CC100088819981B801A7012C2D0E94B83C888198
:10CC2000998160E00E94C0380E946812833041F010
:10CC3000873031F0823011F082E403C081E401C01A
:10CC400080E0DF91CF911F910F91FF90EF90DF90E7
:10CC5000CF90089540E00E949665089541E00E94BB
:10CC6000966508951F93CF93DF93182FEB010E94D1
:10CC70006812833011F082E43EC0812FBE0141E092
:10CC80000E94065AFC01009711F48FEF34C0118600
:10CC900013821282148215821682178210866C818A
:10CCA00070E080E090E0982F872F762F66272D8107
:10CCB00030E040E050E0A90133272227622B732B9C
:10CCC000842B952B2B8130E040E050E0622B732BBE
:10CCD000842B952B2E8130E040E050E0522F4427EA
:10CCE00033272227622B732B842B952B4081518174
:10CCF0000E94B23280E0DF91CF911F9108951F937F
:10CD0000CF93DF93182F41E00E94065AEC01009761
:10CD100001F1812F60E00E94242069856370812FDA
:10CD20000E94242089850E940738892B19F0812FC1
:10CD30006CE105C089850E94FB3D682F812F0E9410
:10CD40002420812F6FEF0E942420812F6FEF0E94FB
:10CD500024208FEFDF91CF911F910895CF92DF9222
:10CD6000EF92FF920F931F93CF93DF93D82EEB0197
:10CD7000C42E21E0281708F4F9C028813FE1F32EE2
:10CD8000F222422F50E0CA01807E907080349105DB
:10CD900009F49AC08134910534F4009789F08097A2
:10CDA00009F0E4C050C08038910509F4B5C0803C5A
:10CDB000910509F4C7C08036910509F0D7C0A4C019
:10CDC00081E08C1508F0D4C00981802F90E00E948A
:10CDD000893CFC01009709F4C9C064817581F4FEA7
:10CDE00003C0EB01C16002C0EB01CE7F1F2D1F709D
:10CDF000F0841F3021F46F2D6095607817C0818515
:10CE0000112389F00E94FB3D8C3139F08E3739F0C7
:10CE10008B3149F4110F115006C0110F04C089E085
:10CE2000189F102D11246F2D6078612B802F90E0BA
:10CE30004D2D0E942A3D802F90E0BE014D2D0E9475
:10CE4000F13C802F5CC088E5D89E70011124E6E992
:10CE5000F3E0EE0EFF1E237F288387010B5A1F4F3E
:10CE6000F80180819181FFEF8F3F9F0749F060E0DB
:10CE70004D2D0E94E58E8FEF9FEFF8019183808307
:10CE80002881203209F472C0233209F46FC0F1E026
:10CE9000FC1508F06DC06981213231F4C62FD0E055
:10CEA0002197CC0FDD1F05C0C62FD0E0CC0FDD1FB2
:10CEB0002197CE0161E04D2D0E94E58EF701EB5ADE
:10CEC000FF4FD183C08352C021E02C1508F050C021
:10CED0001981812F90E00E94103D9B01AC01217EC1
:10CEE0008F2D90E08F709070880F991F282B392B11
:10CEF000812F90E0B9014D2D0E94F13C812F90E0EF
:10CF000060E00E94C03832C020FF02C080E001C053
:10CF100083E00E9483122AC0FF2011F480E015C034
:10CF200000E0802F6D2D0E94A57F182F8D2D692F79
:10CF30000E9424208D2D612F0E9424200F5F0F1549
:10CF400080F314C0FF2021F481E00E94C97F0EC04D
:10CF50008F2D81506D2D0E94A57F182F8D2D692F4B
:10CF60000E9424208D2D612F0E94242081E001C089
:10CF700080E0DF91CF911F910F91FF90EF90DF90B4
:10CF8000CF900895BF92CF92DF92EF92FF920F93CE
:10CF90001F93CF93DF93B82E81E08B1508F437C32E
:10CFA00088E5B89E70011124E6E9F3E0EE0EFF1E5D
:10CFB000E701C95ADF4F888187FD29C38B2D0E9465
:10CFC00010208C01FFEF8F3F9F0709F420C3888159
:10CFD0008068888344E5C42ED12CCE0CDF1CF6017A
:10CFE00080818823F1F0F7016081718182819381D2
:10CFF00068537F4F8F4F9F4F0E941119882389F0EC
:10D00000F6018081882349F0888180FD0AC0F701FC
:10D010008481883531F0883721F0F701EC5AFF4FD1
:10D0200010828091C5079091C607A091C707B09163
:10D03000C807F70180839183A283B383EC5AFF4F23
:10D040008081803508F01082C7010E94F74988234B
:10D05000B1F00830110551F4F701EC5AFF4F80810F
:10D06000882309F4C6C281508083C3C2011511050B
:10D0700009F4BFC20D30110511F400E010E0F70112
:10D08000EC5AFF4F8081D701A80FB11D14960C9365
:10D09000D82ED394D082DD2091F0F701E95AFF4FCA
:10D0A000808190E0EC01C170D07080FDA9C2F701D1
:10D0B0008481883509F4A4C2883709F4A1C2B70174
:10D0C0006C5F7F4F8B2D4D2D0E94AE66882309F03B
:10D0D0008CC28FC2012B09F08CC2F701EC5AFF4FB2
:10D0E000108287010C5F1F4FF701E95AFF4F8081C3
:10D0F00080FD03C087010B5F1F4FF80180818823EB
:10D1000009F443C2C80161E275E043E050E00E94C7
:10D110002CA9892B59F4CBE5DAE4C80103960E94C7
:10D1200061A9C8010E94124BD82E28C2C8010E94D2
:10D1300061A9C8010E94124BD82EC8016FE175E0A9
:10D140000E941AA9892B39F0C8016DE175E00E948F
:10D150001AA9892B19F4C3EDDAE410C2C8016AE1F7
:10D1600075E00E941AA9892B19F4CDECDAE406C205
:10D17000C80167E175E00E941AA9892B19F4C7EC70
:10D18000DAE4FCC1C80164E175E00E941AA9892BA8
:10D1900019F4C1ECDAE4F2C1C80162E175E00E9461
:10D1A0001AA9892B39F0C8016DE075E00E941AA90F
:10D1B000892B19F4C8E3D0E5E1C1C8016BE075E043
:10D1C0000E941AA9892B39F0C80168E075E00E9415
:10D1D0001AA9892B19F4C4E2D0E5D0C1C80163E0D3
:10D1E00075E00E941AA9892B19F4C2EDDFE4C6C1CB
:10D1F000C80161E075E00E941AA9892B19F4C9EDF4
:10D20000D1E6BCC1C8016EEF74E00E941AA9892B57
:10D2100019F4CDECD9E5B2C1C8016CEF74E00E94FD
:10D220001AA9892B19F4C5E6D1E6A8C1C80169EF8E
:10D2300074E00E941AA9892B19F4C1EFD0E69EC1AF
:10D24000C80166EF74E00E941AA9892B19F4CBED8E
:10D25000DFE594C1C80164EF74E00E941AA9892B2C
:10D2600019F4C7E1DFE58AC1C80162EF74E00E94EA
:10D270001AA9892B19F4C4EFDFE480C1C80160EF5B
:10D2800074E00E941AA9892B19F4CDEFD4E576C178
:10D29000C8016DEE74E00E941AA9892B19F4C5E744
:10D2A000D3E56CC1C8016AEE74E00E941AA9892B0B
:10D2B00019F4C6E3DEE562C1C80167EE74E00E94BE
:10D2C0001AA9892B19F4C7EBDDE558C1C80164EE32
:10D2D00074E00E941AA9892B19F4CAE2D3E54EC161
:10D2E000C80161EE74E00E941AA9892B19F4C7E005
:10D2F000DCE644C1C8016FED74E00E941AA9892BD5
:10D3000019F4CFE7DDE53AC1C8016CED74E00E9485
:10D310001AA9892B19F4C6EAD2E530C1C80169ED12
:10D3200074E00E941AA9892B19F4CAE6DDE426C12B
:10D33000C80166ED74E00E941AA9892B19F4C1E2B4
:10D34000DDE41CC1C80163ED74E00E941AA9892BB9
:10D3500039F0C80160ED74E00E941AA9892B19F414
:10D36000CEEED0E50BC1C8016BEC74E00E941AA9A7
:10D37000892B51F1C80166EC74E00E941AA9892B2F
:10D3800069F1C80161EC74E00E941AA9892BE1F0EF
:10D39000C8016CEB74E00E941AA9892BF9F0C8014E
:10D3A00067EB74E00E941AA9892B71F0C80162EB47
:10D3B00074E00E941AA9892B89F0C8016DEA74E013
:10D3C0000E941AA9892B19F4CDEFDCE5D7C0C8015A
:10D3D00068EA74E00E941AA9892B19F4C2E8DCE516
:10D3E000CDC0C80163EA74E00E941AA9892B19F420
:10D3F000C7E3DCE5C3C0C8016EE974E00E941AA966
:10D40000892B19F4C8EFDBE5B9C0C8016BE974E0FA
:10D410000E941AA9892B19F4C4EBDBE5AFC0C8013F
:10D4200063E974E00E941AA9892B19F4CCEAD8E5C3
:10D43000A5C0C8016CE874E00E941AA9892B19F4F0
:10D44000CCE5DBE59BC0C80163E874E00E941AA943
:10D45000892B19F4CBEAD9E591C0C8016BE774E0D8
:10D460000E941AA9892B19F4CBEBD5E587C0C80116
:10D4700064E774E00E941AA9892B19F4C8E5D9E57C
:10D480007DC0C8016BE674E00E941AA9892B19F4CB
:10D49000C4E5D9E573C0C80163E674E00E941AA927
:10D4A000892B19F4C1E6D6E569C0C8016BE574E0C3
:10D4B0000E941AA9892B19F4C2E5D7E55FC0C801FB
:10D4C00064E574E00E941AA9892B19F4CFEAD4E527
:10D4D00055C0C8016DE474E00E941AA9892B19F4A3
:10D4E000CDE1D4E54BC0C80169E474E00E941AA9FB
:10D4F000892B19F4CCEFD1E541C0C80166E474E092
:10D500000E941AA9892B19F4CBECD1E537C0C801C8
:10D5100062E474E00E941AA9892B19F4C1E6D0E5EF
:10D520002DC0C80169E374E00E941AA9892B19F47F
:10D53000CDEEDFE423C0C80165E374E00E941AA9C0
:10D54000892B19F4C1E7DFE419C0C80160E374E076
:10D550000E941AA9892B19F4C1E5DFE40FC0C801A4
:10D560006BE274E00E941AA9892B19F4C8EBDDE480
:10D5700005C08B2D61E00E942E4C05C08B2DB8019B
:10D580004D2DFE0109958823A1F18B2D68E274E0F1
:10D590000E94FE202EC0CD2B31F0B7016C5F7F4F73
:10D5A000F701948106C0B7016B5F7F4FDA94F701F2
:10D5B0009581E4E0F1E012C0891779F48181D816F1
:10D5C000C0F00280F381E02D309779F08B2D099522
:10D5D000682F8F3F51F08B2D06C0349680818823B1
:10D5E00059F78B2D61E00E942420F701EC5AFF4F80
:10D5F0001082F701E95AFF4F80818F77808307C03F
:10D60000C7010E94F749882309F064CDC4CFDF9198
:10D61000CF911F910F91FF90EF90DF90CF90BF902F
:10D6200008956F5F7F4F42E00E94AE668FEF0895CE
:10D630006F5F7F4F41E00E94AE668FEF08958230AA
:10D64000C0F4282F30E088E590E0289FF001299F62
:10D65000F00D389FF00D1124EA56FC4FEC5AFF4FA5
:10D660001082339610828FEF9FEF929382930E94E5
:10D67000A49008951F93182F823118F026EF3EE0F2
:10D6800031C00E94C06BFC012581223079F023302B
:10D69000B9F0812F90E02130E9F49C0154E0220F91
:10D6A000331F5A95E1F72A58354F1CC0212F30E01F
:10D6B00044E0220F331F4A95E1F72A56344F12C037
:10D6C000212F30E094E0220F331F9A95E1F72A547E
:10D6D000334F08C09C0184E0220F331F8A95E1F785
:10D6E0002A52324FC9011F910895882319F02BE463
:10D6F0003FE015C00E94C06BFC018581823039F08B
:10D70000833041F0813049F427E03FE008C028E150
:10D710003FE005C029E23FE002C02AE33FE0C90143
:10D7200008951F93182F833218F027EA38E125C097
:10D730000E94C06BFC018581823059F0833081F0FA
:10D740008130A9F481E1189F90011124255A304FAE
:10D7500014C081E1189F9001112422553E4E0DC046
:10D7600081E1189F900111242F5F3B4E06C081E19B
:10D77000189F900111242C5A394EC9011F91089508
:10D780008EE395E0089580913F0590E008958091A3
:10D790004D05089580913E05089590913E0598238A
:10D7A00009F091E0892F08952CEF3FEF41E050E020
:10D7B0004BBFF90127913791479156915070B901AC
:10D7C000CA0108958FEF9FEFA1E0B0E0ABBFFC016D
:10D7D0008791823029F4079902C080E8089582E099
:10D7E0000895EEE5F5E080819181892B29F0838110
:10D7F000882311F4118210828381882311F08150D3
:10D800008383349685E0EE36F80769F708950E9421
:10D810004D32F89488E181BD8BE081BDFFCF0E943D
:10D820008E38DC010097C1F0EEE5F5E02081318112
:10D830008D919C9111972817390739F012968D9187
:10D840009C9113972817390711F41182108234968E
:10D8500085E0EE36F80751F708957F928F929F92F8
:10D86000AF92BF92CF92DF92EF92FF920F931F93EE
:10D87000DF93CF9300D000D000D0CDB7DEB7782EA5
:10D880005B01042FFE01319686E0DF011D928A952F
:10D89000E9F7CF010E94256FEEE5F5E014E088245A
:10D8A0009924143029F480819181892B09F4182D51
:10D8B000808191818A159B0509F0E5C0F401EE0F86
:10D8C000FF1FEE0FFF1FE25AFA4F88E08383F40137
:10D8D000EE0FFF1FEE0FFF1FE05AFA4F80818F5FA0
:10D8E0008083833008F403C1C5010E94893C6C0128
:10D8F000009709F4FCC0BFEF7B16B1F5FC01448131
:10D900005581002319F0C501BA0129C0C501D6010E
:10D9100018966C910E948F44F6011185C5010E94F2
:10D92000C184BC01812F0E946E44D60114962D91B2
:10D930003D914D915C9117979A0144275527C50158
:10D94000B9010E94C43EF60182819381009749F09B
:10D950000E94893CFC0164817581808191810E94D3
:10D96000B13E0E94233E82C0DC0114962D913D9170
:10D970004D915C911797002369F07E010894E11C9A
:10D98000F11CC70160E000E00E944A6F872D68E04B
:10D99000A7016AC000E0FC0182819381892B09F014
:10D9A00001E07E010894E11CF11CC701D601189624
:10D9B0006C910E944A6F872D67E0A7010E94E36F78
:10D9C000F60181858F778B8382819381892B41F446
:10D9D000C5010E94C184BC01CE0104960E94256F3E
:10D9E0000E94C1778823E1F3872D69E08E010F5FE4
:10D9F0001F4FA8010E94E36FD60114964D915D91CF
:10DA00006D917C911797C8010E94316F0E94C17778
:10DA10008823E1F3872D6DE05E010894A11CB11C01
:10DA2000A5010E94E36FF601828193810E948E38E6
:10DA30008C010097D9F0DC016D917C91C5010E94A9
:10DA4000256FF8012481358146815781C50160E049
:10DA500000E00E944A6F0E94C1778823E1F3872D7E
:10DA600068E0AE014F5F5F4F0E94E36F880C991C26
:10DA7000880C991C8EE595E0880E991ED4011D92A4
:10DA80001C9281E035C00894811C911C3496B4E04E
:10DA90008B16910409F005CF143041F48FEF66E046
:10DAA000AE014F5F5F4F0E94E36F21C00E94153EA1
:10DAB0008A159B0519F40E94864007C08FEF65E028
:10DAC000AE014F5F5F4F0E94E36FE12FF0E0EE0F7A
:10DAD000FF1FEE0FFF1FDF01A25ABA4F1196BC9233
:10DAE000AE92E05AFA4F108288E013968C9380E051
:10DAF00026960FB6F894DEBF0FBECDBFCF91DF9153
:10DB00001F910F91FF90EF90DF90CF90BF90AF905B
:10DB10009F908F907F9008957F928F929F92AF9267
:10DB2000BF92CF92DF92EF92FF920F931F93DF93FA
:10DB3000CF9300D000D000D0CDB7DEB7782E4B0108
:10DB40007A01CB010E94893C5C01009709F452C024
:10DB5000C7010E94893C6C01009709F44BC0D501B4
:10DB600019968C910E94FB3D8C01F60181850E94E3
:10DB7000FB3D9801281B390BC90137FF03C0909565
:10DB800081959F4F0297B4F03FEF731621F481E027
:10DB90000E94AC3E2FC0FE01319686E0DF011D924F
:10DBA0008A95E9F781E08983872D61E2AF010E94C0
:10DBB000E36F20C000E0872DB70141E00E942D6C8B
:10DBC000882389F0F6018085D50118969C918927D4
:10DBD00087FF04C0E0E0F0E8EE2AFF2AC401B701A5
:10DBE0000E94503C07C00E94C1778823E1F30F5F79
:10DBF000043109F726960FB6F894DEBF0FBECDBFED
:10DC0000CF91DF911F910F91FF90EF90DF90CF9018
:10DC1000BF90AF909F908F907F9008951F93CF9368
:10DC2000DF93EB016115710599F08F3F71F410E0FE
:10DC30008FEFBE0140E00E942D6C0E94C1778823C7
:10DC4000E1F31F5F1A30A1F703C040E00E942D6C82
:10DC5000DF91CF911F910895CF93DF93C0E0D0E083
:10DC6000CE010E940CACFE01E25CFA4F6081861787
:10DC700019F0CE010E941EACA8952196C032D105A4
:10DC800079F7DF91CF910895982F909520913E05D7
:10DC9000922390933E0582FF02C00E94CB300E94E7
:10DCA0002C6E089590913E05982B90933E0582FF2F
:10DCB00002C00E94CB300E942C6E08951F93182F33
:10DCC00082FD136011FD116010934D050E942C6EB2
:10DCD000812F0E945D231F9108951F93182F883074
:10DCE00008F017E080913F05181751F010933F0599
:10DCF0000E942C6E812F68E04EE421E00E94D71331
:10DD00001F910895809343050E942C6E0895909171
:10DD10004305973008F091E080E1EEE3F5E0DF01A4
:10DD20001D928A95E9F788E1809342059093430517
:10DD300097E090933F0584E18093440582E08093CF
:10DD4000490582E380934A058CE080933E059093D9
:10DD50004D0583E090E00E94E48C0E942C6E0895B3
:10DD60000E944D3284E06EEB71E00E940B2085E052
:10DD700066EC71E00E940B2085E99DE968EC70E09B
:10DD80000E94691E80E060E00E942A1F83E00E94DA
:10DD9000916BBC0182E00E94FE200E942B3B0E94FE
:10DDA0009B830E94876E0E94076C08958EE395E026
:10DDB00060E070E040E250E00E94FCAB80914005E2
:10DDC000909141058F5F9F4F11F40E94876E809163
:10DDD0003F05883018F087E080933F0580914B0520
:10DDE00090914C05885F974020F010924C0510925E
:10DDF0004B0580914305873010F0109243058AEF60
:10DE00009FEFA1E0B0E0ABBFFC019791892F81505B
:10DE10008E3F10F490936F000895682780E097E09C
:10DE200067FF03C0660F692701C0660F8F5F8830E8
:10DE3000B9F7862F08952091E8053091E905909370
:10DE4000E9058093E805C9010895FC01862F8F77C5
:10DE50008083660F672F661F770B71956F776183DD
:10DE60000895FC01CB01AA27BB278F77828327E186
:10DE700076956795579547952A95D1F7842F8F7793
:10DE8000838397E076956795579547959A95D1F74F
:10DE9000448308950F93FC01862F8F778283DA01E4
:10DEA000C9017AE0B695A795979587957A95D1F7A8
:10DEB0008F7366956074862B8383DA01C90163E0F2
:10DEC000B695A795979587956A95D1F78F778483AF
:10DED000822F82958077858340FF02C0886085838A
:10DEE000002319F08581816085830F910895E82FC3
:10DEF000F0E0E855FA4F8081811181E00895CF92DA
:10DF0000DF92EF92FF921F93CF93DF93782F162F1C
:10DF10007A01A895209193058091940530E090E0D6
:10DF200001972817390709F445C08091930583307C
:10DF300021F4809194058823E9F19091930589E07B
:10DF4000989FE0011124C159DA4F672F60686883F8
:10DF500080E00E940D6F1983612F0E940D6F982F32
:10DF6000E2E0CE2ED12CCC0EDD1EE60110E0E11455
:10DF7000F10431F0F70181917F018F77888301C02F
:10DF80001882892F69910E940D6F982F1F5F16309C
:10DF900071F787FD9095F6019683809193058F5FC9
:10DFA0008093930580919305843010F0109293052F
:10DFB00081E001C080E0DF91CF911F91FF90EF9051
:10DFC000DF90CF9008950F931F93CF93DF93082F87
:10DFD000162FEA0102C00E946F12802F612FAE013E
:10DFE0000E947F6F8823B9F3DF91CF911F910F912A
:10DFF0000895DF93CF9300D000D000D0CDB7DEB727
:10E00000FE01319696E0DF011D929A95E9F749836A
:10E01000AF010E94E36F26960FB6F894DEBF0FBEE5
:10E02000CDBFCF91DF9108952F923F924F925F9293
:10E030006F927F928F929F92AF92BF92CF92DF9218
:10E04000EF92FF920F931F93DF93CF93CDB7DEB77D
:10E05000E4970FB6F894DEBF0FBECDBF5C01DC01C4
:10E060008C9187FFF7C61FE7612E6822A5014E5FDE
:10E070005F4FF3E08F2E912C8A0C9B1C13968C9192
:10E080001397C82EDD24D694DC2CCC24D794C794C7
:10E0900012967C901297872D90E0C82AD92A8E017B
:10E0A0000E5F1F4F86E0F801282F11922A95E9F79D
:10E0B00011969C91963170F5943108F064C09930B6
:10E0C000B0F4973008F0BCC0933009F469C09430C4
:10E0D00038F4913009F4D6C1923009F0BBC666C35A
:10E0E000953009F474C3963008F090C0D4C19031D3
:10E0F00009F4E6C1913150F49D3009F49AC19E3083
:10E1000009F4C5C09B3009F0A5C642C1933108F49B
:10E1100065C277C29E3109F4D3C29F31C0F49931F0
:10E1200009F473C29A3130F49731C1F1983108F093
:10E1300005C22BC09B3109F44EC39B3108F477C252
:10E140009C3109F4B0C29D3109F084C6BFC290343D
:10E1500009F456C6913450F4903209F489C19032D2
:10E1600008F4CAC2943209F075C65EC3923409F449
:10E170001EC6923408F430C6933409F4F1C59037C2
:10E1800009F068C604C0FF24DEC180E0D9C1850162
:10E1900076E0E72EF12CEA0CFB1C4CC680E0CFC1E8
:10E1A000C114D10409F44DC6D50114961C911497DD
:10E1B00015968C91282F30E086FD1068322F22278B
:10E1C000330F330FF501668170E06F77707053E0A5
:10E1D000660F771F5A95E1F7878190E080779070FE
:10E1E00044E0959587954A95E1F7682B792B622B4A
:10E1F000732BC60144E00E94F13CC601612F44E04C
:10E200000E942A3DC6010E940F6C1BC6D5011496C0
:10E210008C911497382F3295330F330F307C20E0D8
:10E22000A601422B532B15968C91882319F0CA0115
:10E2300061E002C0CA0160E044E00E94E58E01C6D0
:10E24000F5018581E82FF0E0D50117966C916F7785
:10E2500040E0983009F441E09F0127703070369516
:10E26000322F222737952795D50114968C91149734
:10E2700090E0282B392BE074F070EE0FFF1F1696FC
:10E280000C910E2BC601EE240E945A38DAC5C60145
:10E290000E948E385C01009781F48E01025F1F4F4F
:10E2A0008BE0F80111928A95E9F7DF86CE8680E847
:10E2B0008E8BC8010E94803B5801D50112962D918A
:10E2C0003C9113972115310511F1822F8F778A83A5
:10E2D000220F232F221F330B3195822F8F778B83B1
:10E2E00012968D919C9113970E94103D9B01AC0159
:10E2F000F2E0EF2EF12CEC0EFD1EC70160E000E015
:10E300000E944A6F862D6FE0A7010E94E36F8C2D5B
:10E310008F778A83CC0CCD2CCC1CDD08D1948C2D2E
:10E320008F778B83F50181858C8372E0E72EF12C4A
:10E33000EC0EFD1E862D69E0A7010E94E36FD5015A
:10E3400014962D913D914D915C91179700E0129696
:10E350008D919C911397892B09F001E0C701F5017C
:10E3600060850E944A6F8E010E5F1F4F862D6EE002
:10E37000A8010E94E36FD50114964D915D916D91B6
:10E380007C911797C8010E94316F862D6DE094C073
:10E39000F501248130E040E050E0E781D501159699
:10E3A0008C91159790E09695982F8827979587954B
:10E3B0007C010027F7FC0095102F16966C91962F84
:10E3C0009295990F990F907C80E0AA2797FDA095D0
:10E3D000BA2FE82AF92A0A2B1B2BE22AF32A042B4C
:10E3E000152B8E2F90E0A0E0B0E087709070A070A9
:10E3F000B07055E1880F991FAA1FBB1F5A95D1F71E
:10E40000E82AF92A0A2B1B2BD801C7010197A10979
:10E41000B1098F5F9F4FAF4FB04008F012C5E6952E
:10E42000E695E695C801B701A6012E2F0E947189D5
:10E4300008C5D50114962C91149730E015966C916F
:10E44000159770E07695762F6627779567951696DF
:10E450004C91942F9295990F990F907C80E0682BA6
:10E46000792B622B732BC60144E00E94CF3CE9C498
:10E470000E946812843009F4E4C4F50182810E948C
:10E480008312DFC4C114D10409F4DBC4862DB601A4
:10E490000E940E6ED6C4C601D50114966C910E94DE
:10E4A000DA3DF50182818A8383818B83C6010E94D4
:10E4B000B6388C83862D69E0A8010E94E36FC1C441
:10E4C000B8016E5F7F4FC601AE01475E5F4F0E948D
:10E4D0002D85282F2F772A83880F892F881F990B46
:10E4E00091958F778B83898D8D838A8D8E831F8203
:10E4F000862D61E1A8010E94E36FFE017B96D801A1
:10E500009E01205E3F4F81918D93E217F307D9F76B
:10E51000862D62E1AE014E5F5F4F0E94E36FFE0108
:10E52000B0969E012C5D3F4F8191D8018D938D0156
:10E53000E217F307C9F7862D63E14CC083E08D5FD6
:10E5400023E0F22EF80E943189F4F5018581682FCD
:10E5500070E07695762F662777956795848190E0B1
:10E56000682B792B86818983198E21C08E01075EE5
:10E570001F4FC601BE016F5F7F4FA8010E942D850E
:10E58000BC01D50194E00CC0F801EF0DF11D14960B
:10E590008C91149780839F5FF3941196973019F0B4
:10E5A000FAE0FF1588F7FE01EF0DF11D118EC6018F
:10E5B00049819E01275E3F4F0E948485282F2F7737
:10E5C0002A83880F892F881F990B91958F778B83CA
:10E5D000862D60E1AE014E5F5F4F6FCF913121F428
:10E5E000C6010E94B28403C0C6010E94A3849C019C
:10E5F0008F778A83220F232F221F330B3195822F8F
:10E60000E5CFC6010E947F851CC48C2D8F778A833D
:10E61000C601880F892F881F990B91958F778B835F
:10E62000C6010E94358C8C83862D69E145CFD501CA
:10E6300015968C911597082F10E01695102F00272E
:10E640001795079516962C911697922F9295990FDC
:10E65000990F907C80E0082B192B14968C9190E0F8
:10E66000082B192B7601E4E0EE0CFF1CEA95E1F78C
:10E6700071E0C72ED12C60E1A62EB12CAE0CBF1CD0
:10E6800060E0C60180239123892B09F061E0C70176
:10E690000E942B8DCC0CDD1C0894E11CF11CEA14AB
:10E6A000FB0471F7CEC3772009F0CBC38DE08A83DA
:10E6B00082E08B8381E08C838D83862D6CE18ACF11
:10E6C000C601F501648145810E946588D5011496D3
:10E6D0006C918C2D8F778A83C601880F892F881FB4
:10E6E000990B91958F778B836C83C6010E94D58798
:10E6F0008D83862D6EE16ECF8C2D8F778A83C60138
:10E70000880F892F881F990B91958F778B83C6016E
:10E710000E9442879EA38DA3FF2425E2222E312C46
:10E720002C0E3D1E99E2492E512C4C0E5D1EC80147
:10E73000902EE92E85E3A82EB12CAC0EBD1E26C06E
:10E7400080E1B1010E948C818FA198A58C159D0557
:10E7500009F58201F8018181882399F08081F0FC1C
:10E7600004C08C8381818D830BC08E83D801119668
:10E770008C918F83862D6FE1492D5E2D0E94E36F72
:10E78000F3940E5F1F4F0A151B0521F78DA19EA163
:10E79000892BB1F6F0FC05C0FC821F821E821D820F
:10E7A00002C0FE821F82862D6FE114CFF5014581E4
:10E7B00050E05695542F442757954795848190E013
:10E7C000482B592B862DB6010E948C6D3AC3C60189
:10E7D0000E948D3C36C3D50116964C91169750E099
:10E7E00015966C91159770E06F7770707695762F0F
:10E7F000662777956795CA018170907090E4899F2C
:10E80000902D88271124682B792B14968C9190E0F9
:10E81000682B792BE6E056954795EA95E1F741702C
:10E82000C6010E94E0370DC3FE013896DF011D923C
:10E830008A95E9F70E94C06B8C01B6E07B1609F45B
:10E84000AEC0B715A8F0E2E07E1609F44BC0E7159C
:10E8500038F0772041F1F1E07F1609F0F2C22CC0C8
:10E8600024E0721609F473C0271508F47EC052C064
:10E870008BE0781609F432C1871560F098E07916BC
:10E8800009F4CEC0791608F491C0A9E07A1609F00F
:10E89000D8C2D1C0B4E1B71508F02FC1E6E17E16A9
:10E8A00009F0CFC221C218860E94CA6B8F70898777
:10E8B0000E94C76B877049C0D50113968C918F70E9
:10E8C0000E94526E0E94C76BF4019181982B892F90
:10E8D00087700E945E6ED50113968C9186FFE3CF00
:10E8E00081E015C0F50183818F700E94446E0E9403
:10E8F000C76BD40111969C9190959823892F8770AE
:10E900000E945E6EF501838186FFCDCF80E00E947C
:10E91000C97FC9CFD50113968C91882361F0F4018A
:10E9200082818795882787959181892BD8011696B2
:10E930008C930E942C6E83E08887F80186818F7704
:10E9400089878681881F8827881F8A8703C2D50107
:10E9500013968C91853310F4F801808784E08887C2
:10E96000D80118968C918987F5C1F501838164E0FF
:10E970000E94A57F9C0185E08887822F8F778987F9
:10E98000C901880F892F881F990B91958F778A87E6
:10E99000832F82958695869583708B87DBC1D50101
:10E9A00013968C9164E00E94BE7FE4CFF4018181D4
:10E9B000082F10E01695102F002717950795D50101
:10E9C00013968C9190E0082B192BBFE0003F1B079A
:10E9D00028F0EFE30F3F1E0709F033C2D40112966F
:10E9E0006C91633011F0613069F4BFE30F3F1B0796
:10E9F00029F4862F90E00E94E48C04C0C80170E0E6
:10EA00000E94948C87E08887F50183818987D401EF
:10EA100011968C918A87C8010E94638C8F77BDCF35
:10EA2000F5018381882319F00E945A8B02C00E944D
:10EA3000C78988E08EC181E0888738E0C32ED12C59
:10EA4000CC0EDD1E862D65E2A6010E94E36FD40187
:10EA500011966C9170E07695762F6627779567957D
:10EA6000F501838190E0682B792B862D0E946A7DC9
:10EA70007B018C011886862D65E2A6010E94E36F5A
:10EA800078868E2D8F77898797E016950795F7946E
:10EA9000E7949A95D1F78E2D8F778A8787E0169520
:10EAA0000795F794E7948A95D1F78E2D8F778B870A
:10EAB000B7E016950795F794E794BA95D1F78E2DA0
:10EAC0008F778C87A7E016950795F794E794AA951A
:10EAD000D1F7ED86862D64E2A601EFCC7886862DEF
:10EAE00064E2AE01485F5F4F0E94E36F82E390E013
:10EAF0000E94D7190E94B06EA4C180E00E948312C8
:10EB000081E08887862D65E2AE01485F5F4F0E94F5
:10EB1000E36FF0E17F1609F47EC0F71588F02DE071
:10EB2000721689F1271520F08CE07816C1F41AC00E
:10EB30009EE0791609F442C0AFE07A1681F453C022
:10EB4000B2E17B1609F47EC07B1608F46BC0E3E1EA
:10EB50007E1609F488C0F4E17F1609F49BC0EE2408
:10EB6000FF24A4C0D40111968C9190E09695982F23
:10EB7000882797958795F501238130E0822B932B89
:10EB80000E94BC7C92C0D40111968C91119790E0A8
:10EB90009695982F882797958795F501238130E0E2
:10EBA00013966C91139767956627679512964C910B
:10EBB000642B822B932B0E94C67C77C0D4011196C4
:10EBC0008C91119790E09695982F88279795879527
:10EBD000F501238130E012966C916770822B932BA4
:10EBE0000E94D17C62C0D40111968C91119790E063
:10EBF0009695982F882797958795F501238130E082
:10EC000012966C9112976770822B932B13964C91EE
:10EC10000E94DC7C4AC0D50113968C918F700E94B3
:10EC20009A7C43C0F5018381D40112966C911297AE
:10EC300067956627679511969C91692B8F700E9446
:10EC4000A57C33C0F401818190E09695982F8827A8
:10EC500097958795D50113962C9130E0822B932BB5
:10EC60000E94857C22C0F401818190E09695982FC6
:10EC7000882797958795D50113962C9130E063816D
:10EC80006795662767954281642B822B932B0E94A0
:10EC90008F7C0BC0F4018181879588278795D501EA
:10ECA00013969C91892B0E94B17C7C0118868E0161
:10ECB000085F1F4F862D65E2A8010E94E36F85E182
:10ECC00088878E2D8F778987C701880F892F881FA6
:10ECD000990B8F778A878F2D82958695869583707D
:10ECE0008B87862D64E2E8CBF4016381A62FB0E028
:10ECF000818190E09695982F882797958795F501C3
:10ED0000E380FF2462956370AD0106E05695479558
:10ED10000A95E1F741709D01277030703695322FCA
:10ED2000222737952795F4015281E52FF0E02E2B0D
:10ED30003F2BA870B070F4E0AA0FBB1FFA95E1F763
:10ED4000F40104810A2B8E299F29EE240E945A384F
:10ED500085E18887862D64E2AE01485F5F4FADCBC9
:10ED600000E010E0602EF801E855FA4F808188231A
:10ED7000A1F4F02E802F64E00E94E36F809198054B
:10ED8000801710F400939805FFE3FF1560F0085515
:10ED90001A4F8EE1D8018C9306C063940F5F1F4F0A
:10EDA00000341105F9F684E0809399054AC08091FA
:10EDB0009905833008F045C083E080939905F501FB
:10EDC000828180939A05838180939B0584818093BF
:10EDD0009C0510929D0535C080919905823088F57B
:10EDE00082E080939905D50112968C9112978093B9
:10EDF0009A0513968C9180939B0510929C0521C0D7
:10EE0000809199058823E9F481E080939905F501C3
:10EE1000828180939A0510929B0513C08A3019F461
:10EE20008DE00E941016D80112968C910E94101647
:10EE30000F5F1F4FF8018281882319F00E151F05FF
:10EE400069F7FFE3F61530F0E62DF0E0E855FA4FEC
:10EE50008EE18083E4960FB6F894DEBF0FBECDBF7F
:10EE6000CF91DF911F910F91FF90EF90DF90CF90A6
:10EE7000BF90AF909F908F907F906F905F904F90DA
:10EE80003F902F9008950E94147008950F931F9340
:10EE9000CF93DF93EC01162F009709F46CC086E046
:10EEA000DE011D928A95E9F70E94C06B20919605BC
:10EEB0003091970554E0220F331F5A95E1F7FC017A
:10EEC000858596858217930720F4109297051092F6
:10EED00096051F77DE011D93E0919605F091970549
:10EEE0008E2F8F7789839D012F5F3F4FCF01880F32
:10EEF000892F881F990B91958F7711968C93A90173
:10EF00004F5F5F4FEE0FFF1FDF01A959B24F8C918A
:10EF10008F77E9018983EA012196E859F24F8081D0
:10EF2000880F8E779C91991F9927991F892BDA0159
:10EF300011968C938E010F5F1F4F8081829586956D
:10EF400086958370898382E00E94CD6B882329F0A7
:10EF500089818460898381E001C080E00E94FD9105
:10EF6000E8012196809196059091970501969093DE
:10EF7000970580939605CE01DF91CF911F910F9158
:10EF80000895AF92BF92DF92EF92FF920F931F937B
:10EF9000DF93CF93CDB7DEB729970FB6F894DEBFD6
:10EFA0000FBECDBFDD24DA94F4E1EF2EF0E7FF2EA3
:10EFB0003EC087FF04C010929E05D092A00520910C
:10EFC0009E05293040F4E22FF0E0E156FA4F8083AD
:10EFD0002F5F20939E0580919E05893041F5809199
:10EFE0009F0587FF24C00FE915E090E0F8016191CB
:10EFF0008F01892F0E940D6F982FF5E0073A1F07A8
:10F00000A9F787FD90958091A705981761F468C1CD
:10F01000F092E905E092E805E091E805F091E90554
:10F020008FE995E0099510929E05D092A0050E9467
:10F030006E182FEF8F3F920709F0BBCF0E94011887
:10F040000A970CF439C19091930580919405981713
:10F0500019F19091940589E0989F700111248FE631
:10F0600095E0E80EF91E00E010E0F70181917F01C4
:10F070000E9412180F5F1F4F09301105B1F78091E0
:10F0800094058F5F8093940580919405843008F4F3
:10F0900013C11092940510C180916E05882311F060
:10F0A000DD240DC181E080936E05409195054034CB
:10F0B00029F080919905882309F473C08FEF898323
:10F0C000809199058130B1F0813030F0823021F1AA
:10F0D000833009F056C036C080E48A8380919A0557
:10F0E000982F97709B838F5F80939A05E4E0EE2EB4
:10F0F000F12C4CC081E48A8380919A0587708B83C0
:10F1000080919B05982F9F779C838F5F80939B05B1
:10F110009E012B5F3F4F2FC082E48A8380919A0526
:10F1200087708B8380919B058F778C8380919C0562
:10F13000982F9F779D838F5F80939C059E012A5F08
:10F140003F4F19C083E48A8380919A0587708B832F
:10F1500080919B058F778C8380919C058F778D8321
:10F1600080919D05982F9F779E838F5F80939D054B
:10F170009E01295F3F4F87FF02C0109299057901D8
:10F1800007C01092990572E0E72EF12CEC0EFD1EDF
:10F1900080919905882319F44F5F40939505DD24EC
:10F1A00069C04134E9F58FEF898383E08A830E9447
:10F1B0006812682FCE0103960E9446777C018091E9
:10F1C00095058F5F809395050E94123E8C01FC018E
:10F1D000848D81FF22C0F80180819181668D44E099
:10F1E0000E942A3DF80146815781608571858081A2
:10F1F000918124E00E94B83CF801828193810097BC
:10F2000029F06285738544E00E94F13CF801808119
:10F2100091810E940F6C0E94F16BDD24D3942AC06F
:10F22000403410F01092950590919505892F8068D3
:10F23000898382E08A83903448F4E92FF0E0E8552E
:10F24000FA4F8081882311F0815080839F5F9093D3
:10F250009505809198059E012D5F3F4F891718F401
:10F2600080E480939505DD24790104C0F7011192B3
:10F270007F0102C0CE010996E816F906B8F3FF2413
:10F280008E010F5F1F4F69E0A62EB12CAC0EBD1E84
:10F290008F2DF80160810E940D6FF82EF801819189
:10F2A0008F010E9412180A151B0590F3F7FCF094C9
:10F2B0008F2D0E94121801C0DD2410926E058D2D35
:10F2C00029960FB6F894DEBF0FBECDBFCF91DF9168
:10F2D0001F910F91FF90EF90DF90BF90AF90089536
:10F2E0008091E8059091E905892B09F095CE90CEA3
:10F2F0000F931F93DF93CF9300D000D000D0CDB7F2
:10F30000DEB7682F8E010F5F1F4FC8010E9446773E
:10F310008FEF63E0A8010E94E36F26960FB6F89482
:10F32000DEBF0FBECDBFCF91DF911F910F9108952A
:10F33000EF92FF920F931F93CF93DF93182F80E0EC
:10F340000E94831282E390E00E94D71984E00E9419
:10F350008312112319F00E94443202C00E948032AD
:10F3600084EF91E00E94D7190E945D260E946423D9
:10F3700084E690E00E94D7191123D9F00E947F23E0
:10F380008C0180E090E060E040E00E94E73380E0A4
:10F3900090E060E041E00E94E73383E090E00E946B
:10F3A000D07A84E690E00E94D7190E947F23EC0176
:10F3B0005FC04AE0E42EF12C0E9464230E945D2687
:10F3C00060E070E080E090E040E20E94D03204C053
:10F3D00084E190E00E94D7190E949E308823C1F3F7
:10F3E0000E947F238C010E94642360E070E080E033
:10F3F00090E841E00E94D03260E070E080E090E070
:10F4000041E00E94D03204C084E190E00E94D7190C
:10F410000E949E308823C1F384E690E00E94D719B1
:10F420000E947F23EC010531110534F0C801880FDB
:10F43000991FC817D907C4F48E2D8A50823060F006
:10F44000C7010E94603204C084E190E00E94D71995
:10F450000E949E308823C1F30894E11CF11C20E136
:10F46000E216F10409F0A8CF80E090E00E9460323B
:10F470000E945D26C8014497855A9B40B0F081E008
:10F4800060E00E942A1F0431110514F48DE101C0CF
:10F490008EE10E94916BBC0182E00E94FE2080E020
:10F4A0000E94831288EE93E002C086E990E00E94F9
:10F4B000D719C801880F991F8C179D0754F481E054
:10F4C000C53FD80734F098012C0F3D1F359527957F
:10F4D0000AC024E0C13BD2071CF428EE33E003C08D
:10F4E0009E01285C3040C901DF91CF911F910F919F
:10F4F000FF90EF900895DF93CF9300D000D000D01D
:10F50000CDB7DEB716B886B187B90E94C06BDC01F3
:10F5100014968C910E94A11EFE01319686E0DF01B7
:10F520001D928A95E9F781E089838FEF62E2AF014E
:10F530000E94E36FE2E6F0E080818D7F8083269673
:10F540000FB6F894DEBF0FBECDBFCF91DF91089507
:10F55000DF93CF9300D000D000D0CDB7DEB7E2E686
:10F56000F0E080818260808380E00E94A11EFE0125
:10F57000319686E0DF011D928A95E9F78FEF62E20E
:10F58000AF010E94E36F83EC87B98FEE86B92696B0
:10F590000FB6F894DEBF0FBECDBFCF91DF910895B7
:10F5A0000F931F93CF93DF93EC0101C0A8950E94A6
:10F5B0009E308823D9F311C0A89504C081E090E063
:10F5C0000E94D7190E949E308823C1F380E090E00A
:10F5D00060E041E00E944E3421970E94602388231E
:10F5E00011F4209749F70E946023082F15E00FC0FF
:10F5F00080E090E060E043E00E944E340E9464238B
:10F6000001C0A8950E949E308823D9F311500E9412
:10F610006023882319F0112359F707C0112329F01B
:10F62000802F002319F081E001C080E0DF91CF91AD
:10F630001F910F910895EF92FF920F931F93CF9315
:10F64000DF937C01C0E0D0E0C7016C2F0E94A7339C
:10F6500080E090E00E94D07A882319F40FEF1FEF2A
:10F6600002C00C2F10E0CF3FD10551F4E80183E038
:10F6700090E00E94D07A882349F00FEF10E00AC092
:10F6800021968FEF0F3F1807F9F204C08FEF0F3F5D
:10F690001807C1F0102FC701612F0E94A73383E024
:10F6A00090E00E94D07A882319F4CFEFDFEF02C0F8
:10F6B000C12FD0E0112331F08FEFCF3FD80711F4E5
:10F6C0001150E9CFCE01DF91CF911F910F91FF90A3
:10F6D000EF9008952F923F924F925F926F927F9298
:10F6E0008F929F92AF92BF92CF92DF92EF92FF9252
:10F6F0000F931F93CF93DF93D82E7B01C42EA22E9E
:10F70000302E0E94A87AC701969587959695879581
:10F71000482E4394CFEFDFEFBB2437E0632E712CEC
:10F720006E207F2023E0822E912C8E209F205A2C49
:10F73000222481E00E9498790E946E230E94642313
:10F740000E946812843009F0C7C083E0D81609F41B
:10F7500046C08D1530F081E0D81631F18D15F8F0E6
:10F760000EC085E0D81640F086E08D1508F057C031
:10F7700088E08D1508F072C0CFEFDFEF9FC0C701A2
:10F780006C2D4A2D0E940E348FE090E00E94D07ABA
:10F79000882309F493C0852D922DEC0189C0C701FF
:10F7A0006C2D0E9487334BC0C7016C2D40E00E9436
:10F7B000E73383E090E00E94D07A882309F0A2C06A
:10F7C000C7016C2D41E00E94E73383E090E00E9486
:10F7D000D07A882309F472C0C1E0D0E069C010E09B
:10F7E00000E00695C701612F40E00E94E73383E007
:10F7F00090E00E94D07A882309F400681F5F1830D7
:10F8000081F7C701602F0E94673383E090E00E9478
:10F81000D07A882309F452C0C02FD0E049C085E0D7
:10F8200090E061E00E94C7338FE090E00E94D07AC0
:10F8300085E0D81661F4C3016C2D0E94C7338FE0B8
:10F8400090E00E94D07A882309F05CC037C0C301E1
:10F850000E941B7BEC0193E0B92E28C085E090E06C
:10F86000642D0E94C7338FE090E00E94D07A87E039
:10F87000D81669F4C4016C2D0E94C7338FE090E064
:10F880000E94D07A882349F0C0E0D0E006C0C401CD
:10F890000E941B7BEC0183E0B82E85E090E061E0E4
:10F8A0000E94C7338FE090E00E94D07AD7FD06C057
:10F8B000332021F08CE291E00E94D71980E00E9471
:10F8C0008312D7FF09C08CE291E00E94D719B3944C
:10F8D00082E08B1508F02DCF0E947B7ACE01DF915C
:10F8E000CF911F910F91FF90EF90DF90CF90BF903D
:10F8F000AF909F908F907F906F905F904F903F90D0
:10F900002F900895C0E0D0E0D3CF0F93BC0188E0E2
:10F9100040E020E000E00E946A7B0F9108950F9381
:10F920009C01462F87E0B90120E001E00E946A7B3C
:10F930000F9108950F93682F86E070E040E020E07B
:10F9400000E00E946A7B0F9108950F93982F462F35
:10F9500085E0692F70E020E001E00E946A7B0F9152
:10F9600008950F93482F85E060E070E020E001E00B
:10F970000E946A7B0F9108950F93BC0183E040E0E1
:10F9800020E000E00E946A7B0F9108950F939C0194
:10F99000462F82E0B90120E001E00E946A7B0F91CE
:10F9A00008950F939C01462F81E0B90120E000E00B
:10F9B0000E946A7B0F9108950F93FC01962F242FCC
:10F9C00080E0BF01492F01E00E946A7B0F910895FA
:10F9D000DF92EF92FF920F931F932091C507309112
:10F9E000C6074091C7075091C8077C0100E010E0AE
:10F9F000E20EF31E041F151F10C081E090E00E946C
:10FA0000D7190E946423C801B7010E9411198823E5
:10FA100091F40E946023882311F0DD2401C0D39467
:10FA20000E949E30882349F30E946023882329F78F
:10FA300089E08D1510F70E949E30882319F480E02C
:10FA400090E008C00E94602390E0811191E081E085
:10FA50009827892F1F910F91FF90EF90DF900895C5
:10FA6000EF92FF920F931F932091C5073091C60725
:10FA70004091C7075091C8077C0100E010E0E20EFA
:10FA8000F31E041F151F01C0A8950E949E308823F5
:10FA9000D9F301C0A8950E946023882331F4C801DE
:10FAA000B7010E9411198823A9F30E949E30882370
:10FAB00019F480E090E009C00E94602390E0882360
:10FAC00009F491E081E09827892F1F910F91FF9011
:10FAD000EF9008952F923F924F925F926F927F9294
:10FAE0008F929F92AF92BF92CF92DF92EF92FF924E
:10FAF0000F931F93DF93CF93CDB7DEB767970FB602
:10FB0000F894DEBF0FBECDBF8B8B7D8B6C8B0E94BC
:10FB1000A87A80E00E9498798E8B9F8B8C899D8932
:10FB20000E94893C9A8B898B009771F0DC011996B1
:10FB30001C92E989FA8914821582168217828C89AF
:10FB40009D8960E00E94623D0E946812843021F02D
:10FB5000CC24DD247601D9C118861F8288EE93E07B
:10FB60000E94E87C01E0CC24DD247601812C912CDC
:10FB7000A12C60E8B62E09870E94601D0A9709F43F
:10FB8000B5C1FB89FF3F51F581E060E00E942A1F6B
:10FB90002DB73EB7295030400FB6F8943EBF0FBE88
:10FBA0002DBFEDB7FEB7319622E0ADB7BEB71196C7
:10FBB0002C9342ED58E15283418303831482C58222
:10FBC000D682E782F0860E94A4208DB79EB7099660
:10FBD0000FB6F8949EBF0FBE8DBF37C09AE09983D1
:10FBE0008C2D8F778A83D701C60157E0B695A795EC
:10FBF000979587955A95D1F78F778B83D701C60153
:10FC00004EE0B695A795979587954A95D1F78F774A
:10FC10008C83D701C60135E1B695A7959795879551
:10FC20003A95D1F78F778D83D701C6012CE1B69530
:10FC3000A795979587952A95D1F78E838B8964E24E
:10FC4000AE014F5F5F4F0E94E36F023028F420E067
:10FC500030E040E050E80EC0802F90E0019720E0B7
:10FC600030E040E050E804C0569547953795279519
:10FC70008A95D2F72D873E874F87588B8E899F892B
:10FC80009C0119012601370135E03C87C1010E9422
:10FC90006E2384E690E00E94E87CC301B201402F0D
:10FCA0000E94D0328AE090E00E94307D811181E094
:10FCB000182F0E947F239B878A878D859E85AF851D
:10FCC000B889482659266A267B2684E690E00E9459
:10FCD000E87CC301B201402F0E94D0328AE090E05C
:10FCE0000E94307D811112600E947F23AA85BB850E
:10FCF0008A1B9B0B97FF03C0909581959F4F80595E
:10FD0000914014F484E005C0112311F01330CCF0BD
:10FD1000812FEC85E150EC87EE2391F0882329F4C4
:10FD200028E33FEF220E331E06C0833021F448EC57
:10FD300050E0240E351E84E690E00E94D719A6CF2D
:10FD4000182F812F815031F0813051F4C828D928E3
:10FD5000EA28FB28B694A794979487940F5F15C060
:10FD6000023028F0880C991CAA1CBB1C0150D5013C
:10FD7000C40180959095A095B095C822D922EA2219
:10FD8000FB2284E690E00E94D71959855F5F59876E
:10FD9000503621F0013208F4EFCE03C0013208F4EE
:10FDA00099C0C114D104E104F10409F493C08FEFA8
:10FDB000C8168FEFD8068FEFE8068FEFF80609F424
:10FDC00095C09B899F3F41F581E060E00E942A1F1A
:10FDD000ADB7BEB719970FB6F894BEBF0FBEADBF93
:10FDE000EDB7FEB7319622E011962C9346EC58E120
:10FDF000528341838F81988594838383C582D68281
:10FE0000E782F0860E94A420ADB7BEB719960FB660
:10FE1000F894BEBF0FBEADBFE989FA89EF2B09F494
:10FE200068C02C893D892115310509F462C0C701DC
:10FE3000B601A9010E94B23288EE93E00E94D71960
:10FE4000BB2489899A8941E050E060E070E000E0DD
:10FE500010E020E030E00E9485340E949E3088232C
:10FE6000E1F384E690E00E947419B39435E0B31690
:10FE700041F784E690E00E94E87CC701B6014C8916
:10FE80005D890E9494328AE090E00E94307D882350
:10FE900081F54B894F3FF1F481E060E00E942A1F19
:10FEA00000D000D00F92EDB7FEB7319622E0ADB78B
:10FEB000BEB711962C9344EB58E1528341838F8156
:10FEC0009885948383830E94A4200F900F900F90B5
:10FED0000F900F9088EE93E00E94D719AF81B885FC
:10FEE0001196B887AF83159709F038CECC24DD245E
:10FEF000760180E00E948312C114D104E104F10470
:10FF000021F488EE93E00E94D7190E947B7A80E06A
:10FF10000E948312B601C70167960FB6F894DEBF40
:10FF20000FBECDBFCF91DF911F910F91FF90EF904A
:10FF3000DF90CF90BF90AF909F908F907F906F9009
:10FF40005F904F903F902F900895662319F022E222
:10FF50003CE002C02AE83CE0F894E82FF0E0EE0F25
:10FF6000FF1FE20FF31F208191818091F20C80FF2F
:10FF700002C0118210827894822F0895E82FF8949D
:10FF80007894F0E0EE0FFF1FE150F34F80819181F4
:10FF900008959091F20C882311F0916001C09E7F2A
:10FFA0009093F20C0895BF92CF92DF92EF92FF925E
:10FFB0000F931F93CF93DF93882339F039EFC32E2C
:10FFC0003CE0D32EC2E2DCE006C023EFC22E2CE0E0
:10FFD000D22ECAE8DCE00E94C06BFC01B0840FEFB7
:10FFE0001CE07E01C0E0D0E018C0F894F8018081E8
:10FFF0009181F70191838083F80180819181892B20
:020000021000EC
:1000000021F0C601BE010E946B91789421960E5F8B
:100010001F4F82E090E0E80EF91ECB1530F3DF9120
:10002000CF911F910F91FF90EF90DF90CF90BF90F5
:10003000089584E0809374001092710083E08093AF
:10004000700008951F920F920FB60F920BB60F9289
:1000500011248F939F93EF93FF938091710090E011
:10006000887F90708032910509F485C081329105B6
:100070005CF480319105D1F08831910509F442C0DA
:10008000089709F07AC016C080349105A9F181342F
:10009000910524F4889709F070C03EC08035910521
:1000A000D9F08835910509F068C00AC08091EA0549
:1000B00087FF02C080EA01C081EA8093730059C0C3
:1000C000E091F005F091F105809173008193F09338
:1000D000F105E093F00546C0E091F005F091F105DF
:1000E000809173008193F093F105E093F005809186
:1000F000EB0581508093EB058091EB058230CCF1CC
:1001000085EC3FC08091EE059091EF0590937300D0
:100110008FEF8093EA052DC08091EA0587FF09C023
:100120008091EE059091EF05809373001092EA059F
:1001300020C08091EC058823F1F08091EB058823A5
:1001400089F0E091F005F091F105819180937300C1
:10015000F093F105E093F0058091EB0581508093D9
:10016000EB0507C084E98093740081E08093ED057E
:100170000AC085E806C085EA04C08FEF8093ED05CC
:1001800084E980937400FF91EF919F918F910F907C
:100190000BBE0F900FBE0F901F90189580917400AA
:1001A00020E090E087709070892B09F021E0822F89
:1001B00008956093EB059093EF058093EE052093EF
:1001C000EC055093F1054093F0058EEF8093EA051E
:1001D0001092ED0585EA8093740008952091ED0555
:1001E000332727FD3095C90108956093EB0590935F
:1001F000EF058093EE052093EC055093F1054093B5
:10020000F0058EEF8093EA051092ED0585EA809364
:10021000740001C0A8958091ED058823D9F3209141
:10022000ED05332727FD3095C90108958130B1F0E0
:10023000813070F0823019F0833021F406C0E6EF8F
:10024000F5E008C020E030E007C0E8EFF5E002C0CC
:10025000E2EFF5E020813181C9010895E4EFF5E096
:10026000F9CF8130D1F0813058F0823019F08330ED
:10027000B9F403C0E6EFF5E005C0E8EFF5E002C031
:10028000E2EFF5E0808191818617970749F071834D
:10029000608381E08093FA050895E4EFF5E0F2CF02
:1002A000089524E0880F991F2A95E1F721E00E9424
:1002B000F580089534E0880F991F3A95E1F720E022
:1002C0000E94F5800895DF93CF9300D0CDB7DEB7BD
:1002D00094E06030790718F020E030E017C0611535
:1002E000710571F0CB0144E0880F991F4A95E1F741
:1002F00062E0AE014F5F5F4F20E00E94F58004C0D6
:100300000E9416819A83898329813A81C9010F90BD
:100310000F90CF91DF9108950F931F93282FFB012A
:1003200000811181C80154E0880F991F5A95E1F7A7
:10033000622FAF0120E00E94F580C8011F910F914C
:100340000895CF92DF92EF92FF920F931F93DF9366
:10035000CF9300D0CDB7DEB77B0194E06030790752
:1003600010F50E9416819A83898320E030E06E01A7
:100370000894C11CD11C0CC0C80164E0880F991FEF
:100380006A95E1F762E0A60120E00E94F5809801FD
:1003900009811A810115110521F00E151F0561F75C
:1003A00004C0EF2811F02FEF3FEFC9010F900F901D
:1003B000CF91DF911F910F91FF90EF90DF90CF9041
:1003C0000895CF93DF93EC0180E0BE010E94A181EC
:1003D0009C0184E020303807B8F082E0BE010E9422
:1003E000A1819C0184E02030380770F083E0BE01D9
:1003F0000E94A1819C0184E02030380728F081E030
:10040000BE010E94A1819C01C901DF91CF91089595
:100410008091FA05882351F080E090E068E042EF97
:1004200055E021E00E94F5801092FA0508950F939F
:100430001F93DF93CF9300D0CDB7DEB70091F405C3
:100440001091F50501151105A1F0C80174E0880FA0
:10045000991F7A95E1F762E0AE014F5F5F4F20E0B0
:100460000E94F58069817A8181E00E9431810E9439
:100470000882C8010F900F90CF91DF911F910F91CB
:100480000895DF92EF92FF920F931F93DF93CF9324
:1004900000D0CDB7DEB7D82E8B01CB0101978F5F8F
:1004A000934058F5CB01F4E0880F991FFA95E1F7D6
:1004B00062E07E010894E11CF11CA70120E00E948B
:1004C000F5808D2DB8010E94A181009731F46981DA
:1004D0007A818D2D0E9431810EC024E080309207F8
:1004E00050F4E4E0880F991FEA95E1F762E0A70174
:1004F00021E00E94F5800E9408820F900F90CF911A
:10050000DF911F910F91FF90EF90DF9008955F9220
:100510006F927F928F929F92AF92BF92CF92DF9213
:10052000EF92FF920F931F93DF93CF93CDB7DEB778
:1005300062970FB6F894DEBF0FBECDBF982E7A8BB0
:10054000698B542E852E390184E06030780708F0DD
:1005500067C06115710521F0892D0E94418207C095
:100560000E941782009709F45BC09A8B898B892DB2
:100570000E9416819A838983E52CF82CCC24DD24F3
:100580005E010894A11CB11C17C0C80124E0880FAB
:10059000991F2A95E1F760E1A50120E00E94F5800E
:1005A000852D982DB501F30109951816190614F437
:1005B000C80107C06801C80109811A810115110528
:1005C00021F7C816D90611F480E090E0F701918375
:1005D000808389899A89B4E0880F991FBA95E1F7D9
:1005E00062E0A70121E00E94F580C114D10431F43A
:1005F00069897A89892D0E9431810DC0C601A4E0E4
:10060000880F991FAA95E1F762E0AE014F5E5F4F38
:1006100021E00E94F5800E94088229893A8902C05F
:1006200020E030E0C90162960FB6F894DEBF0FBE3D
:10063000CDBFCF91DF911F910F91FF90EF90DF9091
:10064000CF90BF90AF909F908F907F906F905F9072
:100650000895EF92FF920F931F93DF93CF93CDB73F
:10066000DEB762970FB6F894DEBF0FBECDBF482F3E
:100670007A8B698BCB0101978F5F934008F04BC059
:10068000842F0E9441828091F4059091F5059A8310
:1006900089837E010894E11CF11C0CC0C80154E060
:1006A000880F991F5A95E1F762E0A70120E00E94A8
:1006B000F580C80109811A810115110579F70097A4
:1006C00031F469897A8981E00E9431810CC044E06B
:1006D000880F991F4A95E1F762E0AE014F5E5F4FC8
:1006E00021E00E94F580CE0103966FEF70E04EE0AE
:1006F00050E00E943AA989899A8934E0880F991FAD
:100700003A95E1F760E1AE014F5F5F4F21E00E9453
:10071000F5800E94088262960FB6F894DEBF0FBE85
:10072000CDBFCF91DF911F910F91FF90EF90089572
:100730000E9429830895CF92DF92EF92FF920F9348
:100740001F93DF93CF93CDB7DEB760970FB6F894C2
:10075000DEBF0FBECDBF88E0E2EFF5E0DF011D9206
:100760008A95E9F781E090E09093F5058093F40590
:1007700081E08093FA05A8950E940882CE01039635
:100780006FEF70E04EE050E00E943AA901E010E007
:1007900060E1E62EF12C6E010894C11CD11CB3E07F
:1007A0000F3F1B0739F00F5F1F4F1A83098301505A
:1007B000104002C01A8219820E946F12C70160E1C4
:1007C000A60121E00E94F5800F5F1F4F80E190E0BD
:1007D000E80EF91E94E00030190709F760960FB68D
:1007E000F894DEBF0FBECDBFCF91DF911F910F9167
:1007F000FF90EF90DF90CF900895CF92DF92EF922D
:10080000FF920F931F93DF93CF93CDB7DEB760971F
:100810000FB6F894DEBF0FBECDBF80E090E068E079
:1008200042EF55E020E00E94F5801092FA0589E041
:100830000E94221D882329F08EE00E94221D882319
:1008400071F48091F4059091F5058F5F9F4F31F51C
:100850008091F2059091F3058F5F9F4FF9F484E04A
:100860006EEB71E00E940B2085E066EC71E00E9467
:100870000B2085E99DE968EC70E00E94691E80E02C
:1008800060E00E942A1F83E00E94916BBC0182E01D
:100890000E94FE200E949B830E94076C0091F2053B
:1008A0001091F3056E010894C11CD11C1EC0C80133
:1008B00074E0880F991F7A95E1F760E1A60120E0C6
:1008C0000E94F580F980EA808B819C8101978F5F7F
:1008D0009F4320F080E0B8010E942983A8950E94E0
:1008E0004A1D8F2D9E2D9C018901C80101978F5FA4
:1008F0009340E8F28091F6059091F705805094407E
:1009000028F082E060E070E00E9431818091F8057B
:100910009091F9058050944028F083E060E070E009
:100920000E9431810E94088260960FB6F894DEBF63
:100930000FBECDBFCF91DF911F910F91FF90EF9030
:10094000DF90CF900895BC0180E00E94A1819C01BE
:10095000009731F480E060E070E00E94A1819C018A
:10096000C9010895BC0180E00E9463819C01009749
:1009700031F480E060E070E00E9463819C01C90175
:100980000895EF92FF920F931F93DF93CF93CDB70C
:10099000DEB760970FB6F894DEBF0FBECDBF8C01F7
:1009A000009719F420E030E016C080E00E94168124
:1009B0009A8389837E010894E11CF11C05C08B8118
:1009C0009C818017910739F084E0B7010E948C81E7
:1009D0009C010097A1F7C90160960FB6F894DEBF9D
:1009E0000FBECDBFCF91DF911F910F91FF90EF9080
:1009F0000895DF92EF92FF920F931F93DF93CF93AF
:100A0000CDB7DEB760970FB6F894DEBF0FBECDBF8F
:100A1000D62E0E94C1848C01009789F060E17E018E
:100A20000894E11CF11CA7010E945A818D818D154B
:100A300031F0DD82C80160E1A7010E94518160961A
:100A40000FB6F894DEBF0FBECDBFCF91DF911F91DF
:100A50000F91FF90EF90DF900895EF92FF920F9328
:100A60001F93DF93CF93CDB7DEB760970FB6F8949F
:100A7000DEBF0FBECDBF8B017A0124E0803092072C
:100A800070F5009781F480E00E941681009759F478
:100A90000115110511F0F8011082E114F104F9F0CB
:100AA000F70110821CC060E1AE014F5F5F4F0E94F2
:100AB0005A810115110519F08D81F8018083E11427
:100AC000F10451F0D701FE0136968BE001900D92B2
:100AD0008150E1F7F70113862B813C8102C020E0B1
:100AE00030E0C90160960FB6F894DEBF0FBECDBFEF
:100AF000CF91DF911F910F91FF90EF900895BC016E
:100B000080E00E9498830895EF92FF920F931F93C5
:100B1000DF93CF93CDB7DEB760970FB6F894DEBF03
:100B20000FBECDBF7C01D9012115310569F16115D9
:100B3000710551F180E0E81684E0F80628F57C8321
:100B40006B834D83FE0136969E012F5E3F4F02C0A0
:100B5000819311968C91882321F0E217F307C1F756
:100B600004C0E217F30708F4108280E0B7018E0199
:100B70000F5F1F4FA8012CED35E80E9487827C0192
:100B800060E1A8010E945181C70160960FB6F894F8
:100B9000DEBF0FBECDBFCF91DF911F910F91FF90B0
:100BA000EF900895FC01A62F9A0180E090E0BF012C
:100BB0004A2F0E94848508959B01BC01009769F02B
:100BC000C9012115310549F06B5F7F4F05964BE058
:100BD00050E00E9453A99C0102C020E030E0C9010E
:100BE00008950F931F93CF93DF938C01EB0182E065
:100BF0000E941681998388830AC0828193819F779E
:100C00008017910771F04F5F32964730B1F780E15E
:100C1000BE010E948C819C01009719F0FE0140E00A
:100C2000ECCFC901DF91CF911F910F910895DF9310
:100C3000CF93CDB7DEB760970FB6F894DEBF0FBE87
:100C4000CDBFBE016F5F7F4F0E94F185BC01009751
:100C500019F082E00E94988360960FB6F894DEBF88
:100C60000FBECDBFCF91DF9108956F927F928F928B
:100C70009F92AF92BF92CF92DF92EF92FF920F932B
:100C80001F93DF93CF93CDB7DEB760970FB6F8947D
:100C9000DEBF0FBECDBF4C018091FB05882309F05C
:100CA0007CC0C4010E948E388C01009709F475C085
:100CB000DC0112968D919C911397892B09F46DC0DC
:100CC0001896BC90C401BE016F5F7F4F0E94F185F2
:100CD0007C010097A1F40E9417827C01009709F41F
:100CE0005EC082E00E9416819A838983805094407E
:100CF00010F01A82198282E0B7010E9431818EE0E1
:100D0000FE013396DF011D928A95E9F79C828B8262
:100D100025E0C22ED12CCC0EDD1E91E1692E712C66
:100D20006C0E7D1EAB2CBB24A7FCB094AA24BB0C7C
:100D3000AA1CBB241DC00E948E388C01009719F19B
:100D4000FC0120813181D6012D933C9340E050E09D
:100D5000808587FF02C041E050E04A155B0521F025
:100D60003068F6013183208382E090E0C80ED91EFE
:100D7000D80112968D919C9113978815990519F0B9
:100D8000C614D704C1F6C70160E1AE014F5F5F4FE3
:100D90000E9451810E94088202C0EE24FF24C701F4
:100DA00060960FB6F894DEBF0FBECDBFCF91DF9136
:100DB0001F910F91FF90EF90DF90CF90BF90AF9079
:100DC0009F908F907F906F900895CF92DF92EF92D7
:100DD000FF920F931F93DF93CF93CDB7DEB760974A
:100DE0000FB6F894DEBF0FBECDBF9C018091FB050E
:100DF0008823C1F5C901BE016F5F7F4F0E94F18555
:100E0000892B81F181E08093FB05EB80FC80C70199
:100E10000E94893C892B11F18E010B5F1F4F3FE02F
:100E2000C32ED12CCC0EDD1EF801208131813F77FD
:100E3000C90101978E5F9F4358F4C9010E94893C04
:100E4000892B61F0F80160817181C7010E94503CDB
:100E50000C151D0519F00E5F1F4FE6CF1092FB0514
:100E600081E001C080E060960FB6F894DEBF0FBE4F
:100E7000CDBFCF91DF911F910F91FF90EF90DF9049
:100E8000CF900895CF92DF92EF92FF920F931F932E
:100E9000DF93CF93CDB7DEB760970FB6F894DEBF80
:100EA0000FBECDBF7C0183E00E9416818C016E01D4
:100EB0000894C11CD11C0CC0C80164E0A6010E94AA
:100EC0005A818B819C818E159F0528F409811A8196
:100ED0000115110589F7C80160960FB6F894DEBFB9
:100EE0000FBECDBFCF91DF911F910F91FF90EF907B
:100EF000DF90CF9008959F92AF92BF92CF92DF92F2
:100F0000EF92FF920F931F93DF93CF93CDB7DEB78E
:100F100060970FB6F894DEBF0FBECDBF6C01962E62
:100F20005A0189012115310519F48E010F5F1F4FF8
:100F3000C6010E9442877C0120C0C70160E1A80170
:100F40000E945A81F801828193818C159D05C1F41C
:100F500020E030E08481891539F4A114B10491F0C6
:100F6000F501F182E0820EC02F5F3F4F32962630AE
:100F7000310581F7F801E080F180E114F104E9F630
:100F80002FEF3FEFC90160960FB6F894DEBF0FBE9A
:100F9000CDBFCF91DF911F910F91FF90EF90DF9028
:100FA000CF90BF90AF909F9008950F931F93DF93C2
:100FB000CF93CDB7DEB762970FB6F894DEBF0FBE02
:100FC000CDBF9C0101978F5F9F43B8F48FEF9FEFD8
:100FD0009A838983C9018E010F5F1F4FA8019E016B
:100FE0002D5F3F4F0E947B8797FD07C0880F991F99
:100FF000080F191FF801878101C080E062960FB6C3
:10100000F894DEBF0FBECDBFCF91DF911F910F913E
:101010000895EF92FF920F931F93DF93CF93CDB775
:10102000DEB762970FB6F894DEBF0FBECDBF9C014E
:1010300001978F5F9F43E0F58FEF9FEF9A8389833E
:1010400053E0E52EF12CEC0EFD1EC9018E010F5F61
:101050001F4FA80197010E947B878630910540F5BC
:10106000FC013296EE0FFF1FE00FF11F1282880F76
:10107000991F080F191FF8011782FE013896A0E08A
:10108000B0E0A701BE016C5E7F4F80818111119697
:101090003296E617F707C9F769817A81AB2B21F4FD
:1010A00083E00E94988304C0CB0160E10E945181DB
:1010B00062960FB6F894DEBF0FBECDBFCF91DF9121
:1010C0001F910F91FF90EF9008958F929F92AF9292
:1010D000BF92CF92DF92EF92FF920F931F93DF9315
:1010E000CF93CDB7DEB762970FB6F894DEBF0FBED1
:1010F000CDBF8C01A62EB42E01978F5F9F4308F0C1
:101100009DC08FEF9FEF9A838983442321F4C80108
:101110000E94098893C0B3E0CB2ED12CCC0EDD1EEB
:10112000C8017E010894E11CF11CA70196010E94F0
:101130007B878630910578F4FC01EE0FFF1FEE0DE2
:10114000FF1D87818B1509F479C0B78289819A8147
:1011500060E1A60171C0C8010E9442877C019A83A8
:1011600089834601E8E0CE2ED12CCC0EDD1E29C0AD
:1011700060E1A4010E945A818D819E8180179107B0
:1011800021F5F60120E030E08081882381F4F90127
:101190003296EE0FFF1FDE011196EA0FFB1FA282AF
:1011A000220F331FA20FB31F1796BC923FC02F5FB1
:1011B0003F4F32962630310539F78B819C819A83D7
:1011C000898389819A81009799F60E9417820097F6
:1011D000A9F19A83898380E1FE013396DF011D9294
:1011E0008A95E9F7FC82EB821E830D83AF82B88675
:1011F00083E0B7010E94A181BFEF8F3F9B0731F4CD
:1012000069817A8183E00E94988318C0009741F435
:1012100069817A8183E00E9431810E94088206C040
:1012200062E0AE014F5F5F4F0E94518189819A81D8
:1012300060E1AE014D5F5F4F0E94518162960FB633
:10124000F894DEBF0FBECDBFCF91DF911F910F91FC
:10125000FF90EF90DF90CF90BF90AF909F908F90D6
:101260000895CF92DF92EF92FF920F931F93DF9337
:10127000CF93CDB7DEB760970FB6F894DEBF0FBE41
:10128000CDBF7C0101978F5F9F43E0F4C7010E94AF
:1012900042878C016E010894C11CD11C10C0C8018A
:1012A00064E0A6010E945A818B819C818E159F0566
:1012B00049F483E0B8010E94988309811A810115DD
:1012C000110569F760960FB6F894DEBF0FBECDBF6B
:1012D000CF91DF911F910F91FF90EF90DF90CF9012
:1012E0000895EF92FF920F931F93DF93CF93CDB7A3
:1012F000DEB728970FB6F894DEBF0FBECDBF7B01D7
:101300008C018091FC059091FD05892B99F1E98272
:10131000FA820B831C8318861F82122F20FF0AC0BB
:1013200058874F83CA0160E070E040E050E00E94BF
:101330002D85AC0111FF05C08F8198859068988735
:101340008F8341155105B1F08091FC059091FD0509
:101350005E834D8368E0AE014F5F5F4F21E00E94E6
:10136000F5808091FC059091FD0508969093FD0510
:101370008093FC0528960FB6F894DEBF0FBECDBF54
:10138000CF91DF911F910F91FF90EF9008955F92A1
:101390006F927F928F929F92AF92BF92CF92DF9285
:1013A000EF92FF920F931F93DF93CF93CDB7DEB7EA
:1013B0006C970FB6F894DEBF0FBECDBF0E946812C7
:1013C000582E80E00E94831280E090E060E040E0D0
:1013D00050E00E948F44FE01319686E0DF011D92AD
:1013E0008A95E9F710E0FE2E0F2F812F67E04F2D31
:1013F000502F0E94E36F84E190E00E94D7191F5F95
:10140000103499F70E94CC3A1E861D86A12C10E458
:10141000B12EBDE0EB2EF12CEC0EFD1E30C0C5014F
:1014200068E0A70120E00E94F5808D859E85BFEFD2
:101430008F3F9B0701F10E94893C8C010097D9F0F6
:101440006B896F70FC01808191810E94DA3D8F85EC
:101450009889D80113969C938E93129789899A89BB
:10146000A0E0B0E0F80184839583A683B7838B89DD
:101470009C8990FD108688E090E0A80EB91E8D85AD
:101480009E858F5F9F4F59F61D8A1E8A1F8A188E70
:10149000A5E16A2E712C6C0E7D1EF7E08F2E912C2B
:1014A0008C0E9D1EC7C0C50168E0A30120E00E940C
:1014B000F5808D899E89AF89B88D80509040A0407D
:1014C000B14008F0B3C0E98CFA8CE114F10409F4DE
:1014D000ADC0F0E0EF16F0E4FF0608F0A7C08B8D7A
:1014E0009C8DD92EDD1CDD24DD1CDD0C009711F454
:1014F000870111C08C011F77C80160E070E040E0F7
:1015000050E00E942D85E816F90619F421E0D22A50
:1015100002C0098D1A8D2D893E894F89588DCD2C99
:10152000DD24211531054105510509F044C00E9413
:10153000123E7C01C0FE09C0AC014C5D5F4FC8018A
:1015400060E070E00E942D858C01C8010E948E38F9
:101550008C01009711F1DC0114964D915C91159767
:101560008D919C91119718966C910E948F44F8016F
:10157000818560E070E00E946E44D80112968D91E2
:101580009C9113970E948E38FC01009731F0648182
:101590007581808191810E94B13EC1FE04C0F70136
:1015A000848D8160848FD7015C968C915C9782607A
:1015B0005C968C933BC0802F8F778F83000F012F19
:1015C000001F110B1195802F8F778887822F8F77BF
:1015D000898777E056954795379527957A95D1F77E
:1015E000822F8F778A8767E056954795379527959D
:1015F0006A95D1F7822F8F778B8793E0CC0CDD1C17
:101600009A95E1F787E056954795379527958A95FE
:10161000D1F7822F87708C298C878FEF6CE0A40123
:101620000E94E36F0E94C1778823E1F3E8E0F0E0D5
:10163000AE0EBF1E8D899E89AF89B88D80509040B7
:10164000A040B14008F42FCF07E61DE0C50168E0D7
:10165000A80120E00E94F58088E090E0A80EB91E65
:10166000085F1F4F9EE00736190781F783E00E944D
:10167000831284E690E00E94D7198F8598890E9492
:101680005E8F852D0E9483126C960FB6F894DEBF94
:101690000FBECDBFCF91DF911F910F91FF90EF90C3
:1016A000DF90CF90BF90AF909F908F907F906F9082
:1016B0005F9008958F929F92AF92BF92CF92DF92E8
:1016C000EF92FF920F931F93DF93CF93CDB7DEB7C7
:1016D00028970FB6F894DEBF0FBECDBF00E010E430
:1016E000FF248BE0882E912C5E010894A11CB11C74
:1016F0002FC08F2D90E0889DF001899DF00D989D61
:10170000F00D1124E05AF64FC080D180A281B38140
:1017100044815581668177818185282F30E02F7043
:10172000307038872F83808587FD03C0316038870C
:101730002F835E834D83BC83AB83DA82C982C80169
:1017400068E0A50121E00E94F580F394085F1F4F37
:101750008091200CF81668F20E94C06B2FEF3FEFCB
:101760003A832983FC01858596859C838B83C801F8
:1017700068E0AE014F5F5F4F21E00E94F5800E945C
:10178000123EFC01085F1F4F1093FD050093FC05FE
:1017900042A153A1848D4115510531F080FD02C055
:1017A00021E009C023E007C04081518180FD02C0D3
:1017B00020E001C022E060E070E080E090E00E9464
:1017C000718910E0812F6BE040E050E00E94E36FF0
:1017D0001F5F1034B9F710E00E94C1778823E1F34E
:1017E0001F5F1630C9F76FEF7FEF8FEF9FEF4FEF5F
:1017F0005FEF20E00E947189E090FC05F090FD050C
:101800001092FD051092FC0507E61DE0C70168E097
:10181000A80121E00E94F58088E090E0E80EF91E22
:10182000085F1F4F9EE00736190781F728960FB60D
:10183000F894DEBF0FBECDBFCF91DF911F910F9106
:10184000FF90EF90DF90CF90BF90AF909F908F90E0
:101850000895EEEFF5E08FEF9FEF91838083379649
:1018600026E0EE3DF207C9F708950F931F938C0110
:1018700087E69DE0B8010E949691482F9801220FBB
:10188000331F442311F02F5F3F4FEEEFF5E08081CF
:1018900091818217930749F4868180FF0CC044230D
:1018A00011F487E40DC082E50BC086E0E73DF80740
:1018B00011F03796ECCF442311F487E601C082E79C
:1018C0001F910F9108950F931F932FE0803F920770
:1018D00018F02FEF3FEF24C09C013695279543E089
:1018E0002D3F3407D8F4890116950795169507956D
:1018F00026E0969587952A95E1F78452904F0E94AD
:101900000CAC90E00770107002C0959587950A9511
:10191000E2F780FD03C021E030E002C023E030E0C8
:10192000C9011F910F910895EF92FF920F931F939A
:10193000CF93DF937B012FE0803F920708F03DC0FB
:101940006330710519F061307105B9F59C01369568
:10195000279543E02D3F340780F5890116950795BB
:1019600016950795EC0156E0D695C7955A95E1F77F
:10197000C452D04FCE010E940CAC482F9801277062
:10198000307083E0E816F10451F481E090E002C089
:10199000880F991F2A95E2F7642F682B0AC081E00F
:1019A00090E002C0880F991F2A95E2F7682F609592
:1019B0006423A895CE010E941EACDF91CF911F91A8
:1019C0000F91FF90EF9008951F93CF93DF930397AC
:1019D00011F010E001C01FEFCCEDDFE0A895CE01C3
:1019E000612F0E941EAC21968FE0CC3FD807B1F743
:1019F000DF91CF911F910895CF93DF93EC01662380
:101A000031F087E69DE0BE010E946B9105C087E63C
:101A10009DE0BE010E948091CC0FCD2FCC1FDD0B2D
:101A2000D19581E090E002C0880F991FCA95E2F736
:101A30002091DE063091DF06282B392B3093DF060C
:101A40002093DE0688EB9BE09093E1068093E0060E
:101A5000DF91CF9108951F93CF93DF93EC01162F61
:101A60008FE0C03FD80708F587E69DE0BE010E94E1
:101A70009691181761F0CE01612F0E94FC8CCE0167
:101A800060E00E948F90CE0161E00E948F900E94E2
:101A9000C06BFC01858596858C179D0730F4C07F4F
:101AA0002F96D687C5870E942C6EDF91CF911F910C
:101AB0000895DF92EF92FF920F931F93DF93CF93DE
:101AC00000D000D000D0CDB7DEB78C01D62E009765
:101AD00009F462C0FC01E080F1806623F9F0C701DF
:101AE00061E00E94D530882309F456C08091C50773
:101AF0009091C607A091C707B091C807F8018283EB
:101B00009383A483B5838681816086836E2D617003
:101B1000C701969587950E94FC8C0BC0C70160E0B9
:101B20000E94D5308823C1F18FEF9FEFF801918398
:101B30008083F801868183FF06C0C701969587954B
:101B400060E00E948F90F801868184FF06C0C70183
:101B50009695879561E00E948F908E2D8F7789836F
:101B6000C701880F892F881F990B91958F778A83DA
:101B70008F2D82958695869583708B831C82DD20C0
:101B800011F081E08C838FEF63E2AE014F5F5F4F16
:101B90000E94E36F81E001C080E026960FB6F894C2
:101BA000DEBF0FBECDBFCF91DF911F910F91FF9090
:101BB000EF90DF9008956F927F928F929F92AF92F5
:101BC000BF92CF92DF92EF92FF920F931F93CF932A
:101BD000DF930E942A23882309F4E8C00E94C06B87
:101BE0008C01FC01638570E080E090E022E330E04E
:101BF00040E050E00E945BA73B014C01F801648586
:101C000070E080E090E024E630E040E050E00E94A8
